Component: ARM Compiler 5.06 update 6 (build 750) Tool: armlink [4d35ed]

==============================================================================

Section Cross References

    mbed/TARGET_NUCLEO_F070RB/TOOLCHAIN_ARM_STD/analogin_api.o(i.adc_read) refers to mbed/TARGET_NUCLEO_F070RB/TOOLCHAIN_ARM_STD/stm32f0xx_hal_adc.o(i.HAL_ADC_ConfigChannel) for HAL_ADC_ConfigChannel
    mbed/TARGET_NUCLEO_F070RB/TOOLCHAIN_ARM_STD/analogin_api.o(i.adc_read) refers to mbed/TARGET_NUCLEO_F070RB/TOOLCHAIN_ARM_STD/stm32f0xx_hal_adc.o(i.HAL_ADC_Start) for HAL_ADC_Start
    mbed/TARGET_NUCLEO_F070RB/TOOLCHAIN_ARM_STD/analogin_api.o(i.adc_read) refers to mbed/TARGET_NUCLEO_F070RB/TOOLCHAIN_ARM_STD/stm32f0xx_hal_adc.o(i.HAL_ADC_PollForConversion) for HAL_ADC_PollForConversion
    mbed/TARGET_NUCLEO_F070RB/TOOLCHAIN_ARM_STD/analogin_api.o(i.adc_read) refers to mbed/TARGET_NUCLEO_F070RB/TOOLCHAIN_ARM_STD/stm32f0xx_hal_adc.o(i.HAL_ADC_GetValue) for HAL_ADC_GetValue
    mbed/TARGET_NUCLEO_F070RB/TOOLCHAIN_ARM_STD/analogin_api.o(i.adc_read) refers to mbed/TARGET_NUCLEO_F070RB/TOOLCHAIN_ARM_STD/analogin_api.o(.bss) for .bss
    mbed/TARGET_NUCLEO_F070RB/TOOLCHAIN_ARM_STD/analogin_api.o(i.analogin_init) refers to mbed/TARGET_NUCLEO_F070RB/TOOLCHAIN_ARM_STD/mbed.ar(mbed_pinmap_common.o)(i.pinmap_peripheral) for pinmap_peripheral
    mbed/TARGET_NUCLEO_F070RB/TOOLCHAIN_ARM_STD/analogin_api.o(i.analogin_init) refers to mbed/TARGET_NUCLEO_F070RB/TOOLCHAIN_ARM_STD/mbed.ar(mbed_assert.o)(i.mbed_assert_internal) for mbed_assert_internal
    mbed/TARGET_NUCLEO_F070RB/TOOLCHAIN_ARM_STD/analogin_api.o(i.analogin_init) refers to mbed/TARGET_NUCLEO_F070RB/TOOLCHAIN_ARM_STD/mbed.ar(mbed_pinmap_common.o)(i.pinmap_function) for pinmap_function
    mbed/TARGET_NUCLEO_F070RB/TOOLCHAIN_ARM_STD/analogin_api.o(i.analogin_init) refers to mbed/TARGET_NUCLEO_F070RB/TOOLCHAIN_ARM_STD/mbed.ar(mbed_pinmap_common.o)(i.pinmap_pinout) for pinmap_pinout
    mbed/TARGET_NUCLEO_F070RB/TOOLCHAIN_ARM_STD/analogin_api.o(i.analogin_init) refers to mbed/TARGET_NUCLEO_F070RB/TOOLCHAIN_ARM_STD/stm32f0xx_hal_adc.o(i.HAL_ADC_Init) for HAL_ADC_Init
    mbed/TARGET_NUCLEO_F070RB/TOOLCHAIN_ARM_STD/analogin_api.o(i.analogin_init) refers to mbed/TARGET_NUCLEO_F070RB/TOOLCHAIN_ARM_STD/mbed.ar(mbed_error.o)(i.error) for error
    mbed/TARGET_NUCLEO_F070RB/TOOLCHAIN_ARM_STD/analogin_api.o(i.analogin_init) refers to mbed/TARGET_NUCLEO_F070RB/TOOLCHAIN_ARM_STD/stm32f0xx_hal_adc_ex.o(i.HAL_ADCEx_Calibration_Start) for HAL_ADCEx_Calibration_Start
    mbed/TARGET_NUCLEO_F070RB/TOOLCHAIN_ARM_STD/analogin_api.o(i.analogin_init) refers to mbed/TARGET_NUCLEO_F070RB/TOOLCHAIN_ARM_STD/PeripheralPins.o(.constdata) for PinMap_ADC
    mbed/TARGET_NUCLEO_F070RB/TOOLCHAIN_ARM_STD/analogin_api.o(i.analogin_init) refers to mbed/TARGET_NUCLEO_F070RB/TOOLCHAIN_ARM_STD/analogin_api.o(.conststring) for .conststring
    mbed/TARGET_NUCLEO_F070RB/TOOLCHAIN_ARM_STD/analogin_api.o(i.analogin_init) refers to mbed/TARGET_NUCLEO_F070RB/TOOLCHAIN_ARM_STD/analogin_api.o(.data) for .data
    mbed/TARGET_NUCLEO_F070RB/TOOLCHAIN_ARM_STD/analogin_api.o(i.analogin_init) refers to mbed/TARGET_NUCLEO_F070RB/TOOLCHAIN_ARM_STD/analogin_api.o(.bss) for .bss
    mbed/TARGET_NUCLEO_F070RB/TOOLCHAIN_ARM_STD/analogin_api.o(i.analogin_read) refers to mbed/TARGET_NUCLEO_F070RB/TOOLCHAIN_ARM_STD/analogin_api.o(i.adc_read) for adc_read
    mbed/TARGET_NUCLEO_F070RB/TOOLCHAIN_ARM_STD/analogin_api.o(i.analogin_read) refers to C:\Keil_v5\ARM\ARMCC\Bin\..\lib\armlib\fz_ps.l(fflti.o)(.text) for __aeabi_ui2f
==============================================================================

Removing Unused input sections from the image.

    Removing mbed/TARGET_NUCLEO_F070RB/TOOLCHAIN_ARM_STD/analogin_api.o(.rev16_text), (4 bytes).
    Removing mbed/TARGET_NUCLEO_F070RB/TOOLCHAIN_ARM_STD/analogin_api.o(.revsh_text), (4 bytes).
    Removing mbed/TARGET_NUCLEO_F070RB/TOOLCHAIN_ARM_STD/analogin_api.o(i.adc_read), (184 bytes).
    Removing mbed/TARGET_NUCLEO_F070RB/TOOLCHAIN_ARM_STD/analogin_api.o(i.analogin_init), (316 bytes).
    Removing mbed/TARGET_NUCLEO_F070RB/TOOLCHAIN_ARM_STD/analogin_api.o(i.analogin_read), (24 bytes).
    Removing mbed/TARGET_NUCLEO_F070RB/TOOLCHAIN_ARM_STD/analogin_api.o(i.analogin_read_u16), (18 bytes).
    Removing mbed/TARGET_NUCLEO_F070RB/TOOLCHAIN_ARM_STD/analogin_api.o(.bss), (76 bytes).
    Removing mbed/TARGET_NUCLEO_F070RB/TOOLCHAIN_ARM_STD/analogin_api.o(.conststring), (91 bytes).
    Removing mbed/TARGET_NUCLEO_F070RB/TOOLCHAIN_ARM_STD/analogin_api.o(.data), (4 bytes).
    Removing mbed/TARGET_NUCLEO_F070RB/TOOLCHAIN_ARM_STD/analogout_api.o(.rev16_text), (4 bytes).
    Removing mbed/TARGET_NUCLEO_F070RB/TOOLCHAIN_ARM_STD/analogout_api.o(.revsh_text), (4 bytes).
    Removing mbed/TARGET_NUCLEO_F070RB/TOOLCHAIN_ARM_STD/can_api.o(.rev16_text), (4 bytes).
    Removing mbed/TARGET_NUCLEO_F070RB/TOOLCHAIN_ARM_STD/can_api.o(.revsh_text), (4 bytes).
    Removing mbed/TARGET_NUCLEO_F070RB/TOOLCHAIN_ARM_STD/cmsis_nvic.o(.rev16_text), (4 bytes).
    Removing mbed/TARGET_NUCLEO_F070RB/TOOLCHAIN_ARM_STD/cmsis_nvic.o(.revsh_text), (4 bytes).
    Removing mbed/TARGET_NUCLEO_F070RB/TOOLCHAIN_ARM_STD/cmsis_nvic.o(i.NVIC_GetVector), (12 bytes).
    Removing mbed/TARGET_NUCLEO_F070RB/TOOLCHAIN_ARM_STD/gpio_api.o(.rev16_text), (4 bytes).
    Removing mbed/TARGET_NUCLEO_F070RB/TOOLCHAIN_ARM_STD/gpio_api.o(.revsh_text), (4 bytes).
==============================================================================

Image Symbol Table

    Local Symbols

    Symbol Name                              Value     Ov Type        Size  Object(Section)

    ../../../clib/unwind_pr.c                0x00000000   Number         0  C:\Keil_v5\ARM\ARMCC\Bin\..\lib\cpplib\cpprt_p.l(unwind_prcommon.o) ABSOLUTE
    ../../../clib/unwind_pr.c                0x00000000   Number         0  C:\Keil_v5\ARM\ARMCC\Bin\..\lib\cpplib\cpprt_p.l(unwind_pr0.o) ABSOLUTE
    ../../../clib/unwinder.c                 0x00000000   Number         0  C:\Keil_v5\ARM\ARMCC\Bin\..\lib\cpplib\cpprt_p.l(unwind_activity.o) ABSOLUTE
    ../../../clib/unwinder.c                 0x00000000   Number         0  C:\Keil_v5\ARM\ARMCC\Bin\..\lib\cpplib\cpprt_p.l(unwind_activity.o) ABSOLUTE
    ../../../clib/unwinder.c                 0x00000000   Number         0  C:\Keil_v5\ARM\ARMCC\Bin\..\lib\cpplib\cpprt_p.l(unwinder.o) ABSOLUTE
    ../../../clib/unwinder.c                 0x00000000   Number         0  C:\Keil_v5\ARM\ARMCC\Bin\..\lib\cpplib\cpprt_p.l(unwinder.o) ABSOLUTE
    ../../../edgfe/lib_src/arm_exceptions.c  0x00000000   Number         0  C:\Keil_v5\ARM\ARMCC\Bin\..\lib\cpplib\cpprt_p.l(arm_exceptions_mem.o) ABSOLUTE
    ../../../edgfe/lib_src/arm_exceptions.c  0x00000000   Number         0  C:\Keil_v5\ARM\ARMCC\Bin\..\lib\cpplib\cpprt_p.l(arm_exceptions_terminate.o) ABSOLUTE
    ../../../edgfe/lib_src/arm_exceptions.c  0x00000000   Number         0  C:\Keil_v5\ARM\ARMCC\Bin\..\lib\cpplib\cpprt_p.l(arm_exceptions_support.o) ABSOLUTE
    ../../../edgfe/lib_src/arm_exceptions.c  0x00000000   Number         0  C:\Keil_v5\ARM\ARMCC\Bin\..\lib\cpplib\cpprt_p.l(arm_exceptions_callterm.o) ABSOLUTE
    ../../../edgfe/lib_src/arm_exceptions.c  0x00000000   Number         0  C:\Keil_v5\ARM\ARMCC\Bin\..\lib\cpplib\cpprt_p.l(arm_exceptions_globs.o) ABSOLUTE
    ../../../edgfe/lib_src/arm_noexceptions.c 0x00000000   Number         0  C:\Keil_v5\ARM\ARMCC\Bin\..\lib\cpplib\cpprt_p.l(arm_begincatch_noexceptions.o) ABSOLUTE
    ../../../edgfe/lib_src/pure_virt.c       0x00000000   Number         0  C:\Keil_v5\ARM\ARMCC\Bin\..\lib\cpplib\cpprt_p.l(pure_virt.o) ABSOLUTE
    ../../../edgfe/lib_src/typeinfo.c        0x00000000   Number         0  C:\Keil_v5\ARM\ARMCC\Bin\..\lib\cpplib\cpprt_p.l(lib_rtti_impl.o) ABSOLUTE
    ../../../edgfe/lib_src/typeinfo.c        0x00000000   Number         0  C:\Keil_v5\ARM\ARMCC\Bin\..\lib\cpplib\cpprt_p.l(type_info_dtor.o) ABSOLUTE
    ../../array_helpers.cpp                  0x00000000   Number         0  C:\Keil_v5\ARM\ARMCC\Bin\..\lib\cpplib\cpprt_p.l(aeabi_vec_dtor_noexceptions.o) ABSOLUTE
    ../../array_helpers.cpp                  0x00000000   Number         0  C:\Keil_v5\ARM\ARMCC\Bin\..\lib\cpplib\cpprt_p.l(aeabi_vec_ctor_nocookie_nodtor.o) ABSOLUTE
    ../clib/angel/boardlib.s                 0x00000000   Number         0  C:\Keil_v5\ARM\ARMCC\Bin\..\lib\armlib\c_p.l(boardinit3.o) ABSOLUTE
    ../clib/angel/boardlib.s                 0x00000000   Number         0  C:\Keil_v5\ARM\ARMCC\Bin\..\lib\armlib\c_p.l(boardinit1.o) ABSOLUTE
    ../clib/angel/handlers.s                 0x00000000   Number         0  C:\Keil_v5\ARM\ARMCC\Bin\..\lib\armlib\c_p.l(__scatter_copy.o) ABSOLUTE
    ../clib/angel/handlers.s                 0x00000000   Number         0  C:\Keil_v5\ARM\ARMCC\Bin\..\lib\armlib\c_p.l(__scatter_zi.o) ABSOLUTE
    ../clib/angel/kernel.s                   0x00000000   Number         0  C:\Keil_v5\ARM\ARMCC\Bin\..\lib\armlib\c_p.l(__rtentry2.o) ABSOLUTE
    ../clib/angel/kernel.s                   0x00000000   Number         0  C:\Keil_v5\ARM\ARMCC\Bin\..\lib\armlib\c_p.l(__rtentry4.o) ABSOLUTE
    ../clib/angel/kernel.s                   0x00000000   Number         0  C:\Keil_v5\ARM\ARMCC\Bin\..\lib\armlib\c_p.l(__rtentry.o) ABSOLUTE
    ../clib/angel/rt.s                       0x00000000   Number         0  C:\Keil_v5\ARM\ARMCC\Bin\..\lib\armlib\c_p.l(rt_ctype_table.o) ABSOLUTE
    ../clib/angel/rt.s                       0x00000000   Number         0  C:\Keil_v5\ARM\ARMCC\Bin\..\lib\armlib\c_p.l(rt_locale.o) ABSOLUTE
    ../clib/angel/rt.s                       0x00000000   Number         0  C:\Keil_v5\ARM\ARMCC\Bin\..\lib\armlib\c_p.l(rt_heap_descriptor_intlibspace.o) ABSOLUTE
    ../clib/angel/rt.s                       0x00000000   Number         0  C:\Keil_v5\ARM\ARMCC\Bin\..\lib\armlib\c_p.l(rt_locale_intlibspace.o) ABSOLUTE
    ../clib/angel/rt.s                       0x00000000   Number         0  C:\Keil_v5\ARM\ARMCC\Bin\..\lib\armlib\c_p.l(rt_raise.o) ABSOLUTE
    ../clib/angel/rt.s                       0x00000000   Number         0  C:\Keil_v5\ARM\ARMCC\Bin\..\lib\armlib\c_p.l(rt_div0.o) ABSOLUTE
    ../clib/angel/rt.s                       0x00000000   Number         0  C:\Keil_v5\ARM\ARMCC\Bin\..\lib\armlib\c_p.l(aeabi_idiv0_sigfpe.o) ABSOLUTE
    ../clib/angel/rt.s                       0x00000000   Number         0  C:\Keil_v5\ARM\ARMCC\Bin\..\lib\armlib\c_p.l(rt_eh_globals_addr_intlibspace.o) ABSOLUTE
    ../clib/angel/rt.s                       0x00000000   Number         0  C:\Keil_v5\ARM\ARMCC\Bin\..\lib\armlib\c_p.l(rt_errno_addr.o) ABSOLUTE
    ../clib/angel/rt.s                       0x00000000   Number         0  C:\Keil_v5\ARM\ARMCC\Bin\..\lib\armlib\c_p.l(rt_errno_addr_intlibspace.o) ABSOLUTE
    ../clib/angel/rt.s                       0x00000000   Number         0  C:\Keil_v5\ARM\ARMCC\Bin\..\lib\armlib\c_p.l(aeabi_idiv0.o) ABSOLUTE
    ../clib/angel/rt.s                       0x00000000   Number         0  C:\Keil_v5\ARM\ARMCC\Bin\..\lib\armlib\c_p.l(rt_heap_descriptor.o) ABSOLUTE
    ../clib/angel/rt.s                       0x00000000   Number         0  C:\Keil_v5\ARM\ARMCC\Bin\..\lib\armlib\c_p.l(rt_eh_globals_addr.o) ABSOLUTE
    ../clib/angel/scatterp.s                 0x00000000   Number         0  C:\Keil_v5\ARM\ARMCC\Bin\..\lib\armlib\c_p.l(__scatter.o) ABSOLUTE
    ../clib/angel/startup.s                  0x00000000   Number         0  C:\Keil_v5\ARM\ARMCC\Bin\..\lib\armlib\c_p.l(__main.o) ABSOLUTE
    ../clib/angel/sys.s                      0x00000000   Number         0  C:\Keil_v5\ARM\ARMCC\Bin\..\lib\armlib\c_p.l(indicate_semi.o) ABSOLUTE
    ../clib/angel/sys.s                      0x00000000   Number         0  C:\Keil_v5\ARM\ARMCC\Bin\..\lib\armlib\c_p.l(libspace.o) ABSOLUTE
    ../clib/angel/sys.s                      0x00000000   Number         0  C:\Keil_v5\ARM\ARMCC\Bin\..\lib\armlib\c_p.l(use_no_semi.o) ABSOLUTE
    ../clib/angel/sys.s                      0x00000000   Number         0  C:\Keil_v5\ARM\ARMCC\Bin\..\lib\armlib\c_p.l(mutex_dummy.o) ABSOLUTE
    ../clib/angel/sysapp.c                   0x00000000   Number         0  C:\Keil_v5\ARM\ARMCC\Bin\..\lib\armlib\c_p.l(sys_exit.o) ABSOLUTE
    ../clib/angel/sysapp.c                   0x00000000   Number         0  C:\Keil_v5\ARM\ARMCC\Bin\..\lib\armlib\c_p.l(sys_wrch.o) ABSOLUTE
    ../clib/arm_runtime.c                    0x00000000   Number         0  C:\Keil_v5\ARM\ARMCC\Bin\..\lib\armlib\c_p.l(init_aeabi.o) ABSOLUTE
    ../clib/arm_runtime.c                    0x00000000   Number         0  C:\Keil_v5\ARM\ARMCC\Bin\..\lib\armlib\c_p.l(init_aeabi.o) ABSOLUTE
    ../clib/armsys.c                         0x00000000   Number         0  C:\Keil_v5\ARM\ARMCC\Bin\..\lib\armlib\c_p.l(no_argv.o) ABSOLUTE
    ../clib/armsys.c                         0x00000000   Number         0  C:\Keil_v5\ARM\ARMCC\Bin\..\lib\armlib\c_p.l(_get_argv_nomalloc.o) ABSOLUTE
    ../clib/armsys.c                         0x00000000   Number         0  C:\Keil_v5\ARM\ARMCC\Bin\..\lib\armlib\c_p.l(argv_veneer.o) ABSOLUTE
    ../clib/armsys.c                         0x00000000   Number         0  C:\Keil_v5\ARM\ARMCC\Bin\..\lib\armlib\c_p.l(_get_argv.o) ABSOLUTE
    ../clib/assert.c                         0x00000000   Number         0  C:\Keil_v5\ARM\ARMCC\Bin\..\lib\armlib\c_p.l(assert_stdio.o) ABSOLUTE
    ../clib/bigflt.c                         0x00000000   Number         0  C:\Keil_v5\ARM\ARMCC\Bin\..\lib\armlib\c_p.l(bigflt0.o) ABSOLUTE
    ../clib/btod.c                           0x00000000   Number         0  C:\Keil_v5\ARM\ARMCC\Bin\..\lib\armlib\c_p.l(btod.o) ABSOLUTE
    ../clib/ctype.c                          0x00000000   Number         0  C:\Keil_v5\ARM\ARMCC\Bin\..\lib\armlib\c_p.l(isspace.o) ABSOLUTE
    ../clib/division.c                       0x00000000   Number         0  C:\Keil_v5\ARM\ARMCC\Bin\..\lib\armlib\c_p.l(lludiv10.o) ABSOLUTE
    ../clib/division.c                       0x00000000   Number         0  C:\Keil_v5\ARM\ARMCC\Bin\..\lib\armlib\c_p.l(rtudiv10.o) ABSOLUTE
    ../clib/division.s                       0x00000000   Number         0  C:\Keil_v5\ARM\ARMCC\Bin\..\lib\armlib\c_p.l(aeabi_sdivfast.o) ABSOLUTE
    ../clib/division.s                       0x00000000   Number         0  C:\Keil_v5\ARM\ARMCC\Bin\..\lib\armlib\c_p.l(aeabi_sdivfast_div0.o) ABSOLUTE
    ../clib/fenv.c                           0x00000000   Number         0  C:\Keil_v5\ARM\ARMCC\Bin\..\lib\armlib\c_p.l(_rserrno.o) ABSOLUTE
    ../clib/heap1.c                          0x00000000   Number         0  C:\Keil_v5\ARM\ARMCC\Bin\..\lib\armlib\c_p.l(h1_init_mt.o) ABSOLUTE
    ../clib/heap1.c                          0x00000000   Number         0  C:\Keil_v5\ARM\ARMCC\Bin\..\lib\armlib\c_p.l(h1_free_mt.o) ABSOLUTE
    ../clib/heap1.c                          0x00000000   Number         0  C:\Keil_v5\ARM\ARMCC\Bin\..\lib\armlib\c_p.l(h1_alloc_mt.o) ABSOLUTE
    ../clib/heap1.c                          0x00000000   Number         0  C:\Keil_v5\ARM\ARMCC\Bin\..\lib\armlib\c_p.l(h1_free.o) ABSOLUTE
    ../clib/heap1.c                          0x00000000   Number         0  C:\Keil_v5\ARM\ARMCC\Bin\..\lib\armlib\c_p.l(h1_alloc.o) ABSOLUTE
    ../clib/heap1.c                          0x00000000   Number         0  C:\Keil_v5\ARM\ARMCC\Bin\..\lib\armlib\c_p.l(h1_extend.o) ABSOLUTE
    ../clib/heap1.c                          0x00000000   Number         0  C:\Keil_v5\ARM\ARMCC\Bin\..\lib\armlib\c_p.l(h1_extend_mt.o) ABSOLUTE
    ../clib/heap1.c                          0x00000000   Number         0  C:\Keil_v5\ARM\ARMCC\Bin\..\lib\armlib\c_p.l(h1_final_mt.o) ABSOLUTE
    ../clib/heap1.c                          0x00000000   Number         0  C:\Keil_v5\ARM\ARMCC\Bin\..\lib\armlib\c_p.l(h1_final.o) ABSOLUTE
    ../clib/heap1.c                          0x00000000   Number         0  C:\Keil_v5\ARM\ARMCC\Bin\..\lib\armlib\c_p.l(h1_init.o) ABSOLUTE
    ../clib/heap2.c                          0x00000000   Number         0  C:\Keil_v5\ARM\ARMCC\Bin\..\lib\armlib\c_p.l(heap2mt.o) ABSOLUTE
    ../clib/heap2.c                          0x00000000   Number         0  C:\Keil_v5\ARM\ARMCC\Bin\..\lib\armlib\c_p.l(heap2.o) ABSOLUTE
    ../clib/heap2.c                          0x00000000   Number         0  C:\Keil_v5\ARM\ARMCC\Bin\..\lib\armlib\c_p.l(fdtree.o) ABSOLUTE
    ../clib/heapalloc.c                      0x00000000   Number         0  C:\Keil_v5\ARM\ARMCC\Bin\..\lib\armlib\c_p.l(free.o) ABSOLUTE
    ../clib/heapalloc.c                      0x00000000   Number         0  C:\Keil_v5\ARM\ARMCC\Bin\..\lib\armlib\c_p.l(malloc.o) ABSOLUTE
    ../clib/heapalloc.c                      0x00000000   Number         0  C:\Keil_v5\ARM\ARMCC\Bin\..\lib\armlib\c_p.l(maybetermalloc2.o) ABSOLUTE
    ../clib/heapalloc.c                      0x00000000   Number         0  C:\Keil_v5\ARM\ARMCC\Bin\..\lib\armlib\c_p.l(maybetermalloc2.o) ABSOLUTE
    ../clib/heapalloc.c                      0x00000000   Number         0  C:\Keil_v5\ARM\ARMCC\Bin\..\lib\armlib\c_p.l(maybetermalloc1.o) ABSOLUTE
    ../clib/heapalloc.c                      0x00000000   Number         0  C:\Keil_v5\ARM\ARMCC\Bin\..\lib\armlib\c_p.l(hrguard.o) ABSOLUTE
    ../clib/heapalloc.c                      0x00000000   Number         0  C:\Keil_v5\ARM\ARMCC\Bin\..\lib\armlib\c_p.l(heapstubs.o) ABSOLUTE
    ../clib/heapalloc.c                      0x00000000   Number         0  C:\Keil_v5\ARM\ARMCC\Bin\..\lib\armlib\c_p.l(init_alloc.o) ABSOLUTE
    ../clib/heapalloc.c                      0x00000000   Number         0  C:\Keil_v5\ARM\ARMCC\Bin\..\lib\armlib\c_p.l(hguard.o) ABSOLUTE
    ../clib/heapalloc.c                      0x00000000   Number         0  C:\Keil_v5\ARM\ARMCC\Bin\..\lib\armlib\c_p.l(term_alloc.o) ABSOLUTE
    ../clib/heapalloc.c                      0x00000000   Number         0  C:\Keil_v5\ARM\ARMCC\Bin\..\lib\armlib\c_p.l(maybetermalloc1.o) ABSOLUTE
    ../clib/heapaux.c                        0x00000000   Number         0  C:\Keil_v5\ARM\ARMCC\Bin\..\lib\armlib\c_p.l(heapauxi.o) ABSOLUTE
    ../clib/heapaux.c                        0x00000000   Number         0  C:\Keil_v5\ARM\ARMCC\Bin\..\lib\armlib\c_p.l(heapauxa.o) ABSOLUTE
    ../clib/libinit.s                        0x00000000   Number         0  C:\Keil_v5\ARM\ARMCC\Bin\..\lib\armlib\c_p.l(libinit2.o) ABSOLUTE
    ../clib/libinit.s                        0x00000000   Number         0  C:\Keil_v5\ARM\ARMCC\Bin\..\lib\armlib\c_p.l(libshutdown2.o) ABSOLUTE
    ../clib/libinit.s                        0x00000000   Number         0  C:\Keil_v5\ARM\ARMCC\Bin\..\lib\armlib\c_p.l(libinit.o) ABSOLUTE
    ../clib/locale.c                         0x00000000   Number         0  C:\Keil_v5\ARM\ARMCC\Bin\..\lib\armlib\c_p.l(_mbrtowc.o) ABSOLUTE
    ../clib/locale.c                         0x00000000   Number         0  C:\Keil_v5\ARM\ARMCC\Bin\..\lib\armlib\c_p.l(_wcrtomb.o) ABSOLUTE
    ../clib/locale.s                         0x00000000   Number         0  C:\Keil_v5\ARM\ARMCC\Bin\..\lib\armlib\c_p.l(lc_ctype_c.o) ABSOLUTE
    ../clib/locale.s                         0x00000000   Number         0  C:\Keil_v5\ARM\ARMCC\Bin\..\lib\armlib\c_p.l(lc_numeric_c.o) ABSOLUTE
    ../clib/longlong.c                       0x00000000   Number         0  C:\Keil_v5\ARM\ARMCC\Bin\..\lib\armlib\c_p.l(llmul.o) ABSOLUTE
    ../clib/longlong.c                       0x00000000   Number         0  C:\Keil_v5\ARM\ARMCC\Bin\..\lib\armlib\c_p.l(llushr.o) ABSOLUTE
    ../clib/longlong.c                       0x00000000   Number         0  C:\Keil_v5\ARM\ARMCC\Bin\..\lib\armlib\c_p.l(llshl.o) ABSOLUTE
    ../clib/memcpset.c                       0x00000000   Number         0  C:\Keil_v5\ARM\ARMCC\Bin\..\lib\armlib\c_p.l(rt_memclr.o) ABSOLUTE
    ../clib/memcpset.c                       0x00000000   Number         0  C:\Keil_v5\ARM\ARMCC\Bin\..\lib\armlib\c_p.l(rt_memcpy.o) ABSOLUTE
    ../clib/memcpset.c                       0x00000000   Number         0  C:\Keil_v5\ARM\ARMCC\Bin\..\lib\armlib\c_p.l(rt_memcpy.o) ABSOLUTE
    ../clib/memcpset.c                       0x00000000   Number         0  C:\Keil_v5\ARM\ARMCC\Bin\..\lib\armlib\c_p.l(aeabi_memset.o) ABSOLUTE
    ../clib/memcpset.s                       0x00000000   Number         0  C:\Keil_v5\ARM\ARMCC\Bin\..\lib\armlib\c_p.l(strcmpv6m.o) ABSOLUTE
    ../clib/misc.s                           0x00000000   Number         0  C:\Keil_v5\ARM\ARMCC\Bin\..\lib\armlib\c_p.l(printf_stubs.o) ABSOLUTE
    ../clib/printf.c                         0x00000000   Number         0  C:\Keil_v5\ARM\ARMCC\Bin\..\lib\armlib\c_p.l(__printf_nopercent.o) ABSOLUTE
    ../clib/printf.c                         0x00000000   Number         0  C:\Keil_v5\ARM\ARMCC\Bin\..\lib\armlib\c_p.l(_printf_fp_hex.o) ABSOLUTE
    ../clib/printf.c                         0x00000000   Number         0  C:\Keil_v5\ARM\ARMCC\Bin\..\lib\armlib\c_p.l(_printf_fp_dec.o) ABSOLUTE
    ../clib/printf.c                         0x00000000   Number         0  C:\Keil_v5\ARM\ARMCC\Bin\..\lib\armlib\c_p.l(__printf_flags.o) ABSOLUTE
    ../clib/printf.c                         0x00000000   Number         0  C:\Keil_v5\ARM\ARMCC\Bin\..\lib\armlib\c_p.l(vsprintf.o) ABSOLUTE
    ../clib/printf.c                         0x00000000   Number         0  C:\Keil_v5\ARM\ARMCC\Bin\..\lib\armlib\c_p.l(__printf_flags_ss.o) ABSOLUTE
    ../clib/printf.c                         0x00000000   Number         0  C:\Keil_v5\ARM\ARMCC\Bin\..\lib\armlib\c_p.l(_printf_hex_int_ll_ptr.o) ABSOLUTE
    ../clib/printf.c                         0x00000000   Number         0  C:\Keil_v5\ARM\ARMCC\Bin\..\lib\armlib\c_p.l(_printf_oct_int_ll.o) ABSOLUTE
    ../clib/printf.c                         0x00000000   Number         0  C:\Keil_v5\ARM\ARMCC\Bin\..\lib\armlib\c_p.l(c89vfprintf.o) ABSOLUTE
    ../clib/printf.c                         0x00000000   Number         0  C:\Keil_v5\ARM\ARMCC\Bin\..\lib\armlib\c_p.l(c89vsprintf.o) ABSOLUTE
    ../clib/printf.c                         0x00000000   Number         0  C:\Keil_v5\ARM\ARMCC\Bin\..\lib\armlib\c_p.l(__printf_wp.o) ABSOLUTE
    ../clib/printf.c                         0x00000000   Number         0  C:\Keil_v5\ARM\ARMCC\Bin\..\lib\armlib\c_p.l(c89vsnprintf.o) ABSOLUTE
    ../clib/printf.c                         0x00000000   Number         0  C:\Keil_v5\ARM\ARMCC\Bin\..\lib\armlib\c_p.l(_printf_char_common.o) ABSOLUTE
    ../clib/printf.c                         0x00000000   Number         0  C:\Keil_v5\ARM\ARMCC\Bin\..\lib\armlib\c_p.l(__printf_ss_wp.o) ABSOLUTE
    ../clib/printf.c                         0x00000000   Number         0  C:\Keil_v5\ARM\ARMCC\Bin\..\lib\armlib\c_p.l(__printf_flags_ss_wp.o) ABSOLUTE
    ../clib/printf.c                         0x00000000   Number         0  C:\Keil_v5\ARM\ARMCC\Bin\..\lib\armlib\c_p.l(_printf_truncate.o) ABSOLUTE
    ../clib/printf.c                         0x00000000   Number         0  C:\Keil_v5\ARM\ARMCC\Bin\..\lib\armlib\c_p.l(_printf_fp_infnan.o) ABSOLUTE
    ../clib/printf.c                         0x00000000   Number         0  C:\Keil_v5\ARM\ARMCC\Bin\..\lib\armlib\c_p.l(__2sprintf.o) ABSOLUTE
    ../clib/printf.c                         0x00000000   Number         0  C:\Keil_v5\ARM\ARMCC\Bin\..\lib\armlib\c_p.l(_printf_hex_int_ptr.o) ABSOLUTE
    ../clib/printf.c                         0x00000000   Number         0  C:\Keil_v5\ARM\ARMCC\Bin\..\lib\armlib\c_p.l(_printf_charcount.o) ABSOLUTE
    ../clib/printf.c                         0x00000000   Number         0  C:\Keil_v5\ARM\ARMCC\Bin\..\lib\armlib\c_p.l(_printf_dec.o) ABSOLUTE
    ../clib/printf.c                         0x00000000   Number         0  C:\Keil_v5\ARM\ARMCC\Bin\..\lib\armlib\c_p.l(_printf_intcommon.o) ABSOLUTE
    ../clib/printf.c                         0x00000000   Number         0  C:\Keil_v5\ARM\ARMCC\Bin\..\lib\armlib\c_p.l(_printf_str.o) ABSOLUTE
    ../clib/printf.c                         0x00000000   Number         0  C:\Keil_v5\ARM\ARMCC\Bin\..\lib\armlib\c_p.l(_printf_pad.o) ABSOLUTE
    ../clib/printf.c                         0x00000000   Number         0  C:\Keil_v5\ARM\ARMCC\Bin\..\lib\armlib\c_p.l(_printf_hex_int_ll.o) ABSOLUTE
    ../clib/printf.c                         0x00000000   Number         0  C:\Keil_v5\ARM\ARMCC\Bin\..\lib\armlib\c_p.l(noretval__2sprintf.o) ABSOLUTE
    ../clib/printf.c                         0x00000000   Number         0  C:\Keil_v5\ARM\ARMCC\Bin\..\lib\armlib\c_p.l(__printf.o) ABSOLUTE
    ../clib/printf.c                         0x00000000   Number         0  C:\Keil_v5\ARM\ARMCC\Bin\..\lib\armlib\c_p.l(_printf_hex_ll.o) ABSOLUTE
    ../clib/printf.c                         0x00000000   Number         0  C:\Keil_v5\ARM\ARMCC\Bin\..\lib\armlib\c_p.l(_printf_longlong_dec.o) ABSOLUTE
    ../clib/printf.c                         0x00000000   Number         0  C:\Keil_v5\ARM\ARMCC\Bin\..\lib\armlib\c_p.l(_printf_oct_ll.o) ABSOLUTE
    ../clib/printf.c                         0x00000000   Number         0  C:\Keil_v5\ARM\ARMCC\Bin\..\lib\armlib\c_p.l(_printf_wctomb.o) ABSOLUTE
    ../clib/printf.c                         0x00000000   Number         0  C:\Keil_v5\ARM\ARMCC\Bin\..\lib\armlib\c_p.l(_printf_hex_ptr.o) ABSOLUTE
    ../clib/printf.c                         0x00000000   Number         0  C:\Keil_v5\ARM\ARMCC\Bin\..\lib\armlib\c_p.l(_printf_hex_int.o) ABSOLUTE
    ../clib/printf.c                         0x00000000   Number         0  C:\Keil_v5\ARM\ARMCC\Bin\..\lib\armlib\c_p.l(_printf_char_file.o) ABSOLUTE
    ../clib/printf.c                         0x00000000   Number         0  C:\Keil_v5\ARM\ARMCC\Bin\..\lib\armlib\c_p.l(_printf_hex_ll_ptr.o) ABSOLUTE
    ../clib/printf.c                         0x00000000   Number         0  C:\Keil_v5\ARM\ARMCC\Bin\..\lib\armlib\c_p.l(__printf_flags_wp.o) ABSOLUTE
    ../clib/printf.c                         0x00000000   Number         0  C:\Keil_v5\ARM\ARMCC\Bin\..\lib\armlib\c_p.l(_snputc.o) ABSOLUTE
    ../clib/printf.c                         0x00000000   Number         0  C:\Keil_v5\ARM\ARMCC\Bin\..\lib\armlib\c_p.l(__printf_ss.o) ABSOLUTE
    ../clib/printf.c                         0x00000000   Number         0  C:\Keil_v5\ARM\ARMCC\Bin\..\lib\armlib\c_p.l(_sputc.o) ABSOLUTE
    ../clib/printf.c                         0x00000000   Number         0  C:\Keil_v5\ARM\ARMCC\Bin\..\lib\armlib\c_p.l(_printf_wchar.o) ABSOLUTE
    ../clib/printf.c                         0x00000000   Number         0  C:\Keil_v5\ARM\ARMCC\Bin\..\lib\armlib\c_p.l(_printf_char_file_locked.o) ABSOLUTE
    ../clib/printf.c                         0x00000000   Number         0  C:\Keil_v5\ARM\ARMCC\Bin\..\lib\armlib\c_p.l(_printf_char.o) ABSOLUTE
    ../clib/printf.c                         0x00000000   Number         0  C:\Keil_v5\ARM\ARMCC\Bin\..\lib\armlib\c_p.l(_printf_oct_int.o) ABSOLUTE
    ../clib/printf_percent.s                 0x00000000   Number         0  C:\Keil_v5\ARM\ARMCC\Bin\..\lib\armlib\c_p.l(_printf_lld.o) ABSOLUTE
    ../clib/printf_percent.s                 0x00000000   Number         0  C:\Keil_v5\ARM\ARMCC\Bin\..\lib\armlib\c_p.l(_printf_llu.o) ABSOLUTE
    ../clib/printf_percent.s                 0x00000000   Number         0  C:\Keil_v5\ARM\ARMCC\Bin\..\lib\armlib\c_p.l(_printf_ll.o) ABSOLUTE
    ../clib/printf_percent.s                 0x00000000   Number         0  C:\Keil_v5\ARM\ARMCC\Bin\..\lib\armlib\c_p.l(_printf_l.o) ABSOLUTE
    ../clib/printf_percent.s                 0x00000000   Number         0  C:\Keil_v5\ARM\ARMCC\Bin\..\lib\armlib\c_p.l(_printf_lc.o) ABSOLUTE
    ../clib/printf_percent.s                 0x00000000   Number         0  C:\Keil_v5\ARM\ARMCC\Bin\..\lib\armlib\c_p.l(_printf_ls.o) ABSOLUTE
    ../clib/printf_percent.s                 0x00000000   Number         0  C:\Keil_v5\ARM\ARMCC\Bin\..\lib\armlib\c_p.l(_printf_llo.o) ABSOLUTE
    ../clib/printf_percent.s                 0x00000000   Number         0  C:\Keil_v5\ARM\ARMCC\Bin\..\lib\armlib\c_p.l(_printf_llx.o) ABSOLUTE
    ../clib/printf_percent.s                 0x00000000   Number         0  C:\Keil_v5\ARM\ARMCC\Bin\..\lib\armlib\c_p.l(_printf_p.o) ABSOLUTE
    ../clib/printf_percent.s                 0x00000000   Number         0  C:\Keil_v5\ARM\ARMCC\Bin\..\lib\armlib\c_p.l(_printf_s.o) ABSOLUTE
    ../clib/printf_percent.s                 0x00000000   Number         0  C:\Keil_v5\ARM\ARMCC\Bin\..\lib\armlib\c_p.l(_printf_percent.o) ABSOLUTE
    ../clib/printf_percent.s                 0x00000000   Number         0  C:\Keil_v5\ARM\ARMCC\Bin\..\lib\armlib\c_p.l(_printf_lli.o) ABSOLUTE
    ../clib/printf_percent.s                 0x00000000   Number         0  C:\Keil_v5\ARM\ARMCC\Bin\..\lib\armlib\c_p.l(_printf_c.o) ABSOLUTE
    ../clib/printf_percent.s                 0x00000000   Number         0  C:\Keil_v5\ARM\ARMCC\Bin\..\lib\armlib\c_p.l(_printf_n.o) ABSOLUTE
    ../clib/printf_percent.s                 0x00000000   Number         0  C:\Keil_v5\ARM\ARMCC\Bin\..\lib\armlib\c_p.l(_printf_x.o) ABSOLUTE
    ../clib/printf_percent.s                 0x00000000   Number         0  C:\Keil_v5\ARM\ARMCC\Bin\..\lib\armlib\c_p.l(_printf_o.o) ABSOLUTE
    ../clib/printf_percent.s                 0x00000000   Number         0  C:\Keil_v5\ARM\ARMCC\Bin\..\lib\armlib\c_p.l(_printf_i.o) ABSOLUTE
    ../clib/printf_percent.s                 0x00000000   Number         0  C:\Keil_v5\ARM\ARMCC\Bin\..\lib\armlib\c_p.l(_printf_d.o) ABSOLUTE
    ../clib/printf_percent.s                 0x00000000   Number         0  C:\Keil_v5\ARM\ARMCC\Bin\..\lib\armlib\c_p.l(_printf_u.o) ABSOLUTE
    ../clib/printf_percent.s                 0x00000000   Number         0  C:\Keil_v5\ARM\ARMCC\Bin\..\lib\armlib\c_p.l(_printf_f.o) ABSOLUTE
    ../clib/printf_percent.s                 0x00000000   Number         0  C:\Keil_v5\ARM\ARMCC\Bin\..\lib\armlib\c_p.l(_printf_e.o) ABSOLUTE
    ../clib/printf_percent.s                 0x00000000   Number         0  C:\Keil_v5\ARM\ARMCC\Bin\..\lib\armlib\c_p.l(_printf_g.o) ABSOLUTE
    ../clib/printf_percent.s                 0x00000000   Number         0  C:\Keil_v5\ARM\ARMCC\Bin\..\lib\armlib\c_p.l(_printf_a.o) ABSOLUTE
    ../clib/printf_percent.s                 0x00000000   Number         0  C:\Keil_v5\ARM\ARMCC\Bin\..\lib\armlib\c_p.l(_printf_percent_end.o) ABSOLUTE
    ../clib/scanf.c                          0x00000000   Number         0  C:\Keil_v5\ARM\ARMCC\Bin\..\lib\armlib\c_p.l(scanf_fp.o) ABSOLUTE
    ../clib/scanf.c                          0x00000000   Number         0  C:\Keil_v5\ARM\ARMCC\Bin\..\lib\armlib\c_p.l(__0sscanf.o) ABSOLUTE
    ../clib/scanf.c                          0x00000000   Number         0  C:\Keil_v5\ARM\ARMCC\Bin\..\lib\armlib\c_p.l(scanf_char_file.o) ABSOLUTE
    ../clib/scanf.c                          0x00000000   Number         0  C:\Keil_v5\ARM\ARMCC\Bin\..\lib\armlib\c_p.l(_sgetc.o) ABSOLUTE
    ../clib/scanf.c                          0x00000000   Number         0  C:\Keil_v5\ARM\ARMCC\Bin\..\lib\armlib\c_p.l(scanf_infnan.o) ABSOLUTE
    ../clib/scanf.c                          0x00000000   Number         0  C:\Keil_v5\ARM\ARMCC\Bin\..\lib\armlib\c_p.l(_scanf_wstr.o) ABSOLUTE
    ../clib/scanf.c                          0x00000000   Number         0  C:\Keil_v5\ARM\ARMCC\Bin\..\lib\armlib\c_p.l(scanf_char.o) ABSOLUTE
    ../clib/scanf.c                          0x00000000   Number         0  C:\Keil_v5\ARM\ARMCC\Bin\..\lib\armlib\c_p.l(_scanf_wctomb.o) ABSOLUTE
    ../clib/scanf.c                          0x00000000   Number         0  C:\Keil_v5\ARM\ARMCC\Bin\..\lib\armlib\c_p.l(_scanf_str.o) ABSOLUTE
    ../clib/scanf.c                          0x00000000   Number         0  C:\Keil_v5\ARM\ARMCC\Bin\..\lib\armlib\c_p.l(scanf_hexfp.o) ABSOLUTE
    ../clib/scanf.c                          0x00000000   Number         0  C:\Keil_v5\ARM\ARMCC\Bin\..\lib\armlib\c_p.l(_scanf_int.o) ABSOLUTE
    ../clib/scanf.c                          0x00000000   Number         0  C:\Keil_v5\ARM\ARMCC\Bin\..\lib\armlib\c_p.l(_scanf_longlong.o) ABSOLUTE
    ../clib/scanf.c                          0x00000000   Number         0  C:\Keil_v5\ARM\ARMCC\Bin\..\lib\armlib\c_p.l(vfscanf.o) ABSOLUTE
    ../clib/scanf.c                          0x00000000   Number         0  C:\Keil_v5\ARM\ARMCC\Bin\..\lib\armlib\c_p.l(_scanf_mbtowc.o) ABSOLUTE
    ../clib/scanf.c                          0x00000000   Number         0  C:\Keil_v5\ARM\ARMCC\Bin\..\lib\armlib\c_p.l(_scanf.o) ABSOLUTE
    ../clib/scanf.c                          0x00000000   Number         0  C:\Keil_v5\ARM\ARMCC\Bin\..\lib\armlib\c_p.l(scanf_char_file_locked.o) ABSOLUTE
    ../clib/scanf.c                          0x00000000   Number         0  C:\Keil_v5\ARM\ARMCC\Bin\..\lib\armlib\c_p.l(_scanf_wcharmap.o) ABSOLUTE
    ../clib/scanf.c                          0x00000000   Number         0  C:\Keil_v5\ARM\ARMCC\Bin\..\lib\armlib\c_p.l(_chval.o) ABSOLUTE
    ../clib/signal.c                         0x00000000   Number         0  C:\Keil_v5\ARM\ARMCC\Bin\..\lib\armlib\c_p.l(defsig_rtred_formal.o) ABSOLUTE
    ../clib/signal.c                         0x00000000   Number         0  C:\Keil_v5\ARM\ARMCC\Bin\..\lib\armlib\c_p.l(defsig_pvfn_formal.o) ABSOLUTE
    ../clib/signal.c                         0x00000000   Number         0  C:\Keil_v5\ARM\ARMCC\Bin\..\lib\armlib\c_p.l(defsig_pvfn_outer.o) ABSOLUTE
    ../clib/signal.c                         0x00000000   Number         0  C:\Keil_v5\ARM\ARMCC\Bin\..\lib\armlib\c_p.l(defsig_rtmem_formal.o) ABSOLUTE
    ../clib/signal.c                         0x00000000   Number         0  C:\Keil_v5\ARM\ARMCC\Bin\..\lib\armlib\c_p.l(defsig_rtred_inner.o) ABSOLUTE
    ../clib/signal.c                         0x00000000   Number         0  C:\Keil_v5\ARM\ARMCC\Bin\..\lib\armlib\c_p.l(defsig_fpe_formal.o) ABSOLUTE
    ../clib/signal.c                         0x00000000   Number         0  C:\Keil_v5\ARM\ARMCC\Bin\..\lib\armlib\c_p.l(defsig_fpe_outer.o) ABSOLUTE
    ../clib/signal.c                         0x00000000   Number         0  C:\Keil_v5\ARM\ARMCC\Bin\..\lib\armlib\c_p.l(defsig_general.o) ABSOLUTE
    ../clib/signal.c                         0x00000000   Number         0  C:\Keil_v5\ARM\ARMCC\Bin\..\lib\armlib\c_p.l(__raise.o) ABSOLUTE
    ../clib/signal.c                         0x00000000   Number         0  C:\Keil_v5\ARM\ARMCC\Bin\..\lib\armlib\c_p.l(defsig_rtmem_inner.o) ABSOLUTE
    ../clib/signal.c                         0x00000000   Number         0  C:\Keil_v5\ARM\ARMCC\Bin\..\lib\armlib\c_p.l(defsig_other.o) ABSOLUTE
    ../clib/signal.c                         0x00000000   Number         0  C:\Keil_v5\ARM\ARMCC\Bin\..\lib\armlib\c_p.l(defsig_rtred_outer.o) ABSOLUTE
    ../clib/signal.c                         0x00000000   Number         0  C:\Keil_v5\ARM\ARMCC\Bin\..\lib\armlib\c_p.l(defsig_segv_inner.o) ABSOLUTE
    ../clib/signal.c                         0x00000000   Number         0  C:\Keil_v5\ARM\ARMCC\Bin\..\lib\armlib\c_p.l(defsig_pvfn_inner.o) ABSOLUTE
    ../clib/signal.c                         0x00000000   Number         0  C:\Keil_v5\ARM\ARMCC\Bin\..\lib\armlib\c_p.l(defsig_cppl_inner.o) ABSOLUTE
    ../clib/signal.c                         0x00000000   Number         0  C:\Keil_v5\ARM\ARMCC\Bin\..\lib\armlib\c_p.l(defsig_stak_inner.o) ABSOLUTE
    ../clib/signal.c                         0x00000000   Number         0  C:\Keil_v5\ARM\ARMCC\Bin\..\lib\armlib\c_p.l(defsig_abrt_inner.o) ABSOLUTE
    ../clib/signal.c                         0x00000000   Number         0  C:\Keil_v5\ARM\ARMCC\Bin\..\lib\armlib\c_p.l(defsig_fpe_inner.o) ABSOLUTE
    ../clib/signal.c                         0x00000000   Number         0  C:\Keil_v5\ARM\ARMCC\Bin\..\lib\armlib\c_p.l(defsig_abrt_formal.o) ABSOLUTE
    ../clib/signal.c                         0x00000000   Number         0  C:\Keil_v5\ARM\ARMCC\Bin\..\lib\armlib\c_p.l(defsig_abrt_outer.o) ABSOLUTE
    ../clib/signal.c                         0x00000000   Number         0  C:\Keil_v5\ARM\ARMCC\Bin\..\lib\armlib\c_p.l(defsig_exit.o) ABSOLUTE
    ../clib/signal.c                         0x00000000   Number         0  C:\Keil_v5\ARM\ARMCC\Bin\..\lib\armlib\c_p.l(defsig_rtmem_outer.o) ABSOLUTE
    ../clib/signal.s                         0x00000000   Number         0  C:\Keil_v5\ARM\ARMCC\Bin\..\lib\armlib\c_p.l(defsig.o) ABSOLUTE
    ../clib/stdio.c                          0x00000000   Number         0  C:\Keil_v5\ARM\ARMCC\Bin\..\lib\armlib\c_p.l(fopen_locked.o) ABSOLUTE
    ../clib/stdio.c                          0x00000000   Number         0  C:\Keil_v5\ARM\ARMCC\Bin\..\lib\armlib\c_p.l(ferror.o) ABSOLUTE
    ../clib/stdio.c                          0x00000000   Number         0  C:\Keil_v5\ARM\ARMCC\Bin\..\lib\armlib\c_p.l(fflush_locked.o) ABSOLUTE
    ../clib/stdio.c                          0x00000000   Number         0  C:\Keil_v5\ARM\ARMCC\Bin\..\lib\armlib\c_p.l(fputc_locked.o) ABSOLUTE
    ../clib/stdio.c                          0x00000000   Number         0  C:\Keil_v5\ARM\ARMCC\Bin\..\lib\armlib\c_p.l(fgetc_locked.o) ABSOLUTE
    ../clib/stdio.c                          0x00000000   Number         0  C:\Keil_v5\ARM\ARMCC\Bin\..\lib\armlib\c_p.l(fclose.o) ABSOLUTE
    ../clib/stdio.c                          0x00000000   Number         0  C:\Keil_v5\ARM\ARMCC\Bin\..\lib\armlib\c_p.l(stdio_streams.o) ABSOLUTE
    ../clib/stdio.c                          0x00000000   Number         0  C:\Keil_v5\ARM\ARMCC\Bin\..\lib\armlib\c_p.l(setbuf.o) ABSOLUTE
    ../clib/stdio.c                          0x00000000   Number         0  C:\Keil_v5\ARM\ARMCC\Bin\..\lib\armlib\c_p.l(fopen.o) ABSOLUTE
    ../clib/stdio.c                          0x00000000   Number         0  C:\Keil_v5\ARM\ARMCC\Bin\..\lib\armlib\c_p.l(fputs.o) ABSOLUTE
    ../clib/stdio.c                          0x00000000   Number         0  C:\Keil_v5\ARM\ARMCC\Bin\..\lib\armlib\c_p.l(fputc.o) ABSOLUTE
    ../clib/stdio.c                          0x00000000   Number         0  C:\Keil_v5\ARM\ARMCC\Bin\..\lib\armlib\c_p.l(fgets.o) ABSOLUTE
    ../clib/stdio.c                          0x00000000   Number         0  C:\Keil_v5\ARM\ARMCC\Bin\..\lib\armlib\c_p.l(fgetc.o) ABSOLUTE
    ../clib/stdio.c                          0x00000000   Number         0  C:\Keil_v5\ARM\ARMCC\Bin\..\lib\armlib\c_p.l(fflush.o) ABSOLUTE
    ../clib/stdio.c                          0x00000000   Number         0  C:\Keil_v5\ARM\ARMCC\Bin\..\lib\armlib\c_p.l(fclose_locked.o) ABSOLUTE
    ../clib/stdio.c                          0x00000000   Number         0  C:\Keil_v5\ARM\ARMCC\Bin\..\lib\armlib\c_p.l(backspace.o) ABSOLUTE
    ../clib/stdio.c                          0x00000000   Number         0  C:\Keil_v5\ARM\ARMCC\Bin\..\lib\armlib\c_p.l(ftell.o) ABSOLUTE
    ../clib/stdio.c                          0x00000000   Number         0  C:\Keil_v5\ARM\ARMCC\Bin\..\lib\armlib\c_p.l(freadfast.o) ABSOLUTE
    ../clib/stdio.c                          0x00000000   Number         0  C:\Keil_v5\ARM\ARMCC\Bin\..\lib\armlib\c_p.l(fread_bytes_avail.o) ABSOLUTE
    ../clib/stdio.c                          0x00000000   Number         0  C:\Keil_v5\ARM\ARMCC\Bin\..\lib\armlib\c_p.l(fwritefast.o) ABSOLUTE
    ../clib/stdio.c                          0x00000000   Number         0  C:\Keil_v5\ARM\ARMCC\Bin\..\lib\armlib\c_p.l(fgets_locked.o) ABSOLUTE
    ../clib/stdio.c                          0x00000000   Number         0  C:\Keil_v5\ARM\ARMCC\Bin\..\lib\armlib\c_p.l(flushlinebuffered.o) ABSOLUTE
    ../clib/stdio.c                          0x00000000   Number         0  C:\Keil_v5\ARM\ARMCC\Bin\..\lib\armlib\c_p.l(fputs_locked.o) ABSOLUTE
    ../clib/stdio.c                          0x00000000   Number         0  C:\Keil_v5\ARM\ARMCC\Bin\..\lib\armlib\c_p.l(filbuf.o) ABSOLUTE
    ../clib/stdio.c                          0x00000000   Number         0  C:\Keil_v5\ARM\ARMCC\Bin\..\lib\armlib\c_p.l(flsbuf.o) ABSOLUTE
    ../clib/stdio.c                          0x00000000   Number         0  C:\Keil_v5\ARM\ARMCC\Bin\..\lib\armlib\c_p.l(backspace_locked.o) ABSOLUTE
    ../clib/stdio.c                          0x00000000   Number         0  C:\Keil_v5\ARM\ARMCC\Bin\..\lib\armlib\c_p.l(freadfast_locked.o) ABSOLUTE
    ../clib/stdio.c                          0x00000000   Number         0  C:\Keil_v5\ARM\ARMCC\Bin\..\lib\armlib\c_p.l(initio_locked.o) ABSOLUTE
    ../clib/stdio.c                          0x00000000   Number         0  C:\Keil_v5\ARM\ARMCC\Bin\..\lib\armlib\c_p.l(setvbuf_locked.o) ABSOLUTE
    ../clib/stdio.c                          0x00000000   Number         0  C:\Keil_v5\ARM\ARMCC\Bin\..\lib\armlib\c_p.l(ferror_locked.o) ABSOLUTE
    ../clib/stdio.c                          0x00000000   Number         0  C:\Keil_v5\ARM\ARMCC\Bin\..\lib\armlib\c_p.l(fseek.o) ABSOLUTE
    ../clib/stdio.c                          0x00000000   Number         0  C:\Keil_v5\ARM\ARMCC\Bin\..\lib\armlib\c_p.l(setvbuf.o) ABSOLUTE
    ../clib/stdio.c                          0x00000000   Number         0  C:\Keil_v5\ARM\ARMCC\Bin\..\lib\armlib\c_p.l(initio.o) ABSOLUTE
    ../clib/stdio.c                          0x00000000   Number         0  C:\Keil_v5\ARM\ARMCC\Bin\..\lib\armlib\c_p.l(streamlock.o) ABSOLUTE
    ../clib/stdio.c                          0x00000000   Number         0  C:\Keil_v5\ARM\ARMCC\Bin\..\lib\armlib\c_p.l(stdio.o) ABSOLUTE
    ../clib/stdio.c                          0x00000000   Number         0  C:\Keil_v5\ARM\ARMCC\Bin\..\lib\armlib\c_p.l(fread_bytes_avail_locked.o) ABSOLUTE
    ../clib/stdio.c                          0x00000000   Number         0  C:\Keil_v5\ARM\ARMCC\Bin\..\lib\armlib\c_p.l(fwritefast_locked.o) ABSOLUTE
    ../clib/stdio.c                          0x00000000   Number         0  C:\Keil_v5\ARM\ARMCC\Bin\..\lib\armlib\c_p.l(flushlinebuffered_locked.o) ABSOLUTE
    ../clib/stdio.c                          0x00000000   Number         0  C:\Keil_v5\ARM\ARMCC\Bin\..\lib\armlib\c_p.l(ungetc.o) ABSOLUTE
    ../clib/stdlib.c                         0x00000000   Number         0  C:\Keil_v5\ARM\ARMCC\Bin\..\lib\armlib\c_p.l(bsearchnoex.o) ABSOLUTE
    ../clib/stdlib.c                         0x00000000   Number         0  C:\Keil_v5\ARM\ARMCC\Bin\..\lib\armlib\c_p.l(abort.o) ABSOLUTE
    ../clib/string.c                         0x00000000   Number         0  C:\Keil_v5\ARM\ARMCC\Bin\..\lib\armlib\c_p.l(strncmp.o) ABSOLUTE
    ../clib/string.c                         0x00000000   Number         0  C:\Keil_v5\ARM\ARMCC\Bin\..\lib\armlib\c_p.l(strlen.o) ABSOLUTE
    ../clib/string.c                         0x00000000   Number         0  C:\Keil_v5\ARM\ARMCC\Bin\..\lib\armlib\c_p.l(strncpy.o) ABSOLUTE
    ../clib/time.c                           0x00000000   Number         0  C:\Keil_v5\ARM\ARMCC\Bin\..\lib\armlib\c_p.l(_monlen.o) ABSOLUTE
    ../clib/time.c                           0x00000000   Number         0  C:\Keil_v5\ARM\ARMCC\Bin\..\lib\armlib\c_p.l(localtime_internal.o) ABSOLUTE
    ../clib/time.c                           0x00000000   Number         0  C:\Keil_v5\ARM\ARMCC\Bin\..\lib\armlib\c_p.l(localtime.o) ABSOLUTE
    ../clib/time.c                           0x00000000   Number         0  C:\Keil_v5\ARM\ARMCC\Bin\..\lib\armlib\c_p.l(mktime.o) ABSOLUTE
    ../clib/wchar.c                          0x00000000   Number         0  C:\Keil_v5\ARM\ARMCC\Bin\..\lib\armlib\c_p.l(flsbuf_fwide.o) ABSOLUTE
    ../clib/wchar.c                          0x00000000   Number         0  C:\Keil_v5\ARM\ARMCC\Bin\..\lib\armlib\c_p.l(filbuf_fwide.o) ABSOLUTE
    ../fplib/cfplib/cmpret.c                 0x00000000   Number         0  C:\Keil_v5\ARM\ARMCC\Bin\..\lib\armlib\fz_ps.l(cmpret.o) ABSOLUTE
    ../fplib/cfplib/d2f.c                    0x00000000   Number         0  C:\Keil_v5\ARM\ARMCC\Bin\..\lib\armlib\fz_ps.l(d2f.o) ABSOLUTE
    ../fplib/cfplib/daddsub.c                0x00000000   Number         0  C:\Keil_v5\ARM\ARMCC\Bin\..\lib\armlib\fz_ps.l(daddsub.o) ABSOLUTE
    ../fplib/cfplib/dcmpin.c                 0x00000000   Number         0  C:\Keil_v5\ARM\ARMCC\Bin\..\lib\armlib\fz_ps.l(dcmpin.o) ABSOLUTE
    ../fplib/cfplib/ddiv.c                   0x00000000   Number         0  C:\Keil_v5\ARM\ARMCC\Bin\..\lib\armlib\fz_ps.l(ddiv.o) ABSOLUTE
    ../fplib/cfplib/dmul.c                   0x00000000   Number         0  C:\Keil_v5\ARM\ARMCC\Bin\..\lib\armlib\fz_ps.l(dmul.o) ABSOLUTE
    ../fplib/cfplib/f2d.c                    0x00000000   Number         0  C:\Keil_v5\ARM\ARMCC\Bin\..\lib\armlib\fz_ps.l(f2d.o) ABSOLUTE
    ../fplib/cfplib/fdiv.c                   0x00000000   Number         0  C:\Keil_v5\ARM\ARMCC\Bin\..\lib\armlib\fz_ps.l(fdiv.o) ABSOLUTE
    ../fplib/cfplib/ffix.c                   0x00000000   Number         0  C:\Keil_v5\ARM\ARMCC\Bin\..\lib\armlib\fz_ps.l(ffixi.o) ABSOLUTE
    ../fplib/cfplib/ffix.c                   0x00000000   Number         0  C:\Keil_v5\ARM\ARMCC\Bin\..\lib\armlib\fz_ps.l(ffixui.o) ABSOLUTE
    ../fplib/cfplib/ffix.c                   0x00000000   Number         0  C:\Keil_v5\ARM\ARMCC\Bin\..\lib\armlib\fz_ps.l(dfixui.o) ABSOLUTE
    ../fplib/cfplib/fflt.c                   0x00000000   Number         0  C:\Keil_v5\ARM\ARMCC\Bin\..\lib\armlib\fz_ps.l(fflti.o) ABSOLUTE
    ../fplib/cfplib/fflt.c                   0x00000000   Number         0  C:\Keil_v5\ARM\ARMCC\Bin\..\lib\armlib\fz_ps.l(dflti.o) ABSOLUTE
    ../fplib/cfplib/fpinit.c                 0x00000000   Number         0  C:\Keil_v5\ARM\ARMCC\Bin\..\lib\armlib\fz_ps.l(fpinit.o) ABSOLUTE
    ../fplib/cfplib/ieee_status.c            0x00000000   Number         0  C:\Keil_v5\ARM\ARMCC\Bin\..\lib\armlib\fz_ps.l(ieee_status.o) ABSOLUTE
    ../fplib/cfplib/nan2.c                   0x00000000   Number         0  C:\Keil_v5\ARM\ARMCC\Bin\..\lib\armlib\fz_ps.l(dnan2.o) ABSOLUTE
    ../fplib/cfplib/retnan.c                 0x00000000   Number         0  C:\Keil_v5\ARM\ARMCC\Bin\..\lib\armlib\fz_ps.l(retnan.o) ABSOLUTE
    ../fplib/cfplib/scalbn.c                 0x00000000   Number         0  C:\Keil_v5\ARM\ARMCC\Bin\..\lib\armlib\fz_ps.l(dscalbn.o) ABSOLUTE
    ../fplib/deqf6m.s                        0x00000000   Number         0  C:\Keil_v5\ARM\ARMCC\Bin\..\lib\armlib\fz_ps.l(deqf.o) ABSOLUTE
    ../fplib/drleqf6m.s                      0x00000000   Number         0  C:\Keil_v5\ARM\ARMCC\Bin\..\lib\armlib\fz_ps.l(drlef.o) ABSOLUTE
    ../fplib/fmul6m.s                        0x00000000   Number         0  C:\Keil_v5\ARM\ARMCC\Bin\..\lib\armlib\fz_ps.l(fmul.o) ABSOLUTE
    ../fplib/fpconst.s                       0x00000000   Number         0  C:\Keil_v5\ARM\ARMCC\Bin\..\lib\armlib\fz_ps.l(fpconst.o) ABSOLUTE
    ../fplib/printf1.s                       0x00000000   Number         0  C:\Keil_v5\ARM\ARMCC\Bin\..\lib\armlib\fz_ps.l(printf1.o) ABSOLUTE
    ../fplib/printf2.s                       0x00000000   Number         0  C:\Keil_v5\ARM\ARMCC\Bin\..\lib\armlib\fz_ps.l(printf2.o) ABSOLUTE
    ../fplib/printf2a.s                      0x00000000   Number         0  C:\Keil_v5\ARM\ARMCC\Bin\..\lib\armlib\fz_ps.l(printf2a.o) ABSOLUTE
    ../fplib/printf2b.s                      0x00000000   Number         0  C:\Keil_v5\ARM\ARMCC\Bin\..\lib\armlib\fz_ps.l(printf2b.o) ABSOLUTE
    ../fplib/scanf1.s                        0x00000000   Number         0  C:\Keil_v5\ARM\ARMCC\Bin\..\lib\armlib\fz_ps.l(scanf1.o) ABSOLUTE
    ../fplib/scanf2.s                        0x00000000   Number         0  C:\Keil_v5\ARM\ARMCC\Bin\..\lib\armlib\fz_ps.l(scanf2.o) ABSOLUTE
    ../fplib/scanf2a.s                       0x00000000   Number         0  C:\Keil_v5\ARM\ARMCC\Bin\..\lib\armlib\fz_ps.l(scanf2a.o) ABSOLUTE
    ../fplib/scanf2b.s                       0x00000000   Number         0  C:\Keil_v5\ARM\ARMCC\Bin\..\lib\armlib\fz_ps.l(scanf2b.o) ABSOLUTE
    ../fplib/usenofp.s                       0x00000000   Number         0  C:\Keil_v5\ARM\ARMCC\Bin\..\lib\armlib\fz_ps.l(usenofp.o) ABSOLUTE
    ../mathlib/dunder.c                      0x00000000   Number         0  C:\Keil_v5\ARM\ARMCC\Bin\..\lib\armlib\m_ps.l(dunder.o) ABSOLUTE
    ../mathlib/fpclassify.c                  0x00000000   Number         0  C:\Keil_v5\ARM\ARMCC\Bin\..\lib\armlib\m_ps.l(fpclassify.o) ABSOLUTE
    ../mathlib/frexp.c                       0x00000000   Number         0  C:\Keil_v5\ARM\ARMCC\Bin\..\lib\armlib\m_ps.l(frexp.o) ABSOLUTE
    ../mathlib/ldexp.c                       0x00000000   Number         0  C:\Keil_v5\ARM\ARMCC\Bin\..\lib\armlib\m_ps.l(ldexp.o) ABSOLUTE
    ../mathlib/ldexp.c                       0x00000000   Number         0  C:\Keil_v5\ARM\ARMCC\Bin\..\lib\armlib\m_ps.l(ldexp_x.o) ABSOLUTE
    ../mathlib/narrow.c                      0x00000000   Number         0  C:\Keil_v5\ARM\ARMCC\Bin\..\lib\armlib\m_ps.l(narrow.o) ABSOLUTE
    ../mathlib/qnan.c                        0x00000000   Number         0  C:\Keil_v5\ARM\ARMCC\Bin\..\lib\armlib\m_ps.l(qnan.o) ABSOLUTE
    BufferedSerial.cpp                       0x00000000   Number         0  .\build\bufferedserial.o ABSOLUTE
    BufferedSerial.cpp                       0x00000000   Number         0  .\build\bufferedserial.o ABSOLUTE
    C:\Jenkins\workspace\mbed-2-build-library\drivers\FileBase.cpp 0x00000000   Number         0  mbed/TARGET_NUCLEO_F070RB/TOOLCHAIN_ARM_STD/mbed.ar(FileBase.o) ABSOLUTE
    C:\Jenkins\workspace\mbed-2-build-library\drivers\FileLike.cpp 0x00000000   Number         0  mbed/TARGET_NUCLEO_F070RB/TOOLCHAIN_ARM_STD/mbed.ar(FileLike.o) ABSOLUTE
    C:\Jenkins\workspace\mbed-2-build-library\drivers\FilePath.cpp 0x00000000   Number         0  mbed/TARGET_NUCLEO_F070RB/TOOLCHAIN_ARM_STD/mbed.ar(FilePath.o) ABSOLUTE
    C:\Jenkins\workspace\mbed-2-build-library\drivers\FileSystemLike.cpp 0x00000000   Number         0  mbed/TARGET_NUCLEO_F070RB/TOOLCHAIN_ARM_STD/mbed.ar(FileSystemLike.o) ABSOLUTE
    C:\Jenkins\workspace\mbed-2-build-library\drivers\RawSerial.cpp 0x00000000   Number         0  mbed/TARGET_NUCLEO_F070RB/TOOLCHAIN_ARM_STD/mbed.ar(RawSerial.o) ABSOLUTE
    C:\Jenkins\workspace\mbed-2-build-library\drivers\Serial.cpp 0x00000000   Number         0  mbed/TARGET_NUCLEO_F070RB/TOOLCHAIN_ARM_STD/mbed.ar(Serial.o) ABSOLUTE
    C:\Jenkins\workspace\mbed-2-build-library\drivers\SerialBase.cpp 0x00000000   Number         0  mbed/TARGET_NUCLEO_F070RB/TOOLCHAIN_ARM_STD/mbed.ar(SerialBase.o) ABSOLUTE
    C:\Jenkins\workspace\mbed-2-build-library\drivers\Stream.cpp 0x00000000   Number         0  mbed/TARGET_NUCLEO_F070RB/TOOLCHAIN_ARM_STD/mbed.ar(Stream.o) ABSOLUTE
    C:\Jenkins\workspace\mbed-2-build-library\drivers\Ticker.cpp 0x00000000   Number         0  mbed/TARGET_NUCLEO_F070RB/TOOLCHAIN_ARM_STD/mbed.ar(Ticker.o) ABSOLUTE
    C:\Jenkins\workspace\mbed-2-build-library\drivers\Timer.cpp 0x00000000   Number         0  mbed/TARGET_NUCLEO_F070RB/TOOLCHAIN_ARM_STD/mbed.ar(Timer.o) ABSOLUTE
    C:\Jenkins\workspace\mbed-2-build-library\drivers\TimerEvent.cpp 0x00000000   Number         0  mbed/TARGET_NUCLEO_F070RB/TOOLCHAIN_ARM_STD/mbed.ar(TimerEvent.o) ABSOLUTE
    C:\Jenkins\workspace\mbed-2-build-library\hal\mbed_gpio.c 0x00000000   Number         0  mbed/TARGET_NUCLEO_F070RB/TOOLCHAIN_ARM_STD/mbed.ar(mbed_gpio.o) ABSOLUTE
    C:\Jenkins\workspace\mbed-2-build-library\hal\mbed_lp_ticker_api.c 0x00000000   Number         0  mbed/TARGET_NUCLEO_F070RB/TOOLCHAIN_ARM_STD/mbed.ar(mbed_lp_ticker_api.o) ABSOLUTE
    C:\Jenkins\workspace\mbed-2-build-library\hal\mbed_pinmap_common.c 0x00000000   Number         0  mbed/TARGET_NUCLEO_F070RB/TOOLCHAIN_ARM_STD/mbed.ar(mbed_pinmap_common.o) ABSOLUTE
    C:\Jenkins\workspace\mbed-2-build-library\hal\mbed_ticker_api.c 0x00000000   Number         0  mbed/TARGET_NUCLEO_F070RB/TOOLCHAIN_ARM_STD/mbed.ar(mbed_ticker_api.o) ABSOLUTE
    C:\Jenkins\workspace\mbed-2-build-library\hal\mbed_us_ticker_api.c 0x00000000   Number         0  mbed/TARGET_NUCLEO_F070RB/TOOLCHAIN_ARM_STD/mbed.ar(mbed_us_ticker_api.o) ABSOLUTE
    C:\Jenkins\workspace\mbed-2-build-library\platform\mbed_assert.c 0x00000000   Number         0  mbed/TARGET_NUCLEO_F070RB/TOOLCHAIN_ARM_STD/mbed.ar(mbed_assert.o) ABSOLUTE
    C:\Jenkins\workspace\mbed-2-build-library\platform\mbed_board.c 0x00000000   Number         0  mbed/TARGET_NUCLEO_F070RB/TOOLCHAIN_ARM_STD/mbed_board.o ABSOLUTE
    C:\Jenkins\workspace\mbed-2-build-library\platform\mbed_critical.c 0x00000000   Number         0  mbed/TARGET_NUCLEO_F070RB/TOOLCHAIN_ARM_STD/mbed.ar(mbed_critical.o) ABSOLUTE
    C:\Jenkins\workspace\mbed-2-build-library\platform\mbed_error.c 0x00000000   Number         0  mbed/TARGET_NUCLEO_F070RB/TOOLCHAIN_ARM_STD/mbed.ar(mbed_error.o) ABSOLUTE
    C:\Jenkins\workspace\mbed-2-build-library\platform\mbed_wait_api_no_rtos.c 0x00000000   Number         0  mbed/TARGET_NUCLEO_F070RB/TOOLCHAIN_ARM_STD/mbed.ar(mbed_wait_api_no_rtos.o) ABSOLUTE
    C:\Jenkins\workspace\mbed-2-build-library\platform\retarget.cpp 0x00000000   Number         0  mbed/TARGET_NUCLEO_F070RB/TOOLCHAIN_ARM_STD/retarget.o ABSOLUTE
    C:\Jenkins\workspace\mbed-2-build-library\targets\TARGET_STM\TARGET_STM32F0\TARGET_NUCLEO_F070RB\PeripheralPins.c 0x00000000   Number         0  mbed/TARGET_NUCLEO_F070RB/TOOLCHAIN_ARM_STD/PeripheralPins.o ABSOLUTE
    C:\Jenkins\workspace\mbed-2-build-library\targets\TARGET_STM\TARGET_STM32F0\TARGET_NUCLEO_F070RB\device\TOOLCHAIN_ARM_STD\sys.cpp 0x00000000   Number         0  mbed/TARGET_NUCLEO_F070RB/TOOLCHAIN_ARM_STD/sys.o ABSOLUTE
    C:\Jenkins\workspace\mbed-2-build-library\targets\TARGET_STM\TARGET_STM32F0\TARGET_NUCLEO_F070RB\device\cmsis_nvic.c 0x00000000   Number         0  mbed/TARGET_NUCLEO_F070RB/TOOLCHAIN_ARM_STD/cmsis_nvic.o ABSOLUTE
    C:\Jenkins\workspace\mbed-2-build-library\targets\TARGET_STM\TARGET_STM32F0\TARGET_NUCLEO_F070RB\device\hal_tick.c 0x00000000   Number         0  mbed/TARGET_NUCLEO_F070RB/TOOLCHAIN_ARM_STD/hal_tick.o ABSOLUTE
    C:\Jenkins\workspace\mbed-2-build-library\targets\TARGET_STM\TARGET_STM32F0\TARGET_NUCLEO_F070RB\device\system_stm32f0xx.c 0x00000000   Number         0  mbed/TARGET_NUCLEO_F070RB/TOOLCHAIN_ARM_STD/system_stm32f0xx.o ABSOLUTE
    C:\Jenkins\workspace\mbed-2-build-library\targets\TARGET_STM\TARGET_STM32F0\analogin_api.c 0x00000000   Number         0  mbed/TARGET_NUCLEO_F070RB/TOOLCHAIN_ARM_STD/analogin_api.o ABSOLUTE
    C:\Jenkins\workspace\mbed-2-build-library\targets\TARGET_STM\TARGET_STM32F0\analogout_api.c 0x00000000   Number         0  mbed/TARGET_NUCLEO_F070RB/TOOLCHAIN_ARM_STD/analogout_api.o ABSOLUTE
    C:\Jenkins\workspace\mbed-2-build-library\targets\TARGET_STM\TARGET_STM32F0\can_api.c 0x00000000   Number         0  mbed/TARGET_NUCLEO_F070RB/TOOLCHAIN_ARM_STD/can_api.o ABSOLUTE
    C:\Jenkins\workspace\mbed-2-build-library\targets\TARGET_STM\TARGET_STM32F0\device\stm32f0xx_hal.c 0x00000000   Number         0  mbed/TARGET_NUCLEO_F070RB/TOOLCHAIN_ARM_STD/stm32f0xx_hal.o ABSOLUTE
    C:\Jenkins\workspace\mbed-2-build-library\targets\TARGET_STM\TARGET_STM32F0\device\stm32f0xx_hal_adc.c 0x00000000   Number         0  mbed/TARGET_NUCLEO_F070RB/TOOLCHAIN_ARM_STD/stm32f0xx_hal_adc.o ABSOLUTE
    C:\Jenkins\workspace\mbed-2-build-library\targets\TARGET_STM\TARGET_STM32F0\device\stm32f0xx_hal_adc_ex.c 0x00000000   Number         0  mbed/TARGET_NUCLEO_F070RB/TOOLCHAIN_ARM_STD/stm32f0xx_hal_adc_ex.o ABSOLUTE
    C:\Jenkins\workspace\mbed-2-build-library\targets\TARGET_STM\TARGET_STM32F0\device\stm32f0xx_hal_can.c 0x00000000   Number         0  mbed/TARGET_NUCLEO_F070RB/TOOLCHAIN_ARM_STD/stm32f0xx_hal_can.o ABSOLUTE
    C:\Jenkins\workspace\mbed-2-build-library\targets\TARGET_STM\TARGET_STM32F0\device\stm32f0xx_hal_cec.c 0x00000000   Number         0  mbed/TARGET_NUCLEO_F070RB/TOOLCHAIN_ARM_STD/stm32f0xx_hal_cec.o ABSOLUTE
    C:\Jenkins\workspace\mbed-2-build-library\targets\TARGET_STM\TARGET_STM32F0\device\stm32f0xx_hal_comp.c 0x00000000   Number         0  mbed/TARGET_NUCLEO_F070RB/TOOLCHAIN_ARM_STD/stm32f0xx_hal_comp.o ABSOLUTE
    C:\Jenkins\workspace\mbed-2-build-library\targets\TARGET_STM\TARGET_STM32F0\device\stm32f0xx_hal_cortex.c 0x00000000   Number         0  mbed/TARGET_NUCLEO_F070RB/TOOLCHAIN_ARM_STD/stm32f0xx_hal_cortex.o ABSOLUTE
    C:\Jenkins\workspace\mbed-2-build-library\targets\TARGET_STM\TARGET_STM32F0\device\stm32f0xx_hal_crc.c 0x00000000   Number         0  mbed/TARGET_NUCLEO_F070RB/TOOLCHAIN_ARM_STD/stm32f0xx_hal_crc.o ABSOLUTE
    C:\Jenkins\workspace\mbed-2-build-library\targets\TARGET_STM\TARGET_STM32F0\device\stm32f0xx_hal_crc_ex.c 0x00000000   Number         0  mbed/TARGET_NUCLEO_F070RB/TOOLCHAIN_ARM_STD/stm32f0xx_hal_crc_ex.o ABSOLUTE
    C:\Jenkins\workspace\mbed-2-build-library\targets\TARGET_STM\TARGET_STM32F0\device\stm32f0xx_hal_dac.c 0x00000000   Number         0  mbed/TARGET_NUCLEO_F070RB/TOOLCHAIN_ARM_STD/stm32f0xx_hal_dac.o ABSOLUTE
    C:\Jenkins\workspace\mbed-2-build-library\targets\TARGET_STM\TARGET_STM32F0\device\stm32f0xx_hal_dac_ex.c 0x00000000   Number         0  mbed/TARGET_NUCLEO_F070RB/TOOLCHAIN_ARM_STD/stm32f0xx_hal_dac_ex.o ABSOLUTE
    C:\Jenkins\workspace\mbed-2-build-library\targets\TARGET_STM\TARGET_STM32F0\device\stm32f0xx_hal_dma.c 0x00000000   Number         0  mbed/TARGET_NUCLEO_F070RB/TOOLCHAIN_ARM_STD/stm32f0xx_hal_dma.o ABSOLUTE
    C:\Jenkins\workspace\mbed-2-build-library\targets\TARGET_STM\TARGET_STM32F0\device\stm32f0xx_hal_flash.c 0x00000000   Number         0  mbed/TARGET_NUCLEO_F070RB/TOOLCHAIN_ARM_STD/stm32f0xx_hal_flash.o ABSOLUTE
    C:\Jenkins\workspace\mbed-2-build-library\targets\TARGET_STM\TARGET_STM32F0\device\stm32f0xx_hal_flash_ex.c 0x00000000   Number         0  mbed/TARGET_NUCLEO_F070RB/TOOLCHAIN_ARM_STD/stm32f0xx_hal_flash_ex.o ABSOLUTE
    C:\Jenkins\workspace\mbed-2-build-library\targets\TARGET_STM\TARGET_STM32F0\device\stm32f0xx_hal_gpio.c 0x00000000   Number         0  mbed/TARGET_NUCLEO_F070RB/TOOLCHAIN_ARM_STD/stm32f0xx_hal_gpio.o ABSOLUTE
    C:\Jenkins\workspace\mbed-2-build-library\targets\TARGET_STM\TARGET_STM32F0\device\stm32f0xx_hal_i2c.c 0x00000000   Number         0  mbed/TARGET_NUCLEO_F070RB/TOOLCHAIN_ARM_STD/stm32f0xx_hal_i2c.o ABSOLUTE
    C:\Jenkins\workspace\mbed-2-build-library\targets\TARGET_STM\TARGET_STM32F0\device\stm32f0xx_hal_i2c_ex.c 0x00000000   Number         0  mbed/TARGET_NUCLEO_F070RB/TOOLCHAIN_ARM_STD/stm32f0xx_hal_i2c_ex.o ABSOLUTE
    C:\Jenkins\workspace\mbed-2-build-library\targets\TARGET_STM\TARGET_STM32F0\device\stm32f0xx_hal_i2s.c 0x00000000   Number         0  mbed/TARGET_NUCLEO_F070RB/TOOLCHAIN_ARM_STD/stm32f0xx_hal_i2s.o ABSOLUTE
    C:\Jenkins\workspace\mbed-2-build-library\targets\TARGET_STM\TARGET_STM32F0\device\stm32f0xx_hal_irda.c 0x00000000   Number         0  mbed/TARGET_NUCLEO_F070RB/TOOLCHAIN_ARM_STD/stm32f0xx_hal_irda.o ABSOLUTE
    C:\Jenkins\workspace\mbed-2-build-library\targets\TARGET_STM\TARGET_STM32F0\device\stm32f0xx_hal_iwdg.c 0x00000000   Number         0  mbed/TARGET_NUCLEO_F070RB/TOOLCHAIN_ARM_STD/stm32f0xx_hal_iwdg.o ABSOLUTE
    C:\Jenkins\workspace\mbed-2-build-library\targets\TARGET_STM\TARGET_STM32F0\device\stm32f0xx_hal_pcd.c 0x00000000   Number         0  mbed/TARGET_NUCLEO_F070RB/TOOLCHAIN_ARM_STD/stm32f0xx_hal_pcd.o ABSOLUTE
    C:\Jenkins\workspace\mbed-2-build-library\targets\TARGET_STM\TARGET_STM32F0\device\stm32f0xx_hal_pcd_ex.c 0x00000000   Number         0  mbed/TARGET_NUCLEO_F070RB/TOOLCHAIN_ARM_STD/stm32f0xx_hal_pcd_ex.o ABSOLUTE
    C:\Jenkins\workspace\mbed-2-build-library\targets\TARGET_STM\TARGET_STM32F0\device\stm32f0xx_hal_pwr.c 0x00000000   Number         0  mbed/TARGET_NUCLEO_F070RB/TOOLCHAIN_ARM_STD/stm32f0xx_hal_pwr.o ABSOLUTE
    C:\Jenkins\workspace\mbed-2-build-library\targets\TARGET_STM\TARGET_STM32F0\device\stm32f0xx_hal_pwr_ex.c 0x00000000   Number         0  mbed/TARGET_NUCLEO_F070RB/TOOLCHAIN_ARM_STD/stm32f0xx_hal_pwr_ex.o ABSOLUTE
    C:\Jenkins\workspace\mbed-2-build-library\targets\TARGET_STM\TARGET_STM32F0\device\stm32f0xx_hal_rcc.c 0x00000000   Number         0  mbed/TARGET_NUCLEO_F070RB/TOOLCHAIN_ARM_STD/stm32f0xx_hal_rcc.o ABSOLUTE
    C:\Jenkins\workspace\mbed-2-build-library\targets\TARGET_STM\TARGET_STM32F0\device\stm32f0xx_hal_rcc_ex.c 0x00000000   Number         0  mbed/TARGET_NUCLEO_F070RB/TOOLCHAIN_ARM_STD/stm32f0xx_hal_rcc_ex.o ABSOLUTE
    C:\Jenkins\workspace\mbed-2-build-library\targets\TARGET_STM\TARGET_STM32F0\device\stm32f0xx_hal_rtc.c 0x00000000   Number         0  mbed/TARGET_NUCLEO_F070RB/TOOLCHAIN_ARM_STD/stm32f0xx_hal_rtc.o ABSOLUTE
    C:\Jenkins\workspace\mbed-2-build-library\targets\TARGET_STM\TARGET_STM32F0\device\stm32f0xx_hal_rtc_ex.c 0x00000000   Number         0  mbed/TARGET_NUCLEO_F070RB/TOOLCHAIN_ARM_STD/stm32f0xx_hal_rtc_ex.o ABSOLUTE
    C:\Jenkins\workspace\mbed-2-build-library\targets\TARGET_STM\TARGET_STM32F0\device\stm32f0xx_hal_smartcard.c 0x00000000   Number         0  mbed/TARGET_NUCLEO_F070RB/TOOLCHAIN_ARM_STD/stm32f0xx_hal_smartcard.o ABSOLUTE
    C:\Jenkins\workspace\mbed-2-build-library\targets\TARGET_STM\TARGET_STM32F0\device\stm32f0xx_hal_smartcard_ex.c 0x00000000   Number         0  mbed/TARGET_NUCLEO_F070RB/TOOLCHAIN_ARM_STD/stm32f0xx_hal_smartcard_ex.o ABSOLUTE
    C:\Jenkins\workspace\mbed-2-build-library\targets\TARGET_STM\TARGET_STM32F0\device\stm32f0xx_hal_smbus.c 0x00000000   Number         0  mbed/TARGET_NUCLEO_F070RB/TOOLCHAIN_ARM_STD/stm32f0xx_hal_smbus.o ABSOLUTE
    C:\Jenkins\workspace\mbed-2-build-library\targets\TARGET_STM\TARGET_STM32F0\device\stm32f0xx_hal_spi.c 0x00000000   Number         0  mbed/TARGET_NUCLEO_F070RB/TOOLCHAIN_ARM_STD/stm32f0xx_hal_spi.o ABSOLUTE
    C:\Jenkins\workspace\mbed-2-build-library\targets\TARGET_STM\TARGET_STM32F0\device\stm32f0xx_hal_spi_ex.c 0x00000000   Number         0  mbed/TARGET_NUCLEO_F070RB/TOOLCHAIN_ARM_STD/stm32f0xx_hal_spi_ex.o ABSOLUTE
    C:\Jenkins\workspace\mbed-2-build-library\targets\TARGET_STM\TARGET_STM32F0\device\stm32f0xx_hal_tim.c 0x00000000   Number         0  mbed/TARGET_NUCLEO_F070RB/TOOLCHAIN_ARM_STD/stm32f0xx_hal_tim.o ABSOLUTE
    C:\Jenkins\workspace\mbed-2-build-library\targets\TARGET_STM\TARGET_STM32F0\device\stm32f0xx_hal_tim_ex.c 0x00000000   Number         0  mbed/TARGET_NUCLEO_F070RB/TOOLCHAIN_ARM_STD/stm32f0xx_hal_tim_ex.o ABSOLUTE
    C:\Jenkins\workspace\mbed-2-build-library\targets\TARGET_STM\TARGET_STM32F0\device\stm32f0xx_hal_tsc.c 0x00000000   Number         0  mbed/TARGET_NUCLEO_F070RB/TOOLCHAIN_ARM_STD/stm32f0xx_hal_tsc.o ABSOLUTE
    C:\Jenkins\workspace\mbed-2-build-library\targets\TARGET_STM\TARGET_STM32F0\device\stm32f0xx_hal_uart.c 0x00000000   Number         0  mbed/TARGET_NUCLEO_F070RB/TOOLCHAIN_ARM_STD/stm32f0xx_hal_uart.o ABSOLUTE
    C:\Jenkins\workspace\mbed-2-build-library\targets\TARGET_STM\TARGET_STM32F0\device\stm32f0xx_hal_uart_ex.c 0x00000000   Number         0  mbed/TARGET_NUCLEO_F070RB/TOOLCHAIN_ARM_STD/stm32f0xx_hal_uart_ex.o ABSOLUTE
    C:\Jenkins\workspace\mbed-2-build-library\targets\TARGET_STM\TARGET_STM32F0\device\stm32f0xx_hal_usart.c 0x00000000   Number         0  mbed/TARGET_NUCLEO_F070RB/TOOLCHAIN_ARM_STD/stm32f0xx_hal_usart.o ABSOLUTE
    C:\Jenkins\workspace\mbed-2-build-library\targets\TARGET_STM\TARGET_STM32F0\device\stm32f0xx_hal_wwdg.c 0x00000000   Number         0  mbed/TARGET_NUCLEO_F070RB/TOOLCHAIN_ARM_STD/stm32f0xx_hal_wwdg.o ABSOLUTE
    C:\Jenkins\workspace\mbed-2-build-library\targets\TARGET_STM\TARGET_STM32F0\gpio_api.c 0x00000000   Number         0  mbed/TARGET_NUCLEO_F070RB/TOOLCHAIN_ARM_STD/gpio_api.o ABSOLUTE
    C:\Jenkins\workspace\mbed-2-build-library\targets\TARGET_STM\TARGET_STM32F0\gpio_irq_api.c 0x00000000   Number         0  mbed/TARGET_NUCLEO_F070RB/TOOLCHAIN_ARM_STD/gpio_irq_api.o ABSOLUTE
    C:\Jenkins\workspace\mbed-2-build-library\targets\TARGET_STM\TARGET_STM32F0\i2c_api.c 0x00000000   Number         0  mbed/TARGET_NUCLEO_F070RB/TOOLCHAIN_ARM_STD/i2c_api.o ABSOLUTE
    C:\Jenkins\workspace\mbed-2-build-library\targets\TARGET_STM\TARGET_STM32F0\lp_ticker.c 0x00000000   Number         0  mbed/TARGET_NUCLEO_F070RB/TOOLCHAIN_ARM_STD/lp_ticker.o ABSOLUTE
    C:\Jenkins\workspace\mbed-2-build-library\targets\TARGET_STM\TARGET_STM32F0\mbed_overrides.c 0x00000000   Number         0  mbed/TARGET_NUCLEO_F070RB/TOOLCHAIN_ARM_STD/mbed_overrides.o ABSOLUTE
    C:\Jenkins\workspace\mbed-2-build-library\targets\TARGET_STM\TARGET_STM32F0\pinmap.c 0x00000000   Number         0  mbed/TARGET_NUCLEO_F070RB/TOOLCHAIN_ARM_STD/pinmap.o ABSOLUTE
    C:\Jenkins\workspace\mbed-2-build-library\targets\TARGET_STM\TARGET_STM32F0\port_api.c 0x00000000   Number         0  mbed/TARGET_NUCLEO_F070RB/TOOLCHAIN_ARM_STD/port_api.o ABSOLUTE
    C:\Jenkins\workspace\mbed-2-build-library\targets\TARGET_STM\TARGET_STM32F0\pwmout_api.c 0x00000000   Number         0  mbed/TARGET_NUCLEO_F070RB/TOOLCHAIN_ARM_STD/pwmout_api.o ABSOLUTE
    C:\Jenkins\workspace\mbed-2-build-library\targets\TARGET_STM\TARGET_STM32F0\rtc_api.c 0x00000000   Number         0  mbed/TARGET_NUCLEO_F070RB/TOOLCHAIN_ARM_STD/rtc_api.o ABSOLUTE
    C:\Jenkins\workspace\mbed-2-build-library\targets\TARGET_STM\TARGET_STM32F0\serial_api.c 0x00000000   Number         0  mbed/TARGET_NUCLEO_F070RB/TOOLCHAIN_ARM_STD/serial_api.o ABSOLUTE
    C:\Jenkins\workspace\mbed-2-build-library\targets\TARGET_STM\TARGET_STM32F0\sleep.c 0x00000000   Number         0  mbed/TARGET_NUCLEO_F070RB/TOOLCHAIN_ARM_STD/sleep.o ABSOLUTE
    C:\Jenkins\workspace\mbed-2-build-library\targets\TARGET_STM\TARGET_STM32F0\spi_api.c 0x00000000   Number         0  mbed/TARGET_NUCLEO_F070RB/TOOLCHAIN_ARM_STD/spi_api.o ABSOLUTE
    C:\Jenkins\workspace\mbed-2-build-library\targets\TARGET_STM\TARGET_STM32F0\us_ticker.c 0x00000000   Number         0  mbed/TARGET_NUCLEO_F070RB/TOOLCHAIN_ARM_STD/us_ticker.o ABSOLUTE
    C:\Jenkins\workspace\mbed-2-build-library\targets\TARGET_STM\stm_spi_api.c 0x00000000   Number         0  mbed/TARGET_NUCLEO_F070RB/TOOLCHAIN_ARM_STD/stm_spi_api.o ABSOLUTE
    C:\Jenkins\workspace\mbed-2-build-library\targets\TARGET_STM\trng_api.c 0x00000000   Number         0  mbed/TARGET_NUCLEO_F070RB/TOOLCHAIN_ARM_STD/trng_api.o ABSOLUTE
    C:\\Jenkins\\workspace\\mbed-2-build-library\\drivers\\FileBase.cpp 0x00000000   Number         0  mbed/TARGET_NUCLEO_F070RB/TOOLCHAIN_ARM_STD/mbed.ar(FileBase.o) ABSOLUTE
    C:\\Jenkins\\workspace\\mbed-2-build-library\\drivers\\FileLike.cpp 0x00000000   Number         0  mbed/TARGET_NUCLEO_F070RB/TOOLCHAIN_ARM_STD/mbed.ar(FileLike.o) ABSOLUTE
    C:\\Jenkins\\workspace\\mbed-2-build-library\\drivers\\FilePath.cpp 0x00000000   Number         0  mbed/TARGET_NUCLEO_F070RB/TOOLCHAIN_ARM_STD/mbed.ar(FilePath.o) ABSOLUTE
    C:\\Jenkins\\workspace\\mbed-2-build-library\\drivers\\FileSystemLike.cpp 0x00000000   Number         0  mbed/TARGET_NUCLEO_F070RB/TOOLCHAIN_ARM_STD/mbed.ar(FileSystemLike.o) ABSOLUTE
    C:\\Jenkins\\workspace\\mbed-2-build-library\\drivers\\RawSerial.cpp 0x00000000   Number         0  mbed/TARGET_NUCLEO_F070RB/TOOLCHAIN_ARM_STD/mbed.ar(RawSerial.o) ABSOLUTE
    C:\\Jenkins\\workspace\\mbed-2-build-library\\drivers\\Serial.cpp 0x00000000   Number         0  mbed/TARGET_NUCLEO_F070RB/TOOLCHAIN_ARM_STD/mbed.ar(Serial.o) ABSOLUTE
    C:\\Jenkins\\workspace\\mbed-2-build-library\\drivers\\SerialBase.cpp 0x00000000   Number         0  mbed/TARGET_NUCLEO_F070RB/TOOLCHAIN_ARM_STD/mbed.ar(SerialBase.o) ABSOLUTE
    C:\\Jenkins\\workspace\\mbed-2-build-library\\drivers\\Stream.cpp 0x00000000   Number         0  mbed/TARGET_NUCLEO_F070RB/TOOLCHAIN_ARM_STD/mbed.ar(Stream.o) ABSOLUTE
    C:\\Jenkins\\workspace\\mbed-2-build-library\\drivers\\Ticker.cpp 0x00000000   Number         0  mbed/TARGET_NUCLEO_F070RB/TOOLCHAIN_ARM_STD/mbed.ar(Ticker.o) ABSOLUTE
    C:\\Jenkins\\workspace\\mbed-2-build-library\\drivers\\Timer.cpp 0x00000000   Number         0  mbed/TARGET_NUCLEO_F070RB/TOOLCHAIN_ARM_STD/mbed.ar(Timer.o) ABSOLUTE
    C:\\Jenkins\\workspace\\mbed-2-build-library\\drivers\\TimerEvent.cpp 0x00000000   Number         0  mbed/TARGET_NUCLEO_F070RB/TOOLCHAIN_ARM_STD/mbed.ar(TimerEvent.o) ABSOLUTE
    C:\\Jenkins\\workspace\\mbed-2-build-library\\hal\\mbed_gpio.c 0x00000000   Number         0  mbed/TARGET_NUCLEO_F070RB/TOOLCHAIN_ARM_STD/mbed.ar(mbed_gpio.o) ABSOLUTE
    C:\\Jenkins\\workspace\\mbed-2-build-library\\hal\\mbed_lp_ticker_api.c 0x00000000   Number         0  mbed/TARGET_NUCLEO_F070RB/TOOLCHAIN_ARM_STD/mbed.ar(mbed_lp_ticker_api.o) ABSOLUTE
    C:\\Jenkins\\workspace\\mbed-2-build-library\\hal\\mbed_pinmap_common.c 0x00000000   Number         0  mbed/TARGET_NUCLEO_F070RB/TOOLCHAIN_ARM_STD/mbed.ar(mbed_pinmap_common.o) ABSOLUTE
    C:\\Jenkins\\workspace\\mbed-2-build-library\\hal\\mbed_ticker_api.c 0x00000000   Number         0  mbed/TARGET_NUCLEO_F070RB/TOOLCHAIN_ARM_STD/mbed.ar(mbed_ticker_api.o) ABSOLUTE
    C:\\Jenkins\\workspace\\mbed-2-build-library\\hal\\mbed_us_ticker_api.c 0x00000000   Number         0  mbed/TARGET_NUCLEO_F070RB/TOOLCHAIN_ARM_STD/mbed.ar(mbed_us_ticker_api.o) ABSOLUTE
    C:\\Jenkins\\workspace\\mbed-2-build-library\\platform\\mbed_assert.c 0x00000000   Number         0  mbed/TARGET_NUCLEO_F070RB/TOOLCHAIN_ARM_STD/mbed.ar(mbed_assert.o) ABSOLUTE
    C:\\Jenkins\\workspace\\mbed-2-build-library\\platform\\mbed_board.c 0x00000000   Number         0  mbed/TARGET_NUCLEO_F070RB/TOOLCHAIN_ARM_STD/mbed_board.o ABSOLUTE
    C:\\Jenkins\\workspace\\mbed-2-build-library\\platform\\mbed_critical.c 0x00000000   Number         0  mbed/TARGET_NUCLEO_F070RB/TOOLCHAIN_ARM_STD/mbed.ar(mbed_critical.o) ABSOLUTE
    C:\\Jenkins\\workspace\\mbed-2-build-library\\platform\\mbed_error.c 0x00000000   Number         0  mbed/TARGET_NUCLEO_F070RB/TOOLCHAIN_ARM_STD/mbed.ar(mbed_error.o) ABSOLUTE
    C:\\Jenkins\\workspace\\mbed-2-build-library\\platform\\mbed_wait_api_no_rtos.c 0x00000000   Number         0  mbed/TARGET_NUCLEO_F070RB/TOOLCHAIN_ARM_STD/mbed.ar(mbed_wait_api_no_rtos.o) ABSOLUTE
    C:\\Jenkins\\workspace\\mbed-2-build-library\\platform\\retarget.cpp 0x00000000   Number         0  mbed/TARGET_NUCLEO_F070RB/TOOLCHAIN_ARM_STD/retarget.o ABSOLUTE
    C:\\Jenkins\\workspace\\mbed-2-build-library\\targets\\TARGET_STM\\TARGET_STM32F0\\TARGET_NUCLEO_F070RB\\PeripheralPins.c 0x00000000   Number         0  mbed/TARGET_NUCLEO_F070RB/TOOLCHAIN_ARM_STD/PeripheralPins.o ABSOLUTE
    C:\\Jenkins\\workspace\\mbed-2-build-library\\targets\\TARGET_STM\\TARGET_STM32F0\\TARGET_NUCLEO_F070RB\\device\\TOOLCHAIN_ARM_STD\\startup_stm32f070xb.S 0x00000000   Number         0  mbed/TARGET_NUCLEO_F070RB/TOOLCHAIN_ARM_STD/startup_stm32f070xb.o ABSOLUTE
    C:\\Jenkins\\workspace\\mbed-2-build-library\\targets\\TARGET_STM\\TARGET_STM32F0\\TARGET_NUCLEO_F070RB\\device\\cmsis_nvic.c 0x00000000   Number         0  mbed/TARGET_NUCLEO_F070RB/TOOLCHAIN_ARM_STD/cmsis_nvic.o ABSOLUTE
    C:\\Jenkins\\workspace\\mbed-2-build-library\\targets\\TARGET_STM\\TARGET_STM32F0\\TARGET_NUCLEO_F070RB\\device\\hal_tick.c 0x00000000   Number         0  mbed/TARGET_NUCLEO_F070RB/TOOLCHAIN_ARM_STD/hal_tick.o ABSOLUTE
    C:\\Jenkins\\workspace\\mbed-2-build-library\\targets\\TARGET_STM\\TARGET_STM32F0\\TARGET_NUCLEO_F070RB\\device\\system_stm32f0xx.c 0x00000000   Number         0  mbed/TARGET_NUCLEO_F070RB/TOOLCHAIN_ARM_STD/system_stm32f0xx.o ABSOLUTE
    C:\\Jenkins\\workspace\\mbed-2-build-library\\targets\\TARGET_STM\\TARGET_STM32F0\\analogin_api.c 0x00000000   Number         0  mbed/TARGET_NUCLEO_F070RB/TOOLCHAIN_ARM_STD/analogin_api.o ABSOLUTE
    C:\\Jenkins\\workspace\\mbed-2-build-library\\targets\\TARGET_STM\\TARGET_STM32F0\\analogout_api.c 0x00000000   Number         0  mbed/TARGET_NUCLEO_F070RB/TOOLCHAIN_ARM_STD/analogout_api.o ABSOLUTE
    C:\\Jenkins\\workspace\\mbed-2-build-library\\targets\\TARGET_STM\\TARGET_STM32F0\\can_api.c 0x00000000   Number         0  mbed/TARGET_NUCLEO_F070RB/TOOLCHAIN_ARM_STD/can_api.o ABSOLUTE
    C:\\Jenkins\\workspace\\mbed-2-build-library\\targets\\TARGET_STM\\TARGET_STM32F0\\device\\stm32f0xx_hal.c 0x00000000   Number         0  mbed/TARGET_NUCLEO_F070RB/TOOLCHAIN_ARM_STD/stm32f0xx_hal.o ABSOLUTE
    C:\\Jenkins\\workspace\\mbed-2-build-library\\targets\\TARGET_STM\\TARGET_STM32F0\\device\\stm32f0xx_hal_adc.c 0x00000000   Number         0  mbed/TARGET_NUCLEO_F070RB/TOOLCHAIN_ARM_STD/stm32f0xx_hal_adc.o ABSOLUTE
    C:\\Jenkins\\workspace\\mbed-2-build-library\\targets\\TARGET_STM\\TARGET_STM32F0\\device\\stm32f0xx_hal_adc_ex.c 0x00000000   Number         0  mbed/TARGET_NUCLEO_F070RB/TOOLCHAIN_ARM_STD/stm32f0xx_hal_adc_ex.o ABSOLUTE
    C:\\Jenkins\\workspace\\mbed-2-build-library\\targets\\TARGET_STM\\TARGET_STM32F0\\device\\stm32f0xx_hal_can.c 0x00000000   Number         0  mbed/TARGET_NUCLEO_F070RB/TOOLCHAIN_ARM_STD/stm32f0xx_hal_can.o ABSOLUTE
    C:\\Jenkins\\workspace\\mbed-2-build-library\\targets\\TARGET_STM\\TARGET_STM32F0\\device\\stm32f0xx_hal_cec.c 0x00000000   Number         0  mbed/TARGET_NUCLEO_F070RB/TOOLCHAIN_ARM_STD/stm32f0xx_hal_cec.o ABSOLUTE
    C:\\Jenkins\\workspace\\mbed-2-build-library\\targets\\TARGET_STM\\TARGET_STM32F0\\device\\stm32f0xx_hal_comp.c 0x00000000   Number         0  mbed/TARGET_NUCLEO_F070RB/TOOLCHAIN_ARM_STD/stm32f0xx_hal_comp.o ABSOLUTE
    C:\\Jenkins\\workspace\\mbed-2-build-library\\targets\\TARGET_STM\\TARGET_STM32F0\\device\\stm32f0xx_hal_cortex.c 0x00000000   Number         0  mbed/TARGET_NUCLEO_F070RB/TOOLCHAIN_ARM_STD/stm32f0xx_hal_cortex.o ABSOLUTE
    C:\\Jenkins\\workspace\\mbed-2-build-library\\targets\\TARGET_STM\\TARGET_STM32F0\\device\\stm32f0xx_hal_crc.c 0x00000000   Number         0  mbed/TARGET_NUCLEO_F070RB/TOOLCHAIN_ARM_STD/stm32f0xx_hal_crc.o ABSOLUTE
    C:\\Jenkins\\workspace\\mbed-2-build-library\\targets\\TARGET_STM\\TARGET_STM32F0\\device\\stm32f0xx_hal_crc_ex.c 0x00000000   Number         0  mbed/TARGET_NUCLEO_F070RB/TOOLCHAIN_ARM_STD/stm32f0xx_hal_crc_ex.o ABSOLUTE
    C:\\Jenkins\\workspace\\mbed-2-build-library\\targets\\TARGET_STM\\TARGET_STM32F0\\device\\stm32f0xx_hal_dac.c 0x00000000   Number         0  mbed/TARGET_NUCLEO_F070RB/TOOLCHAIN_ARM_STD/stm32f0xx_hal_dac.o ABSOLUTE
    C:\\Jenkins\\workspace\\mbed-2-build-library\\targets\\TARGET_STM\\TARGET_STM32F0\\device\\stm32f0xx_hal_dac_ex.c 0x00000000   Number         0  mbed/TARGET_NUCLEO_F070RB/TOOLCHAIN_ARM_STD/stm32f0xx_hal_dac_ex.o ABSOLUTE
    C:\\Jenkins\\workspace\\mbed-2-build-library\\targets\\TARGET_STM\\TARGET_STM32F0\\device\\stm32f0xx_hal_dma.c 0x00000000   Number         0  mbed/TARGET_NUCLEO_F070RB/TOOLCHAIN_ARM_STD/stm32f0xx_hal_dma.o ABSOLUTE
    C:\\Jenkins\\workspace\\mbed-2-build-library\\targets\\TARGET_STM\\TARGET_STM32F0\\device\\stm32f0xx_hal_flash.c 0x00000000   Number         0  mbed/TARGET_NUCLEO_F070RB/TOOLCHAIN_ARM_STD/stm32f0xx_hal_flash.o ABSOLUTE
    C:\\Jenkins\\workspace\\mbed-2-build-library\\targets\\TARGET_STM\\TARGET_STM32F0\\device\\stm32f0xx_hal_flash_ex.c 0x00000000   Number         0  mbed/TARGET_NUCLEO_F070RB/TOOLCHAIN_ARM_STD/stm32f0xx_hal_flash_ex.o ABSOLUTE
    C:\\Jenkins\\workspace\\mbed-2-build-library\\targets\\TARGET_STM\\TARGET_STM32F0\\device\\stm32f0xx_hal_gpio.c 0x00000000   Number         0  mbed/TARGET_NUCLEO_F070RB/TOOLCHAIN_ARM_STD/stm32f0xx_hal_gpio.o ABSOLUTE
    C:\\Jenkins\\workspace\\mbed-2-build-library\\targets\\TARGET_STM\\TARGET_STM32F0\\device\\stm32f0xx_hal_i2c.c 0x00000000   Number         0  mbed/TARGET_NUCLEO_F070RB/TOOLCHAIN_ARM_STD/stm32f0xx_hal_i2c.o ABSOLUTE
    C:\\Jenkins\\workspace\\mbed-2-build-library\\targets\\TARGET_STM\\TARGET_STM32F0\\device\\stm32f0xx_hal_i2c_ex.c 0x00000000   Number         0  mbed/TARGET_NUCLEO_F070RB/TOOLCHAIN_ARM_STD/stm32f0xx_hal_i2c_ex.o ABSOLUTE
    C:\\Jenkins\\workspace\\mbed-2-build-library\\targets\\TARGET_STM\\TARGET_STM32F0\\device\\stm32f0xx_hal_i2s.c 0x00000000   Number         0  mbed/TARGET_NUCLEO_F070RB/TOOLCHAIN_ARM_STD/stm32f0xx_hal_i2s.o ABSOLUTE
    C:\\Jenkins\\workspace\\mbed-2-build-library\\targets\\TARGET_STM\\TARGET_STM32F0\\device\\stm32f0xx_hal_irda.c 0x00000000   Number         0  mbed/TARGET_NUCLEO_F070RB/TOOLCHAIN_ARM_STD/stm32f0xx_hal_irda.o ABSOLUTE
    C:\\Jenkins\\workspace\\mbed-2-build-library\\targets\\TARGET_STM\\TARGET_STM32F0\\device\\stm32f0xx_hal_iwdg.c 0x00000000   Number         0  mbed/TARGET_NUCLEO_F070RB/TOOLCHAIN_ARM_STD/stm32f0xx_hal_iwdg.o ABSOLUTE
    C:\\Jenkins\\workspace\\mbed-2-build-library\\targets\\TARGET_STM\\TARGET_STM32F0\\device\\stm32f0xx_hal_pcd.c 0x00000000   Number         0  mbed/TARGET_NUCLEO_F070RB/TOOLCHAIN_ARM_STD/stm32f0xx_hal_pcd.o ABSOLUTE
    C:\\Jenkins\\workspace\\mbed-2-build-library\\targets\\TARGET_STM\\TARGET_STM32F0\\device\\stm32f0xx_hal_pcd_ex.c 0x00000000   Number         0  mbed/TARGET_NUCLEO_F070RB/TOOLCHAIN_ARM_STD/stm32f0xx_hal_pcd_ex.o ABSOLUTE
    C:\\Jenkins\\workspace\\mbed-2-build-library\\targets\\TARGET_STM\\TARGET_STM32F0\\device\\stm32f0xx_hal_pwr.c 0x00000000   Number         0  mbed/TARGET_NUCLEO_F070RB/TOOLCHAIN_ARM_STD/stm32f0xx_hal_pwr.o ABSOLUTE
    C:\\Jenkins\\workspace\\mbed-2-build-library\\targets\\TARGET_STM\\TARGET_STM32F0\\device\\stm32f0xx_hal_pwr_ex.c 0x00000000   Number         0  mbed/TARGET_NUCLEO_F070RB/TOOLCHAIN_ARM_STD/stm32f0xx_hal_pwr_ex.o ABSOLUTE
    C:\\Jenkins\\workspace\\mbed-2-build-library\\targets\\TARGET_STM\\TARGET_STM32F0\\device\\stm32f0xx_hal_rcc.c 0x00000000   Number         0  mbed/TARGET_NUCLEO_F070RB/TOOLCHAIN_ARM_STD/stm32f0xx_hal_rcc.o ABSOLUTE
    C:\\Jenkins\\workspace\\mbed-2-build-library\\targets\\TARGET_STM\\TARGET_STM32F0\\device\\stm32f0xx_hal_rcc_ex.c 0x00000000   Number         0  mbed/TARGET_NUCLEO_F070RB/TOOLCHAIN_ARM_STD/stm32f0xx_hal_rcc_ex.o ABSOLUTE
    C:\\Jenkins\\workspace\\mbed-2-build-library\\targets\\TARGET_STM\\TARGET_STM32F0\\device\\stm32f0xx_hal_rtc.c 0x00000000   Number         0  mbed/TARGET_NUCLEO_F070RB/TOOLCHAIN_ARM_STD/stm32f0xx_hal_rtc.o ABSOLUTE
    C:\\Jenkins\\workspace\\mbed-2-build-library\\targets\\TARGET_STM\\TARGET_STM32F0\\device\\stm32f0xx_hal_rtc_ex.c 0x00000000   Number         0  mbed/TARGET_NUCLEO_F070RB/TOOLCHAIN_ARM_STD/stm32f0xx_hal_rtc_ex.o ABSOLUTE
    C:\\Jenkins\\workspace\\mbed-2-build-library\\targets\\TARGET_STM\\TARGET_STM32F0\\device\\stm32f0xx_hal_smartcard.c 0x00000000   Number         0  mbed/TARGET_NUCLEO_F070RB/TOOLCHAIN_ARM_STD/stm32f0xx_hal_smartcard.o ABSOLUTE
    C:\\Jenkins\\workspace\\mbed-2-build-library\\targets\\TARGET_STM\\TARGET_STM32F0\\device\\stm32f0xx_hal_smartcard_ex.c 0x00000000   Number         0  mbed/TARGET_NUCLEO_F070RB/TOOLCHAIN_ARM_STD/stm32f0xx_hal_smartcard_ex.o ABSOLUTE
    C:\\Jenkins\\workspace\\mbed-2-build-library\\targets\\TARGET_STM\\TARGET_STM32F0\\device\\stm32f0xx_hal_smbus.c 0x00000000   Number         0  mbed/TARGET_NUCLEO_F070RB/TOOLCHAIN_ARM_STD/stm32f0xx_hal_smbus.o ABSOLUTE
    C:\\Jenkins\\workspace\\mbed-2-build-library\\targets\\TARGET_STM\\TARGET_STM32F0\\device\\stm32f0xx_hal_spi.c 0x00000000   Number         0  mbed/TARGET_NUCLEO_F070RB/TOOLCHAIN_ARM_STD/stm32f0xx_hal_spi.o ABSOLUTE
    C:\\Jenkins\\workspace\\mbed-2-build-library\\targets\\TARGET_STM\\TARGET_STM32F0\\device\\stm32f0xx_hal_spi_ex.c 0x00000000   Number         0  mbed/TARGET_NUCLEO_F070RB/TOOLCHAIN_ARM_STD/stm32f0xx_hal_spi_ex.o ABSOLUTE
    C:\\Jenkins\\workspace\\mbed-2-build-library\\targets\\TARGET_STM\\TARGET_STM32F0\\device\\stm32f0xx_hal_tim.c 0x00000000   Number         0  mbed/TARGET_NUCLEO_F070RB/TOOLCHAIN_ARM_STD/stm32f0xx_hal_tim.o ABSOLUTE
    C:\\Jenkins\\workspace\\mbed-2-build-library\\targets\\TARGET_STM\\TARGET_STM32F0\\device\\stm32f0xx_hal_tim_ex.c 0x00000000   Number         0  mbed/TARGET_NUCLEO_F070RB/TOOLCHAIN_ARM_STD/stm32f0xx_hal_tim_ex.o ABSOLUTE
    C:\\Jenkins\\workspace\\mbed-2-build-library\\targets\\TARGET_STM\\TARGET_STM32F0\\device\\stm32f0xx_hal_tsc.c 0x00000000   Number         0  mbed/TARGET_NUCLEO_F070RB/TOOLCHAIN_ARM_STD/stm32f0xx_hal_tsc.o ABSOLUTE
    C:\\Jenkins\\workspace\\mbed-2-build-library\\targets\\TARGET_STM\\TARGET_STM32F0\\device\\stm32f0xx_hal_uart.c 0x00000000   Number         0  mbed/TARGET_NUCLEO_F070RB/TOOLCHAIN_ARM_STD/stm32f0xx_hal_uart.o ABSOLUTE
    C:\\Jenkins\\workspace\\mbed-2-build-library\\targets\\TARGET_STM\\TARGET_STM32F0\\device\\stm32f0xx_hal_uart_ex.c 0x00000000   Number         0  mbed/TARGET_NUCLEO_F070RB/TOOLCHAIN_ARM_STD/stm32f0xx_hal_uart_ex.o ABSOLUTE
    C:\\Jenkins\\workspace\\mbed-2-build-library\\targets\\TARGET_STM\\TARGET_STM32F0\\device\\stm32f0xx_hal_usart.c 0x00000000   Number         0  mbed/TARGET_NUCLEO_F070RB/TOOLCHAIN_ARM_STD/stm32f0xx_hal_usart.o ABSOLUTE
    C:\\Jenkins\\workspace\\mbed-2-build-library\\targets\\TARGET_STM\\TARGET_STM32F0\\device\\stm32f0xx_hal_wwdg.c 0x00000000   Number         0  mbed/TARGET_NUCLEO_F070RB/TOOLCHAIN_ARM_STD/stm32f0xx_hal_wwdg.o ABSOLUTE
    C:\\Jenkins\\workspace\\mbed-2-build-library\\targets\\TARGET_STM\\TARGET_STM32F0\\gpio_api.c 0x00000000   Number         0  mbed/TARGET_NUCLEO_F070RB/TOOLCHAIN_ARM_STD/gpio_api.o ABSOLUTE
    C:\\Jenkins\\workspace\\mbed-2-build-library\\targets\\TARGET_STM\\TARGET_STM32F0\\gpio_irq_api.c 0x00000000   Number         0  mbed/TARGET_NUCLEO_F070RB/TOOLCHAIN_ARM_STD/gpio_irq_api.o ABSOLUTE
    C:\\Jenkins\\workspace\\mbed-2-build-library\\targets\\TARGET_STM\\TARGET_STM32F0\\i2c_api.c 0x00000000   Number         0  mbed/TARGET_NUCLEO_F070RB/TOOLCHAIN_ARM_STD/i2c_api.o ABSOLUTE
    C:\\Jenkins\\workspace\\mbed-2-build-library\\targets\\TARGET_STM\\TARGET_STM32F0\\lp_ticker.c 0x00000000   Number         0  mbed/TARGET_NUCLEO_F070RB/TOOLCHAIN_ARM_STD/lp_ticker.o ABSOLUTE
    C:\\Jenkins\\workspace\\mbed-2-build-library\\targets\\TARGET_STM\\TARGET_STM32F0\\mbed_overrides.c 0x00000000   Number         0  mbed/TARGET_NUCLEO_F070RB/TOOLCHAIN_ARM_STD/mbed_overrides.o ABSOLUTE
    C:\\Jenkins\\workspace\\mbed-2-build-library\\targets\\TARGET_STM\\TARGET_STM32F0\\pinmap.c 0x00000000   Number         0  mbed/TARGET_NUCLEO_F070RB/TOOLCHAIN_ARM_STD/pinmap.o ABSOLUTE
    C:\\Jenkins\\workspace\\mbed-2-build-library\\targets\\TARGET_STM\\TARGET_STM32F0\\port_api.c 0x00000000   Number         0  mbed/TARGET_NUCLEO_F070RB/TOOLCHAIN_ARM_STD/port_api.o ABSOLUTE
    C:\\Jenkins\\workspace\\mbed-2-build-library\\targets\\TARGET_STM\\TARGET_STM32F0\\pwmout_api.c 0x00000000   Number         0  mbed/TARGET_NUCLEO_F070RB/TOOLCHAIN_ARM_STD/pwmout_api.o ABSOLUTE
    C:\\Jenkins\\workspace\\mbed-2-build-library\\targets\\TARGET_STM\\TARGET_STM32F0\\rtc_api.c 0x00000000   Number         0  mbed/TARGET_NUCLEO_F070RB/TOOLCHAIN_ARM_STD/rtc_api.o ABSOLUTE
    C:\\Jenkins\\workspace\\mbed-2-build-library\\targets\\TARGET_STM\\TARGET_STM32F0\\serial_api.c 0x00000000   Number         0  mbed/TARGET_NUCLEO_F070RB/TOOLCHAIN_ARM_STD/serial_api.o ABSOLUTE
    C:\\Jenkins\\workspace\\mbed-2-build-library\\targets\\TARGET_STM\\TARGET_STM32F0\\sleep.c 0x00000000   Number         0  mbed/TARGET_NUCLEO_F070RB/TOOLCHAIN_ARM_STD/sleep.o ABSOLUTE
    C:\\Jenkins\\workspace\\mbed-2-build-library\\targets\\TARGET_STM\\TARGET_STM32F0\\spi_api.c 0x00000000   Number         0  mbed/TARGET_NUCLEO_F070RB/TOOLCHAIN_ARM_STD/spi_api.o ABSOLUTE
    C:\\Jenkins\\workspace\\mbed-2-build-library\\targets\\TARGET_STM\\TARGET_STM32F0\\us_ticker.c 0x00000000   Number         0  mbed/TARGET_NUCLEO_F070RB/TOOLCHAIN_ARM_STD/us_ticker.o ABSOLUTE
    C:\\Jenkins\\workspace\\mbed-2-build-library\\targets\\TARGET_STM\\stm_spi_api.c 0x00000000   Number         0  mbed/TARGET_NUCLEO_F070RB/TOOLCHAIN_ARM_STD/stm_spi_api.o ABSOLUTE
    MyBuffer.cpp                             0x00000000   Number         0  .\build\mybuffer.o ABSOLUTE
    MyBuffer.cpp                             0x00000000   Number         0  .\build\mybuffer.o ABSOLUTE
    RFID.cpp                                 0x00000000   Number         0  .\build\rfid.o ABSOLUTE
    RFID.cpp                                 0x00000000   Number         0  .\build\rfid.o ABSOLUTE
    dc.s                                     0x00000000   Number         0  C:\Keil_v5\ARM\ARMCC\Bin\..\lib\armlib\c_p.l(dc.o) ABSOLUTE
    main.cpp                                 0x00000000   Number         0  .\build\main.o ABSOLUTE
    main.cpp                                 0x00000000   Number         0  .\build\main.o ABSOLUTE
    RESET                                    0x08000000   Section      192  mbed/TARGET_NUCLEO_F070RB/TOOLCHAIN_ARM_STD/startup_stm32f070xb.o(RESET)
    !!!main                                  0x080000c0   Section        8  C:\Keil_v5\ARM\ARMCC\Bin\..\lib\armlib\c_p.l(__main.o)(!!!main)
    !!!scatter                               0x080000c8   Section       60  C:\Keil_v5\ARM\ARMCC\Bin\..\lib\armlib\c_p.l(__scatter.o)(!!!scatter)
    !!handler_copy                           0x08000104   Section       26  C:\Keil_v5\ARM\ARMCC\Bin\..\lib\armlib\c_p.l(__scatter_copy.o)(!!handler_copy)
    !!handler_zi                             0x08000120   Section       28  C:\Keil_v5\ARM\ARMCC\Bin\..\lib\armlib\c_p.l(__scatter_zi.o)(!!handler_zi)
    .ARM.Collect$$_printf_percent$$00000000  0x0800013c   Section        2  C:\Keil_v5\ARM\ARMCC\Bin\..\lib\armlib\c_p.l(_printf_percent.o)(.ARM.Collect$$_printf_percent$$00000000)
    .ARM.Collect$$_printf_percent$$00000001  0x0800013e   Section       10  C:\Keil_v5\ARM\ARMCC\Bin\..\lib\armlib\c_p.l(_printf_n.o)(.ARM.Collect$$_printf_percent$$00000001)
    .ARM.Collect$$_printf_percent$$00000002  0x08000148   Section       10  C:\Keil_v5\ARM\ARMCC\Bin\..\lib\armlib\c_p.l(_printf_p.o)(.ARM.Collect$$_printf_percent$$00000002)
    .ARM.Collect$$_printf_percent$$00000003  0x08000152   Section       10  C:\Keil_v5\ARM\ARMCC\Bin\..\lib\armlib\c_p.l(_printf_f.o)(.ARM.Collect$$_printf_percent$$00000003)
    .ARM.Collect$$_printf_percent$$00000004  0x0800015c   Section       10  C:\Keil_v5\ARM\ARMCC\Bin\..\lib\armlib\c_p.l(_printf_e.o)(.ARM.Collect$$_printf_percent$$00000004)
    .ARM.Collect$$_printf_percent$$00000005  0x08000166   Section       10  C:\Keil_v5\ARM\ARMCC\Bin\..\lib\armlib\c_p.l(_printf_g.o)(.ARM.Collect$$_printf_percent$$00000005)
    .ARM.Collect$$_printf_percent$$00000006  0x08000170   Section       10  C:\Keil_v5\ARM\ARMCC\Bin\..\lib\armlib\c_p.l(_printf_a.o)(.ARM.Collect$$_printf_percent$$00000006)
    .ARM.Collect$$_printf_percent$$00000007  0x0800017a   Section       10  C:\Keil_v5\ARM\ARMCC\Bin\..\lib\armlib\c_p.l(_printf_ll.o)(.ARM.Collect$$_printf_percent$$00000007)
    .ARM.Collect$$_printf_percent$$00000008  0x08000184   Section       10  C:\Keil_v5\ARM\ARMCC\Bin\..\lib\armlib\c_p.l(_printf_i.o)(.ARM.Collect$$_printf_percent$$00000008)
    .ARM.Collect$$_printf_percent$$00000009  0x0800018e   Section       10  C:\Keil_v5\ARM\ARMCC\Bin\..\lib\armlib\c_p.l(_printf_d.o)(.ARM.Collect$$_printf_percent$$00000009)
    .ARM.Collect$$_printf_percent$$0000000A  0x08000198   Section       10  C:\Keil_v5\ARM\ARMCC\Bin\..\lib\armlib\c_p.l(_printf_u.o)(.ARM.Collect$$_printf_percent$$0000000A)
    .ARM.Collect$$_printf_percent$$0000000B  0x080001a2   Section       10  C:\Keil_v5\ARM\ARMCC\Bin\..\lib\armlib\c_p.l(_printf_o.o)(.ARM.Collect$$_printf_percent$$0000000B)
    .ARM.Collect$$_printf_percent$$0000000C  0x080001ac   Section       10  C:\Keil_v5\ARM\ARMCC\Bin\..\lib\armlib\c_p.l(_printf_x.o)(.ARM.Collect$$_printf_percent$$0000000C)
    .ARM.Collect$$_printf_percent$$0000000D  0x080001b6   Section       10  C:\Keil_v5\ARM\ARMCC\Bin\..\lib\armlib\c_p.l(_printf_lli.o)(.ARM.Collect$$_printf_percent$$0000000D)
    .ARM.Collect$$_printf_percent$$0000000E  0x080001c0   Section       10  C:\Keil_v5\ARM\ARMCC\Bin\..\lib\armlib\c_p.l(_printf_lld.o)(.ARM.Collect$$_printf_percent$$0000000E)
    .ARM.Collect$$_printf_percent$$0000000F  0x080001ca   Section       10  C:\Keil_v5\ARM\ARMCC\Bin\..\lib\armlib\c_p.l(_printf_llu.o)(.ARM.Collect$$_printf_percent$$0000000F)
    .ARM.Collect$$_printf_percent$$00000010  0x080001d4   Section       10  C:\Keil_v5\ARM\ARMCC\Bin\..\lib\armlib\c_p.l(_printf_llo.o)(.ARM.Collect$$_printf_percent$$00000010)
    .ARM.Collect$$_printf_percent$$00000011  0x080001de   Section       10  C:\Keil_v5\ARM\ARMCC\Bin\..\lib\armlib\c_p.l(_printf_llx.o)(.ARM.Collect$$_printf_percent$$00000011)
    .ARM.Collect$$_printf_percent$$00000012  0x080001e8   Section       10  C:\Keil_v5\ARM\ARMCC\Bin\..\lib\armlib\c_p.l(_printf_l.o)(.ARM.Collect$$_printf_percent$$00000012)
    .ARM.Collect$$_printf_percent$$00000013  0x080001f2   Section       10  C:\Keil_v5\ARM\ARMCC\Bin\..\lib\armlib\c_p.l(_printf_c.o)(.ARM.Collect$$_printf_percent$$00000013)
    .ARM.Collect$$_printf_percent$$00000014  0x080001fc   Section       10  C:\Keil_v5\ARM\ARMCC\Bin\..\lib\armlib\c_p.l(_printf_s.o)(.ARM.Collect$$_printf_percent$$00000014)
    .ARM.Collect$$_printf_percent$$00000015  0x08000206   Section       10  C:\Keil_v5\ARM\ARMCC\Bin\..\lib\armlib\c_p.l(_printf_lc.o)(.ARM.Collect$$_printf_percent$$00000015)
    .ARM.Collect$$_printf_percent$$00000016  0x08000210   Section       10  C:\Keil_v5\ARM\ARMCC\Bin\..\lib\armlib\c_p.l(_printf_ls.o)(.ARM.Collect$$_printf_percent$$00000016)
    .ARM.Collect$$_printf_percent$$00000017  0x0800021a   Section        4  C:\Keil_v5\ARM\ARMCC\Bin\..\lib\armlib\c_p.l(_printf_percent_end.o)(.ARM.Collect$$_printf_percent$$00000017)
    .ARM.Collect$$libinit$$00000000          0x0800021e   Section        2  C:\Keil_v5\ARM\ARMCC\Bin\..\lib\armlib\c_p.l(libinit.o)(.ARM.Collect$$libinit$$00000000)
    .ARM.Collect$$libinit$$00000002          0x08000220   Section        0  C:\Keil_v5\ARM\ARMCC\Bin\..\lib\armlib\c_p.l(libinit2.o)(.ARM.Collect$$libinit$$00000002)
    .ARM.Collect$$libinit$$00000004          0x08000220   Section        0  C:\Keil_v5\ARM\ARMCC\Bin\..\lib\armlib\c_p.l(libinit2.o)(.ARM.Collect$$libinit$$00000004)
    .ARM.Collect$$libinit$$00000005          0x08000220   Section        8  C:\Keil_v5\ARM\ARMCC\Bin\..\lib\armlib\c_p.l(libinit2.o)(.ARM.Collect$$libinit$$00000005)
    .ARM.Collect$$libinit$$0000000A          0x08000228   Section        0  C:\Keil_v5\ARM\ARMCC\Bin\..\lib\armlib\c_p.l(libinit2.o)(.ARM.Collect$$libinit$$0000000A)
    .ARM.Collect$$libinit$$0000000C          0x08000228   Section        0  C:\Keil_v5\ARM\ARMCC\Bin\..\lib\armlib\c_p.l(libinit2.o)(.ARM.Collect$$libinit$$0000000C)
    .ARM.Collect$$libinit$$0000000E          0x08000228   Section        0  C:\Keil_v5\ARM\ARMCC\Bin\..\lib\armlib\c_p.l(libinit2.o)(.ARM.Collect$$libinit$$0000000E)
    .ARM.Collect$$libinit$$0000000F          0x08000228   Section        6  C:\Keil_v5\ARM\ARMCC\Bin\..\lib\armlib\c_p.l(libinit2.o)(.ARM.Collect$$libinit$$0000000F)
    .ARM.Collect$$libinit$$00000011          0x0800022e   Section        0  C:\Keil_v5\ARM\ARMCC\Bin\..\lib\armlib\c_p.l(libinit2.o)(.ARM.Collect$$libinit$$00000011)
    .ARM.Collect$$libinit$$00000012          0x0800022e   Section       12  C:\Keil_v5\ARM\ARMCC\Bin\..\lib\armlib\c_p.l(libinit2.o)(.ARM.Collect$$libinit$$00000012)
    .ARM.Collect$$libinit$$00000013          0x0800023a   Section        0  C:\Keil_v5\ARM\ARMCC\Bin\..\lib\armlib\c_p.l(libinit2.o)(.ARM.Collect$$libinit$$00000013)
    .ARM.Collect$$libinit$$00000015          0x0800023a   Section        0  C:\Keil_v5\ARM\ARMCC\Bin\..\lib\armlib\c_p.l(libinit2.o)(.ARM.Collect$$libinit$$00000015)
    .ARM.Collect$$libinit$$00000016          0x0800023a   Section       10  C:\Keil_v5\ARM\ARMCC\Bin\..\lib\armlib\c_p.l(libinit2.o)(.ARM.Collect$$libinit$$00000016)
    .ARM.Collect$$libinit$$00000017          0x08000244   Section        0  C:\Keil_v5\ARM\ARMCC\Bin\..\lib\armlib\c_p.l(libinit2.o)(.ARM.Collect$$libinit$$00000017)
    .ARM.Collect$$libinit$$00000019          0x08000244   Section        0  C:\Keil_v5\ARM\ARMCC\Bin\..\lib\armlib\c_p.l(libinit2.o)(.ARM.Collect$$libinit$$00000019)
    .ARM.Collect$$libinit$$0000001B          0x08000244   Section        0  C:\Keil_v5\ARM\ARMCC\Bin\..\lib\armlib\c_p.l(libinit2.o)(.ARM.Collect$$libinit$$0000001B)
    .ARM.Collect$$libinit$$0000001D          0x08000244   Section        0  C:\Keil_v5\ARM\ARMCC\Bin\..\lib\armlib\c_p.l(libinit2.o)(.ARM.Collect$$libinit$$0000001D)
    .ARM.Collect$$libinit$$0000001F          0x08000244   Section        0  C:\Keil_v5\ARM\ARMCC\Bin\..\lib\armlib\c_p.l(libinit2.o)(.ARM.Collect$$libinit$$0000001F)
    .ARM.Collect$$libinit$$00000021          0x08000244   Section        0  C:\Keil_v5\ARM\ARMCC\Bin\..\lib\armlib\c_p.l(libinit2.o)(.ARM.Collect$$libinit$$00000021)
    .ARM.Collect$$libinit$$00000023          0x08000244   Section        0  C:\Keil_v5\ARM\ARMCC\Bin\..\lib\armlib\c_p.l(libinit2.o)(.ARM.Collect$$libinit$$00000023)
    .ARM.Collect$$libinit$$00000024          0x08000244   Section        4  C:\Keil_v5\ARM\ARMCC\Bin\..\lib\armlib\c_p.l(libinit2.o)(.ARM.Collect$$libinit$$00000024)
    .ARM.Collect$$libinit$$00000025          0x08000248   Section        0  C:\Keil_v5\ARM\ARMCC\Bin\..\lib\armlib\c_p.l(libinit2.o)(.ARM.Collect$$libinit$$00000025)
    .ARM.Collect$$libinit$$0000002C          0x08000248   Section        0  C:\Keil_v5\ARM\ARMCC\Bin\..\lib\armlib\c_p.l(libinit2.o)(.ARM.Collect$$libinit$$0000002C)
    .ARM.Collect$$libinit$$0000002E          0x08000248   Section        0  C:\Keil_v5\ARM\ARMCC\Bin\..\lib\armlib\c_p.l(libinit2.o)(.ARM.Collect$$libinit$$0000002E)
    .ARM.Collect$$libinit$$00000030          0x08000248   Section        0  C:\Keil_v5\ARM\ARMCC\Bin\..\lib\armlib\c_p.l(libinit2.o)(.ARM.Collect$$libinit$$00000030)
    .ARM.Collect$$libinit$$00000031          0x08000248   Section        4  C:\Keil_v5\ARM\ARMCC\Bin\..\lib\armlib\c_p.l(libinit2.o)(.ARM.Collect$$libinit$$00000031)
    .ARM.Collect$$libinit$$00000032          0x0800024c   Section        0  C:\Keil_v5\ARM\ARMCC\Bin\..\lib\armlib\c_p.l(libinit2.o)(.ARM.Collect$$libinit$$00000032)
    .ARM.Collect$$libinit$$00000033          0x0800024c   Section        2  C:\Keil_v5\ARM\ARMCC\Bin\..\lib\armlib\c_p.l(libinit2.o)(.ARM.Collect$$libinit$$00000033)
    .ARM.Collect$$libshutdown$$00000004      0x0800024e   Section        0  C:\Keil_v5\ARM\ARMCC\Bin\..\lib\armlib\c_p.l(libshutdown2.o)(.ARM.Collect$$libshutdown$$00000004)
    .ARM.Collect$$rtentry$$00000000          0x0800024e   Section        0  C:\Keil_v5\ARM\ARMCC\Bin\..\lib\armlib\c_p.l(__rtentry.o)(.ARM.Collect$$rtentry$$00000000)
    .ARM.Collect$$rtentry$$00000002          0x0800024e   Section        0  C:\Keil_v5\ARM\ARMCC\Bin\..\lib\armlib\c_p.l(__rtentry2.o)(.ARM.Collect$$rtentry$$00000002)
    .ARM.Collect$$rtentry$$00000004          0x0800024e   Section        6  C:\Keil_v5\ARM\ARMCC\Bin\..\lib\armlib\c_p.l(__rtentry4.o)(.ARM.Collect$$rtentry$$00000004)
    .ARM.Collect$$rtentry$$00000008          0x08000254   Section        8  C:\Keil_v5\ARM\ARMCC\Bin\..\lib\armlib\c_p.l(__rtentry2.o)(.ARM.Collect$$rtentry$$00000008)
    .ARM.Collect$$rtentry$$0000000A          0x0800025c   Section        4  C:\Keil_v5\ARM\ARMCC\Bin\..\lib\armlib\c_p.l(__rtentry2.o)(.ARM.Collect$$rtentry$$0000000A)
    .ARM.Collect$$rtentry$$0000000C          0x08000260   Section        0  C:\Keil_v5\ARM\ARMCC\Bin\..\lib\armlib\c_p.l(__rtentry2.o)(.ARM.Collect$$rtentry$$0000000C)
    .ARM.Collect$$rtentry$$0000000D          0x08000260   Section        8  C:\Keil_v5\ARM\ARMCC\Bin\..\lib\armlib\c_p.l(__rtentry2.o)(.ARM.Collect$$rtentry$$0000000D)
    .emb_text                                0x08000268   Section       56  C:\Keil_v5\ARM\ARMCC\Bin\..\lib\armlib\c_p.l(rt_memcpy.o)(.emb_text)
    .emb_text                                0x080002a0   Section        0  C:\Keil_v5\ARM\ARMCC\Bin\..\lib\armlib\c_p.l(maybetermalloc1.o)(.emb_text)
    .text                                    0x080002a0   Section       28  mbed/TARGET_NUCLEO_F070RB/TOOLCHAIN_ARM_STD/startup_stm32f070xb.o(.text)
    .text                                    0x080002bc   Section        0  C:\Keil_v5\ARM\ARMCC\Bin\..\lib\armlib\c_p.l(h1_alloc.o)(.text)
    .text                                    0x0800031e   Section        0  C:\Keil_v5\ARM\ARMCC\Bin\..\lib\armlib\c_p.l(h1_free.o)(.text)
    .text                                    0x0800036c   Section        0  C:\Keil_v5\ARM\ARMCC\Bin\..\lib\armlib\c_p.l(vsprintf.o)(.text)
    .text                                    0x08000390   Section        0  C:\Keil_v5\ARM\ARMCC\Bin\..\lib\armlib\c_p.l(c89vfprintf.o)(.text)
    .text                                    0x080003a0   Section        0  C:\Keil_v5\ARM\ARMCC\Bin\..\lib\armlib\c_p.l(__2sprintf.o)(.text)
    .text                                    0x080003cc   Section        0  C:\Keil_v5\ARM\ARMCC\Bin\..\lib\armlib\c_p.l(_printf_hex_int_ll_ptr.o)(.text)
    _printf_hex_common                       0x080003cd   Thumb Code     0  C:\Keil_v5\ARM\ARMCC\Bin\..\lib\armlib\c_p.l(_printf_hex_int_ll_ptr.o)(.text)
    .text                                    0x08000464   Section        0  C:\Keil_v5\ARM\ARMCC\Bin\..\lib\armlib\c_p.l(__printf_flags_ss_wp.o)(.text)
    .text                                    0x080005ec   Section        0  C:\Keil_v5\ARM\ARMCC\Bin\..\lib\armlib\c_p.l(__0sscanf.o)(.text)
    .text                                    0x0800062c   Section        0  C:\Keil_v5\ARM\ARMCC\Bin\..\lib\armlib\c_p.l(_scanf_int.o)(.text)
    .text                                    0x08000778   Section        0  C:\Keil_v5\ARM\ARMCC\Bin\..\lib\armlib\c_p.l(fflush.o)(.text)
    .text                                    0x080007e0   Section        0  C:\Keil_v5\ARM\ARMCC\Bin\..\lib\armlib\c_p.l(fopen.o)(.text)
    _freopen_locked                          0x080007e1   Thumb Code     0  C:\Keil_v5\ARM\ARMCC\Bin\..\lib\armlib\c_p.l(fopen.o)(.text)
    .text                                    0x080008c8   Section        0  C:\Keil_v5\ARM\ARMCC\Bin\..\lib\armlib\c_p.l(setbuf.o)(.text)
    .text                                    0x080008e4   Section        0  C:\Keil_v5\ARM\ARMCC\Bin\..\lib\armlib\c_p.l(fclose.o)(.text)
    .text                                    0x08000930   Section        0  C:\Keil_v5\ARM\ARMCC\Bin\..\lib\armlib\c_p.l(strlen.o)(.text)
    .text                                    0x08000974   Section        0  C:\Keil_v5\ARM\ARMCC\Bin\..\lib\armlib\c_p.l(strncmp.o)(.text)
    .text                                    0x08000a14   Section        0  C:\Keil_v5\ARM\ARMCC\Bin\..\lib\armlib\c_p.l(rt_memclr.o)(.text)
    .text                                    0x08000a54   Section      160  C:\Keil_v5\ARM\ARMCC\Bin\..\lib\armlib\c_p.l(strcmpv6m.o)(.text)
    .text                                    0x08000af4   Section      488  C:\Keil_v5\ARM\ARMCC\Bin\..\lib\armlib\c_p.l(aeabi_sdivfast.o)(.text)
    .text                                    0x08000cdc   Section        0  C:\Keil_v5\ARM\ARMCC\Bin\..\lib\armlib\c_p.l(init_aeabi.o)(.text)
    .text                                    0x08000d00   Section        0  C:\Keil_v5\ARM\ARMCC\Bin\..\lib\cpplib\cpprt_p.l(aeabi_vec_dtor_noexceptions.o)(.text)
    .text                                    0x08000d24   Section        0  C:\Keil_v5\ARM\ARMCC\Bin\..\lib\armlib\fz_ps.l(ddiv.o)(.text)
    .text                                    0x0800116c   Section        0  C:\Keil_v5\ARM\ARMCC\Bin\..\lib\armlib\fz_ps.l(dflti.o)(.text)
    .text                                    0x080011c4   Section        0  C:\Keil_v5\ARM\ARMCC\Bin\..\lib\armlib\fz_ps.l(dmul.o)(.text)
    .text                                    0x0800140c   Section        0  C:\Keil_v5\ARM\ARMCC\Bin\..\lib\armlib\fz_ps.l(f2d.o)(.text)
    .text                                    0x08001460   Section        0  C:\Keil_v5\ARM\ARMCC\Bin\..\lib\armlib\fz_ps.l(fdiv.o)(.text)
    .text                                    0x080015c0   Section        0  C:\Keil_v5\ARM\ARMCC\Bin\..\lib\armlib\fz_ps.l(fflti.o)(.text)
    .text                                    0x08001620   Section        8  C:\Keil_v5\ARM\ARMCC\Bin\..\lib\armlib\c_p.l(rt_heap_descriptor.o)(.text)
    .text                                    0x08001628   Section        0  C:\Keil_v5\ARM\ARMCC\Bin\..\lib\armlib\c_p.l(hguard.o)(.text)
    .text                                    0x0800162c   Section        0  C:\Keil_v5\ARM\ARMCC\Bin\..\lib\armlib\c_p.l(init_alloc.o)(.text)
    .text                                    0x080016b4   Section        0  C:\Keil_v5\ARM\ARMCC\Bin\..\lib\armlib\c_p.l(h1_init.o)(.text)
    .text                                    0x080016c2   Section        0  C:\Keil_v5\ARM\ARMCC\Bin\..\lib\armlib\c_p.l(_printf_pad.o)(.text)
    .text                                    0x08001710   Section        0  C:\Keil_v5\ARM\ARMCC\Bin\..\lib\armlib\c_p.l(_printf_truncate.o)(.text)
    .text                                    0x08001734   Section        0  C:\Keil_v5\ARM\ARMCC\Bin\..\lib\armlib\c_p.l(_printf_str.o)(.text)
    .text                                    0x08001786   Section        0  C:\Keil_v5\ARM\ARMCC\Bin\..\lib\armlib\c_p.l(_printf_intcommon.o)(.text)
    .text                                    0x08001838   Section        0  C:\Keil_v5\ARM\ARMCC\Bin\..\lib\armlib\c_p.l(_printf_dec.o)(.text)
    .text                                    0x080018a4   Section        0  C:\Keil_v5\ARM\ARMCC\Bin\..\lib\armlib\c_p.l(_printf_charcount.o)(.text)
    .text                                    0x080018cc   Section        0  C:\Keil_v5\ARM\ARMCC\Bin\..\lib\armlib\c_p.l(_printf_char_common.o)(.text)
    _printf_input_char                       0x080018cd   Thumb Code    10  C:\Keil_v5\ARM\ARMCC\Bin\..\lib\armlib\c_p.l(_printf_char_common.o)(.text)
    .text                                    0x080018fc   Section        0  C:\Keil_v5\ARM\ARMCC\Bin\..\lib\armlib\c_p.l(_sputc.o)(.text)
    .text                                    0x08001908   Section        0  C:\Keil_v5\ARM\ARMCC\Bin\..\lib\armlib\c_p.l(_printf_char_file.o)(.text)
    .text                                    0x08001930   Section        0  C:\Keil_v5\ARM\ARMCC\Bin\..\lib\armlib\c_p.l(_printf_wctomb.o)(.text)
    .text                                    0x080019ec   Section        0  C:\Keil_v5\ARM\ARMCC\Bin\..\lib\armlib\c_p.l(_printf_longlong_dec.o)(.text)
    .text                                    0x08001a5c   Section        0  C:\Keil_v5\ARM\ARMCC\Bin\..\lib\armlib\c_p.l(_printf_oct_int_ll.o)(.text)
    _printf_longlong_oct_internal            0x08001a5d   Thumb Code     0  C:\Keil_v5\ARM\ARMCC\Bin\..\lib\armlib\c_p.l(_printf_oct_int_ll.o)(.text)
    .text                                    0x08001acc   Section        0  C:\Keil_v5\ARM\ARMCC\Bin\..\lib\armlib\c_p.l(_chval.o)(.text)
    .text                                    0x08001aec   Section        0  C:\Keil_v5\ARM\ARMCC\Bin\..\lib\armlib\c_p.l(scanf_char.o)(.text)
    _scanf_char_input                        0x08001aed   Thumb Code    12  C:\Keil_v5\ARM\ARMCC\Bin\..\lib\armlib\c_p.l(scanf_char.o)(.text)
    .text                                    0x08001b1c   Section        0  C:\Keil_v5\ARM\ARMCC\Bin\..\lib\armlib\c_p.l(_sgetc.o)(.text)
    .text                                    0x08001b60   Section        0  C:\Keil_v5\ARM\ARMCC\Bin\..\lib\armlib\c_p.l(ferror.o)(.text)
    .text                                    0x08001b68   Section        0  C:\Keil_v5\ARM\ARMCC\Bin\..\lib\armlib\c_p.l(filbuf.o)(.text)
    .text                                    0x08001dbc   Section        0  C:\Keil_v5\ARM\ARMCC\Bin\..\lib\armlib\c_p.l(flsbuf.o)(.text)
    .text                                    0x08001fac   Section        0  C:\Keil_v5\ARM\ARMCC\Bin\..\lib\armlib\c_p.l(fseek.o)(.text)
    .text                                    0x080020a0   Section        0  C:\Keil_v5\ARM\ARMCC\Bin\..\lib\armlib\c_p.l(setvbuf.o)(.text)
    .text                                    0x080020ec   Section        0  C:\Keil_v5\ARM\ARMCC\Bin\..\lib\armlib\c_p.l(stdio.o)(.text)
    .text                                    0x080021dc   Section        0  C:\Keil_v5\ARM\ARMCC\Bin\..\lib\armlib\c_p.l(initio.o)(.text)
    .text                                    0x08002318   Section        0  C:\Keil_v5\ARM\ARMCC\Bin\..\lib\armlib\c_p.l(defsig_pvfn_outer.o)(.text)
    .text                                    0x08002324   Section        0  C:\Keil_v5\ARM\ARMCC\Bin\..\lib\armlib\c_p.l(h1_extend.o)(.text)
    .text                                    0x08002358   Section        0  C:\Keil_v5\ARM\ARMCC\Bin\..\lib\armlib\c_p.l(lludiv10.o)(.text)
    .text                                    0x080023d2   Section        0  C:\Keil_v5\ARM\ARMCC\Bin\..\lib\armlib\c_p.l(isspace.o)(.text)
    .text                                    0x080023e4   Section        0  C:\Keil_v5\ARM\ARMCC\Bin\..\lib\armlib\c_p.l(_printf_fp_dec.o)(.text)
    _fp_digits                               0x080023e7   Thumb Code   412  C:\Keil_v5\ARM\ARMCC\Bin\..\lib\armlib\c_p.l(_printf_fp_dec.o)(.text)
    .text                                    0x080027fc   Section        0  C:\Keil_v5\ARM\ARMCC\Bin\..\lib\armlib\c_p.l(_printf_fp_hex.o)(.text)
    .text                                    0x08002ad4   Section        0  C:\Keil_v5\ARM\ARMCC\Bin\..\lib\armlib\c_p.l(_printf_char.o)(.text)
    .text                                    0x08002b02   Section        0  C:\Keil_v5\ARM\ARMCC\Bin\..\lib\armlib\c_p.l(_printf_wchar.o)(.text)
    .text                                    0x08002b30   Section        0  C:\Keil_v5\ARM\ARMCC\Bin\..\lib\armlib\c_p.l(_scanf.o)(.text)
    .text                                    0x08002eb0   Section        0  C:\Keil_v5\ARM\ARMCC\Bin\..\lib\armlib\c_p.l(ftell.o)(.text)
    .text                                    0x08002ef4   Section        0  C:\Keil_v5\ARM\ARMCC\Bin\..\lib\armlib\c_p.l(flushlinebuffered.o)(.text)
    .text                                    0x08002f2c   Section        0  C:\Keil_v5\ARM\ARMCC\Bin\..\lib\armlib\c_p.l(_wcrtomb.o)(.text)
    .text                                    0x08002f6c   Section        0  C:\Keil_v5\ARM\ARMCC\Bin\..\lib\armlib\c_p.l(defsig_exit.o)(.text)
    .text                                    0x08002f78   Section        0  C:\Keil_v5\ARM\ARMCC\Bin\..\lib\armlib\c_p.l(defsig_rtred_outer.o)(.text)
    .text                                    0x08002f84   Section        0  C:\Keil_v5\ARM\ARMCC\Bin\..\lib\armlib\c_p.l(defsig_rtmem_outer.o)(.text)
    .text                                    0x08002f90   Section        0  C:\Keil_v5\ARM\ARMCC\Bin\..\lib\armlib\c_p.l(defsig_pvfn_inner.o)(.text)
    .text                                    0x08002fc0   Section        0  C:\Keil_v5\ARM\ARMCC\Bin\..\lib\armlib\c_p.l(rtudiv10.o)(.text)
    .text                                    0x08002fe8   Section        0  C:\Keil_v5\ARM\ARMCC\Bin\..\lib\armlib\c_p.l(heapauxa.o)(.text)
    .text                                    0x08003038   Section        0  C:\Keil_v5\ARM\ARMCC\Bin\..\lib\armlib\c_p.l(sys_exit.o)(.text)
    .text                                    0x08003044   Section       16  C:\Keil_v5\ARM\ARMCC\Bin\..\lib\armlib\c_p.l(rt_ctype_table.o)(.text)
    .text                                    0x08003054   Section        8  C:\Keil_v5\ARM\ARMCC\Bin\..\lib\armlib\c_p.l(rt_locale.o)(.text)
    .text                                    0x0800305c   Section        8  C:\Keil_v5\ARM\ARMCC\Bin\..\lib\armlib\c_p.l(rt_errno_addr.o)(.text)
    .text                                    0x08003064   Section        0  C:\Keil_v5\ARM\ARMCC\Bin\..\lib\armlib\c_p.l(_printf_fp_infnan.o)(.text)
    .text                                    0x080030ec   Section        0  C:\Keil_v5\ARM\ARMCC\Bin\..\lib\armlib\c_p.l(bigflt0.o)(.text)
    .text                                    0x080031c4   Section        0  C:\Keil_v5\ARM\ARMCC\Bin\..\lib\armlib\c_p.l(btod.o)(.text)
    btod_internal_mul                        0x08003205   Thumb Code   492  C:\Keil_v5\ARM\ARMCC\Bin\..\lib\armlib\c_p.l(btod.o)(.text)
    btod_internal_div                        0x080033f1   Thumb Code   520  C:\Keil_v5\ARM\ARMCC\Bin\..\lib\armlib\c_p.l(btod.o)(.text)
    .text                                    0x08003744   Section        0  C:\Keil_v5\ARM\ARMCC\Bin\..\lib\armlib\c_p.l(defsig_general.o)(.text)
    .text                                    0x08003778   Section        0  C:\Keil_v5\ARM\ARMCC\Bin\..\lib\armlib\c_p.l(defsig_rtred_inner.o)(.text)
    .text                                    0x080037ac   Section        0  C:\Keil_v5\ARM\ARMCC\Bin\..\lib\armlib\c_p.l(defsig_rtmem_inner.o)(.text)
    .text                                    0x080037fc   Section        0  C:\Keil_v5\ARM\ARMCC\Bin\..\lib\armlib\c_p.l(sys_wrch.o)(.text)
    .text                                    0x08003808   Section        2  C:\Keil_v5\ARM\ARMCC\Bin\..\lib\armlib\c_p.l(use_no_semi.o)(.text)
    .text                                    0x0800380a   Section        0  C:\Keil_v5\ARM\ARMCC\Bin\..\lib\armlib\c_p.l(indicate_semi.o)(.text)
    i.$Sub$$main                             0x0800380a   Section        0  mbed/TARGET_NUCLEO_F070RB/TOOLCHAIN_ARM_STD/retarget.o(i.$Sub$$main)
    i.<Func3>                                0x08003816   Section        0  mbed/TARGET_NUCLEO_F070RB/TOOLCHAIN_ARM_STD/mbed.ar(SerialBase.o)(i.<Func3>)
    <Func3>                                  0x08003817   Thumb Code     6  mbed/TARGET_NUCLEO_F070RB/TOOLCHAIN_ARM_STD/mbed.ar(SerialBase.o)(i.<Func3>)
    i.HAL_GPIO_Init                          0x0800381c   Section        0  mbed/TARGET_NUCLEO_F070RB/TOOLCHAIN_ARM_STD/stm32f0xx_hal_gpio.o(i.HAL_GPIO_Init)
    i.HAL_GetTick                            0x08003974   Section        0  mbed/TARGET_NUCLEO_F070RB/TOOLCHAIN_ARM_STD/stm32f0xx_hal.o(i.HAL_GetTick)
    i.HAL_IncTick                            0x08003980   Section        0  mbed/TARGET_NUCLEO_F070RB/TOOLCHAIN_ARM_STD/stm32f0xx_hal.o(i.HAL_IncTick)
    i.HAL_Init                               0x08003990   Section        0  mbed/TARGET_NUCLEO_F070RB/TOOLCHAIN_ARM_STD/stm32f0xx_hal.o(i.HAL_Init)
    i.HAL_InitTick                           0x080039b0   Section        0  mbed/TARGET_NUCLEO_F070RB/TOOLCHAIN_ARM_STD/hal_tick.o(i.HAL_InitTick)
    i.HAL_MspInit                            0x08003a98   Section        0  mbed/TARGET_NUCLEO_F070RB/TOOLCHAIN_ARM_STD/stm32f0xx_hal.o(i.HAL_MspInit)
    i.HAL_RCC_ClockConfig                    0x08003a9c   Section        0  mbed/TARGET_NUCLEO_F070RB/TOOLCHAIN_ARM_STD/stm32f0xx_hal_rcc.o(i.HAL_RCC_ClockConfig)
    i.HAL_RCC_GetPCLK1Freq                   0x08003c40   Section        0  mbed/TARGET_NUCLEO_F070RB/TOOLCHAIN_ARM_STD/stm32f0xx_hal_rcc.o(i.HAL_RCC_GetPCLK1Freq)
    i.HAL_RCC_GetSysClockFreq                0x08003c60   Section        0  mbed/TARGET_NUCLEO_F070RB/TOOLCHAIN_ARM_STD/stm32f0xx_hal_rcc.o(i.HAL_RCC_GetSysClockFreq)
    i.HAL_RCC_OscConfig                      0x08003cd0   Section        0  mbed/TARGET_NUCLEO_F070RB/TOOLCHAIN_ARM_STD/stm32f0xx_hal_rcc.o(i.HAL_RCC_OscConfig)
    i.HAL_TIM_Base_Init                      0x08004074   Section        0  mbed/TARGET_NUCLEO_F070RB/TOOLCHAIN_ARM_STD/stm32f0xx_hal_tim.o(i.HAL_TIM_Base_Init)
    i.HAL_TIM_Base_MspInit                   0x080040a6   Section        0  mbed/TARGET_NUCLEO_F070RB/TOOLCHAIN_ARM_STD/stm32f0xx_hal_tim.o(i.HAL_TIM_Base_MspInit)
    i.HAL_TIM_Base_Start                     0x080040a8   Section        0  mbed/TARGET_NUCLEO_F070RB/TOOLCHAIN_ARM_STD/stm32f0xx_hal_tim.o(i.HAL_TIM_Base_Start)
    i.HAL_TIM_OC_Start                       0x080040c0   Section        0  mbed/TARGET_NUCLEO_F070RB/TOOLCHAIN_ARM_STD/stm32f0xx_hal_tim.o(i.HAL_TIM_OC_Start)
    i.HAL_UART_ErrorCallback                 0x08004118   Section        0  mbed/TARGET_NUCLEO_F070RB/TOOLCHAIN_ARM_STD/serial_api.o(i.HAL_UART_ErrorCallback)
    i.HAL_UART_IRQHandler                    0x08004152   Section        0  mbed/TARGET_NUCLEO_F070RB/TOOLCHAIN_ARM_STD/stm32f0xx_hal_uart.o(i.HAL_UART_IRQHandler)
    i.HAL_UART_Init                          0x080042d8   Section        0  mbed/TARGET_NUCLEO_F070RB/TOOLCHAIN_ARM_STD/stm32f0xx_hal_uart.o(i.HAL_UART_Init)
    i.HAL_UART_MspInit                       0x0800434a   Section        0  mbed/TARGET_NUCLEO_F070RB/TOOLCHAIN_ARM_STD/stm32f0xx_hal_uart.o(i.HAL_UART_MspInit)
    i.HAL_UART_RxCpltCallback                0x0800434c   Section        0  mbed/TARGET_NUCLEO_F070RB/TOOLCHAIN_ARM_STD/stm32f0xx_hal_uart.o(i.HAL_UART_RxCpltCallback)
    i.HAL_UART_TxCpltCallback                0x0800434e   Section        0  mbed/TARGET_NUCLEO_F070RB/TOOLCHAIN_ARM_STD/serial_api.o(i.HAL_UART_TxCpltCallback)
    i.NVIC_SetVector                         0x08004360   Section        0  mbed/TARGET_NUCLEO_F070RB/TOOLCHAIN_ARM_STD/cmsis_nvic.o(i.NVIC_SetVector)
    i.SetSysClock_PLL_HSE                    0x080043a4   Section        0  mbed/TARGET_NUCLEO_F070RB/TOOLCHAIN_ARM_STD/system_stm32f0xx.o(i.SetSysClock_PLL_HSE)
    i.Set_GPIO_Clock                         0x08004418   Section        0  mbed/TARGET_NUCLEO_F070RB/TOOLCHAIN_ARM_STD/pinmap.o(i.Set_GPIO_Clock)
    i.SystemCoreClockUpdate                  0x080044d8   Section        0  mbed/TARGET_NUCLEO_F070RB/TOOLCHAIN_ARM_STD/system_stm32f0xx.o(i.SystemCoreClockUpdate)
    i.SystemInit                             0x08004530   Section        0  mbed/TARGET_NUCLEO_F070RB/TOOLCHAIN_ARM_STD/system_stm32f0xx.o(i.SystemInit)
    i.TIM_Base_SetConfig                     0x08004610   Section        0  mbed/TARGET_NUCLEO_F070RB/TOOLCHAIN_ARM_STD/stm32f0xx_hal_tim.o(i.TIM_Base_SetConfig)
    i.UART_AdvFeatureConfig                  0x08004694   Section        0  mbed/TARGET_NUCLEO_F070RB/TOOLCHAIN_ARM_STD/stm32f0xx_hal_uart.o(i.UART_AdvFeatureConfig)
    i.UART_SetConfig                         0x08004760   Section        0  mbed/TARGET_NUCLEO_F070RB/TOOLCHAIN_ARM_STD/stm32f0xx_hal_uart.o(i.UART_SetConfig)
    i._Z12callbackReadv                      0x080048e0   Section        0  .\build\main.o(i._Z12callbackReadv)
    i._Z5setupv                              0x080048f4   Section        0  .\build\main.o(i._Z5setupv)
    i._Z8checkEPCv                           0x080049d4   Section        0  .\build\main.o(i._Z8checkEPCv)
    i._Z9setupNanol                          0x08004a04   Section        0  .\build\main.o(i._Z9setupNanol)
    i._ZN14BufferedSerial4getcEv             0x08004af0   Section        0  .\build\bufferedserial.o(i._ZN14BufferedSerial4getcEv)
    i._ZN14BufferedSerial4putcEi             0x08004b00   Section        0  .\build\bufferedserial.o(i._ZN14BufferedSerial4putcEi)
    i._ZN14BufferedSerial5primeEv            0x08004b1c   Section        0  .\build\bufferedserial.o(i._ZN14BufferedSerial5primeEv)
    i._ZN14BufferedSerial5rxIrqEv            0x08004b70   Section        0  .\build\bufferedserial.o(i._ZN14BufferedSerial5rxIrqEv)
    i._ZN14BufferedSerial5txIrqEv            0x08004b96   Section        0  .\build\bufferedserial.o(i._ZN14BufferedSerial5txIrqEv)
    i._ZN14BufferedSerial8readableEv         0x08004bec   Section        0  .\build\bufferedserial.o(i._ZN14BufferedSerial8readableEv)
    i._ZN14BufferedSerialC1E7PinNameS0_jjPKc 0x08004bfc   Section        0  .\build\bufferedserial.o(i._ZN14BufferedSerialC1E7PinNameS0_jjPKc)
    i._ZN14BufferedSerialD1Ev                0x08004c70   Section        0  .\build\bufferedserial.o(i._ZN14BufferedSerialD1Ev)
    i._ZN4RFID10getVersionEv                 0x08004d10   Section        0  .\build\rfid.o(i._ZN4RFID10getVersionEv)
    i._ZN4RFID11sendCommandEtb               0x08004d2c   Section        0  .\build\rfid.o(i._ZN4RFID11sendCommandEtb)
    i._ZN4RFID11sendMessageEhPhhtb           0x08004fe0   Section        0  .\build\rfid.o(i._ZN4RFID11sendMessageEhPhhtb)
    i._ZN4RFID11stopReadingEv                0x0800500c   Section        0  .\build\rfid.o(i._ZN4RFID11stopReadingEv)
    i._ZN4RFID12calculateCRCEPhh             0x08005030   Section        0  .\build\rfid.o(i._ZN4RFID12calculateCRCEPhh)
    i._ZN4RFID12setReadPowerEs               0x08005078   Section        0  .\build\rfid.o(i._ZN4RFID12setReadPowerEs)
    i._ZN4RFID12startReadingEv               0x080050d0   Section        0  .\build\rfid.o(i._ZN4RFID12startReadingEv)
    i._ZN4RFID13parseResponseEv              0x08005110   Section        0  .\build\rfid.o(i._ZN4RFID13parseResponseEv)
    i._ZN4RFID14setAntennaPortEv             0x080051fc   Section        0  .\build\rfid.o(i._ZN4RFID14setAntennaPortEv)
    i._ZN4RFID14setTagProtocolEh             0x08005224   Section        0  .\build\rfid.o(i._ZN4RFID14setTagProtocolEh)
    i._ZN4RFID17disableReadFilterEv          0x0800524a   Section        0  .\build\rfid.o(i._ZN4RFID17disableReadFilterEv)
    i._ZN4RFID17printMessageArrayEv          0x0800525c   Section        0  .\build\rfid.o(i._ZN4RFID17printMessageArrayEv)
    i._ZN4RFID22setReaderConfigurationEhh    0x080052f4   Section        0  .\build\rfid.o(i._ZN4RFID22setReaderConfigurationEhh)
    i._ZN4RFID5beginER14BufferedSerial       0x0800531e   Section        0  .\build\rfid.o(i._ZN4RFID5beginER14BufferedSerial)
    i._ZN4RFID5checkEv                       0x08005328   Section        0  .\build\rfid.o(i._ZN4RFID5checkEv)
    i._ZN4RFID7setBaudEl                     0x080053e8   Section        0  .\build\rfid.o(i._ZN4RFID7setBaudEl)
    i._ZN4RFID9setRegionEh                   0x08005430   Section        0  .\build\rfid.o(i._ZN4RFID9setRegionEh)
    i._ZN4RFIDC1Ev                           0x0800544e   Section        0  .\build\rfid.o(i._ZN4RFIDC1Ev)
    i._ZN4mbed10FileHandle4flenEv            0x0800545c   Section        0  mbed/TARGET_NUCLEO_F070RB/TOOLCHAIN_ARM_STD/retarget.o(i._ZN4mbed10FileHandle4flenEv)
    i._ZN4mbed10FileHandle4lockEv            0x080054ac   Section        0  mbed/TARGET_NUCLEO_F070RB/TOOLCHAIN_ARM_STD/retarget.o(i._ZN4mbed10FileHandle4lockEv)
    i._ZN4mbed10FileHandle6unlockEv          0x080054ae   Section        0  mbed/TARGET_NUCLEO_F070RB/TOOLCHAIN_ARM_STD/retarget.o(i._ZN4mbed10FileHandle6unlockEv)
    i._ZN4mbed10FileHandleD2Ev               0x080054b0   Section        0  mbed/TARGET_NUCLEO_F070RB/TOOLCHAIN_ARM_STD/retarget.o(i._ZN4mbed10FileHandleD2Ev)
    i._ZN4mbed10SerialBase10_base_getcEv     0x08005528   Section        0  mbed/TARGET_NUCLEO_F070RB/TOOLCHAIN_ARM_STD/mbed.ar(SerialBase.o)(i._ZN4mbed10SerialBase10_base_getcEv)
    i._ZN4mbed10SerialBase10_base_putcEi     0x08005532   Section        0  mbed/TARGET_NUCLEO_F070RB/TOOLCHAIN_ARM_STD/mbed.ar(SerialBase.o)(i._ZN4mbed10SerialBase10_base_putcEi)
    i._ZN4mbed10SerialBase12_irq_handlerEj9SerialIrq 0x08005540   Section        0  mbed/TARGET_NUCLEO_F070RB/TOOLCHAIN_ARM_STD/mbed.ar(SerialBase.o)(i._ZN4mbed10SerialBase12_irq_handlerEj9SerialIrq)
    i._ZN4mbed10SerialBase24interrupt_handler_asynchEv 0x08005570   Section        0  mbed/TARGET_NUCLEO_F070RB/TOOLCHAIN_ARM_STD/mbed.ar(SerialBase.o)(i._ZN4mbed10SerialBase24interrupt_handler_asynchEv)
    i._ZN4mbed10SerialBase4baudEi            0x080055b2   Section        0  mbed/TARGET_NUCLEO_F070RB/TOOLCHAIN_ARM_STD/mbed.ar(SerialBase.o)(i._ZN4mbed10SerialBase4baudEi)
    i._ZN4mbed10SerialBase4lockEv            0x080055d8   Section        0  mbed/TARGET_NUCLEO_F070RB/TOOLCHAIN_ARM_STD/mbed.ar(SerialBase.o)(i._ZN4mbed10SerialBase4lockEv)
    i._ZN4mbed10SerialBase6attachENS_8CallbackIFvvEEENS0_7IrqTypeE 0x080055dc   Section        0  mbed/TARGET_NUCLEO_F070RB/TOOLCHAIN_ARM_STD/mbed.ar(SerialBase.o)(i._ZN4mbed10SerialBase6attachENS_8CallbackIFvvEEENS0_7IrqTypeE)
    i._ZN4mbed10SerialBase6unlockEv          0x08005660   Section        0  mbed/TARGET_NUCLEO_F070RB/TOOLCHAIN_ARM_STD/mbed.ar(SerialBase.o)(i._ZN4mbed10SerialBase6unlockEv)
    i._ZN4mbed10SerialBase8readableEv        0x08005662   Section        0  mbed/TARGET_NUCLEO_F070RB/TOOLCHAIN_ARM_STD/mbed.ar(SerialBase.o)(i._ZN4mbed10SerialBase8readableEv)
    i._ZN4mbed10SerialBaseC1E7PinNameS1_i    0x08005684   Section        0  mbed/TARGET_NUCLEO_F070RB/TOOLCHAIN_ARM_STD/mbed.ar(SerialBase.o)(i._ZN4mbed10SerialBaseC1E7PinNameS1_i)
    i._ZN4mbed10TimerEvent3irqEj             0x08005758   Section        0  mbed/TARGET_NUCLEO_F070RB/TOOLCHAIN_ARM_STD/mbed.ar(TimerEvent.o)(i._ZN4mbed10TimerEvent3irqEj)
    i._ZN4mbed10TimerEvent6insertEj          0x0800575e   Section        0  mbed/TARGET_NUCLEO_F070RB/TOOLCHAIN_ARM_STD/mbed.ar(TimerEvent.o)(i._ZN4mbed10TimerEvent6insertEj)
    i._ZN4mbed10TimerEvent6removeEv          0x08005770   Section        0  mbed/TARGET_NUCLEO_F070RB/TOOLCHAIN_ARM_STD/mbed.ar(TimerEvent.o)(i._ZN4mbed10TimerEvent6removeEv)
    i._ZN4mbed10TimerEventC2Ev               0x08005780   Section        0  mbed/TARGET_NUCLEO_F070RB/TOOLCHAIN_ARM_STD/mbed.ar(TimerEvent.o)(i._ZN4mbed10TimerEventC2Ev)
    i._ZN4mbed10TimerEventD2Ev               0x080057a8   Section        0  mbed/TARGET_NUCLEO_F070RB/TOOLCHAIN_ARM_STD/mbed.ar(TimerEvent.o)(i._ZN4mbed10TimerEventD2Ev)
    i._ZN4mbed26mbed_set_unbuffered_streamEPSt6__FILE 0x080057c0   Section        0  mbed/TARGET_NUCLEO_F070RB/TOOLCHAIN_ARM_STD/retarget.o(i._ZN4mbed26mbed_set_unbuffered_streamEPSt6__FILE)
    i._ZN4mbed5Timer5startEv                 0x080057ca   Section        0  mbed/TARGET_NUCLEO_F070RB/TOOLCHAIN_ARM_STD/mbed.ar(Timer.o)(i._ZN4mbed5Timer5startEv)
    i._ZN4mbed5Timer7read_msEv               0x080057ea   Section        0  mbed/TARGET_NUCLEO_F070RB/TOOLCHAIN_ARM_STD/mbed.ar(Timer.o)(i._ZN4mbed5Timer7read_msEv)
    i._ZN4mbed5TimerC1Ev                     0x08005820   Section        0  mbed/TARGET_NUCLEO_F070RB/TOOLCHAIN_ARM_STD/mbed.ar(Timer.o)(i._ZN4mbed5TimerC1Ev)
    i._ZN4mbed6Serial4lockEv                 0x08005848   Section        0  mbed/TARGET_NUCLEO_F070RB/TOOLCHAIN_ARM_STD/mbed.ar(Serial.o)(i._ZN4mbed6Serial4lockEv)
    i._ZN4mbed6Serial6unlockEv               0x0800584a   Section        0  mbed/TARGET_NUCLEO_F070RB/TOOLCHAIN_ARM_STD/mbed.ar(Serial.o)(i._ZN4mbed6Serial6unlockEv)
    i._ZN4mbed6SerialC1E7PinNameS1_PKci      0x0800584c   Section        0  mbed/TARGET_NUCLEO_F070RB/TOOLCHAIN_ARM_STD/mbed.ar(Serial.o)(i._ZN4mbed6SerialC1E7PinNameS1_PKci)
    i._ZN4mbed6SerialD1Ev                    0x08005880   Section        0  mbed/TARGET_NUCLEO_F070RB/TOOLCHAIN_ARM_STD/mbed.ar(Serial.o)(i._ZN4mbed6SerialD1Ev)
    i._ZN4mbed6Stream4flenEv                 0x080058e4   Section        0  mbed/TARGET_NUCLEO_F070RB/TOOLCHAIN_ARM_STD/mbed.ar(Stream.o)(i._ZN4mbed6Stream4flenEv)
    i._ZN4mbed6Stream4getcEv                 0x080058e8   Section        0  mbed/TARGET_NUCLEO_F070RB/TOOLCHAIN_ARM_STD/mbed.ar(Stream.o)(i._ZN4mbed6Stream4getcEv)
    i._ZN4mbed6Stream4readEPvj               0x0800590e   Section        0  mbed/TARGET_NUCLEO_F070RB/TOOLCHAIN_ARM_STD/mbed.ar(Stream.o)(i._ZN4mbed6Stream4readEPvj)
    i._ZN4mbed6Stream5closeEv                0x08005944   Section        0  mbed/TARGET_NUCLEO_F070RB/TOOLCHAIN_ARM_STD/mbed.ar(Stream.o)(i._ZN4mbed6Stream5closeEv)
    i._ZN4mbed6Stream5lseekEli               0x08005948   Section        0  mbed/TARGET_NUCLEO_F070RB/TOOLCHAIN_ARM_STD/mbed.ar(Stream.o)(i._ZN4mbed6Stream5lseekEli)
    i._ZN4mbed6Stream5writeEPKvj             0x0800594c   Section        0  mbed/TARGET_NUCLEO_F070RB/TOOLCHAIN_ARM_STD/mbed.ar(Stream.o)(i._ZN4mbed6Stream5writeEPKvj)
    i._ZN4mbed6Stream6isattyEv               0x08005982   Section        0  mbed/TARGET_NUCLEO_F070RB/TOOLCHAIN_ARM_STD/mbed.ar(Stream.o)(i._ZN4mbed6Stream6isattyEv)
    i._ZN4mbed6Stream6printfEPKcz            0x08005986   Section        0  mbed/TARGET_NUCLEO_F070RB/TOOLCHAIN_ARM_STD/mbed.ar(Stream.o)(i._ZN4mbed6Stream6printfEPKcz)
    i._ZN4mbed6StreamC2EPKc                  0x080059bc   Section        0  mbed/TARGET_NUCLEO_F070RB/TOOLCHAIN_ARM_STD/mbed.ar(Stream.o)(i._ZN4mbed6StreamC2EPKc)
    i._ZN4mbed6StreamD2Ev                    0x08005a00   Section        0  mbed/TARGET_NUCLEO_F070RB/TOOLCHAIN_ARM_STD/mbed.ar(Stream.o)(i._ZN4mbed6StreamD2Ev)
    i._ZN4mbed6Ticker5setupEj                0x08005a24   Section        0  mbed/TARGET_NUCLEO_F070RB/TOOLCHAIN_ARM_STD/mbed.ar(Ticker.o)(i._ZN4mbed6Ticker5setupEj)
    i._ZN4mbed6Ticker7handlerEv              0x08005a4c   Section        0  mbed/TARGET_NUCLEO_F070RB/TOOLCHAIN_ARM_STD/mbed.ar(Ticker.o)(i._ZN4mbed6Ticker7handlerEv)
    i._ZN4mbed6TickerD1Ev                    0x08005a84   Section        0  mbed/TARGET_NUCLEO_F070RB/TOOLCHAIN_ARM_STD/mbed.ar(Ticker.o)(i._ZN4mbed6TickerD1Ev)
    i._ZN4mbed8FileBase11getPathTypeEv       0x08005acc   Section        0  mbed/TARGET_NUCLEO_F070RB/TOOLCHAIN_ARM_STD/mbed.ar(FileBase.o)(i._ZN4mbed8FileBase11getPathTypeEv)
    i._ZN4mbed8FileBase6lookupEPKcj          0x08005ad0   Section        0  mbed/TARGET_NUCLEO_F070RB/TOOLCHAIN_ARM_STD/mbed.ar(FileBase.o)(i._ZN4mbed8FileBase6lookupEPKcj)
    i._ZN4mbed8FileBaseC1EPKcNS_8PathTypeE   0x08005b40   Section        0  mbed/TARGET_NUCLEO_F070RB/TOOLCHAIN_ARM_STD/mbed.ar(FileBase.o)(i._ZN4mbed8FileBaseC1EPKcNS_8PathTypeE)
    i._ZN4mbed8FileBaseD1Ev                  0x08005b80   Section        0  mbed/TARGET_NUCLEO_F070RB/TOOLCHAIN_ARM_STD/mbed.ar(FileBase.o)(i._ZN4mbed8FileBaseD1Ev)
    i._ZN4mbed8FileLikeC2EPKc                0x08005bcc   Section        0  mbed/TARGET_NUCLEO_F070RB/TOOLCHAIN_ARM_STD/mbed.ar(FileLike.o)(i._ZN4mbed8FileLikeC2EPKc)
    i._ZN4mbed8FileLikeD2Ev                  0x08005bf0   Section        0  mbed/TARGET_NUCLEO_F070RB/TOOLCHAIN_ARM_STD/mbed.ar(FileLike.o)(i._ZN4mbed8FileLikeD2Ev)
    i._ZN4mbed8FilePath10fileSystemEv        0x08005c00   Section        0  mbed/TARGET_NUCLEO_F070RB/TOOLCHAIN_ARM_STD/mbed.ar(FilePath.o)(i._ZN4mbed8FilePath10fileSystemEv)
    i._ZN4mbed8FilePath4fileEv               0x08005c1a   Section        0  mbed/TARGET_NUCLEO_F070RB/TOOLCHAIN_ARM_STD/mbed.ar(FilePath.o)(i._ZN4mbed8FilePath4fileEv)
    i._ZN4mbed8FilePath6existsEv             0x08005c3a   Section        0  mbed/TARGET_NUCLEO_F070RB/TOOLCHAIN_ARM_STD/mbed.ar(FilePath.o)(i._ZN4mbed8FilePath6existsEv)
    i._ZN4mbed8FilePath6isFileEv             0x08005c44   Section        0  mbed/TARGET_NUCLEO_F070RB/TOOLCHAIN_ARM_STD/mbed.ar(FilePath.o)(i._ZN4mbed8FilePath6isFileEv)
    i._ZN4mbed8FilePath8fileNameEv           0x08005c5c   Section        0  mbed/TARGET_NUCLEO_F070RB/TOOLCHAIN_ARM_STD/mbed.ar(FilePath.o)(i._ZN4mbed8FilePath8fileNameEv)
    i._ZN4mbed8FilePathC1EPKc                0x08005c60   Section        0  mbed/TARGET_NUCLEO_F070RB/TOOLCHAIN_ARM_STD/mbed.ar(FilePath.o)(i._ZN4mbed8FilePathC1EPKc)
    i._ZN4mbed9DigitalIncviEv                0x08005ca4   Section        0  .\build\main.o(i._ZN4mbed9DigitalIncviEv)
    i._ZN4mbed9RawSerial4lockEv              0x08005cf8   Section        0  mbed/TARGET_NUCLEO_F070RB/TOOLCHAIN_ARM_STD/mbed.ar(RawSerial.o)(i._ZN4mbed9RawSerial4lockEv)
    i._ZN4mbed9RawSerial6unlockEv            0x08005cfa   Section        0  mbed/TARGET_NUCLEO_F070RB/TOOLCHAIN_ARM_STD/mbed.ar(RawSerial.o)(i._ZN4mbed9RawSerial6unlockEv)
    i._ZN4mbed9RawSerialC1E7PinNameS1_i      0x08005cfc   Section        0  mbed/TARGET_NUCLEO_F070RB/TOOLCHAIN_ARM_STD/mbed.ar(RawSerial.o)(i._ZN4mbed9RawSerialC1E7PinNameS1_i)
    i._ZN4mbed9donothingEv                   0x08005d0c   Section        0  mbed/TARGET_NUCLEO_F070RB/TOOLCHAIN_ARM_STD/mbed.ar(SerialBase.o)(i._ZN4mbed9donothingEv)
    mbed::donothing()                        0x08005d0d   Thumb Code     2  mbed/TARGET_NUCLEO_F070RB/TOOLCHAIN_ARM_STD/mbed.ar(SerialBase.o)(i._ZN4mbed9donothingEv)
    i._ZN4mbed9mbed_getcEPSt6__FILE          0x08005d0e   Section        0  mbed/TARGET_NUCLEO_F070RB/TOOLCHAIN_ARM_STD/retarget.o(i._ZN4mbed9mbed_getcEPSt6__FILE)
    i._ZThn188_N4mbed6Serial4lockEv          0x08005d16   Section        0  mbed/TARGET_NUCLEO_F070RB/TOOLCHAIN_ARM_STD/mbed.ar(Serial.o)(i._ZThn188_N4mbed6Serial4lockEv)
    i._ZThn188_N4mbed6Serial5_getcEv         0x08005d18   Section        0  mbed/TARGET_NUCLEO_F070RB/TOOLCHAIN_ARM_STD/mbed.ar(Serial.o)(i._ZThn188_N4mbed6Serial5_getcEv)
    i._ZThn188_N4mbed6Serial5_putcEi         0x08005d22   Section        0  mbed/TARGET_NUCLEO_F070RB/TOOLCHAIN_ARM_STD/mbed.ar(Serial.o)(i._ZThn188_N4mbed6Serial5_putcEi)
    i._ZThn188_N4mbed6Serial6unlockEv        0x08005d2c   Section        0  mbed/TARGET_NUCLEO_F070RB/TOOLCHAIN_ARM_STD/mbed.ar(Serial.o)(i._ZThn188_N4mbed6Serial6unlockEv)
    i._ZdaPv                                 0x08005d2e   Section        0  mbed/TARGET_NUCLEO_F070RB/TOOLCHAIN_ARM_STD/retarget.o(i._ZdaPv)
    i._Znaj                                  0x08005d3c   Section        0  mbed/TARGET_NUCLEO_F070RB/TOOLCHAIN_ARM_STD/retarget.o(i._Znaj)
    i.__ARM_common_ll_muluu                  0x08005d70   Section        0  C:\Keil_v5\ARM\ARMCC\Bin\..\lib\armlib\c_p.l(btod.o)(i.__ARM_common_ll_muluu)
    i.__ARM_fpclassify                       0x08005da0   Section        0  C:\Keil_v5\ARM\ARMCC\Bin\..\lib\armlib\m_ps.l(fpclassify.o)(i.__ARM_fpclassify)
    i.__aeabi_atexit                         0x08005dcc   Section        0  mbed/TARGET_NUCLEO_F070RB/TOOLCHAIN_ARM_STD/retarget.o(i.__aeabi_atexit)
    i.__aeabi_vec_ctor_nocookie_nodtor       0x08005dd0   Section        0  C:\Keil_v5\ARM\ARMCC\Bin\..\lib\cpplib\cpprt_p.l(aeabi_vec_ctor_nocookie_nodtor.o)(i.__aeabi_vec_ctor_nocookie_nodtor)
    i.__cxa_pure_virtual                     0x08005df2   Section        0  C:\Keil_v5\ARM\ARMCC\Bin\..\lib\cpplib\cpprt_p.l(pure_virt.o)(i.__cxa_pure_virtual)
    i.__sti___8_main_cpp_fdcb111a            0x08005dfc   Section        0  .\build\main.o(i.__sti___8_main_cpp_fdcb111a)
    __sti___8_main_cpp_fdcb111a              0x08005dfd   Thumb Code   132  .\build\main.o(i.__sti___8_main_cpp_fdcb111a)
    i.__user_setup_stackheap                 0x08005ea8   Section        0  mbed/TARGET_NUCLEO_F070RB/TOOLCHAIN_ARM_STD/sys.o(i.__user_setup_stackheap)
    i._is_digit                              0x08005eb8   Section        0  C:\Keil_v5\ARM\ARMCC\Bin\..\lib\armlib\c_p.l(__printf_wp.o)(i._is_digit)
    i._platform_post_stackheap_init          0x08005ec6   Section        0  mbed/TARGET_NUCLEO_F070RB/TOOLCHAIN_ARM_STD/retarget.o(i._platform_post_stackheap_init)
    i._sys_close                             0x08005ed0   Section        0  mbed/TARGET_NUCLEO_F070RB/TOOLCHAIN_ARM_STD/retarget.o(i._sys_close)
    i._sys_flen                              0x08005efc   Section        0  mbed/TARGET_NUCLEO_F070RB/TOOLCHAIN_ARM_STD/retarget.o(i._sys_flen)
    i._sys_istty                             0x08005f24   Section        0  mbed/TARGET_NUCLEO_F070RB/TOOLCHAIN_ARM_STD/retarget.o(i._sys_istty)
    i._sys_open                              0x08005f4c   Section        0  mbed/TARGET_NUCLEO_F070RB/TOOLCHAIN_ARM_STD/retarget.o(i._sys_open)
    i._sys_read                              0x08006118   Section        0  mbed/TARGET_NUCLEO_F070RB/TOOLCHAIN_ARM_STD/retarget.o(i._sys_read)
    i._sys_seek                              0x08006178   Section        0  mbed/TARGET_NUCLEO_F070RB/TOOLCHAIN_ARM_STD/retarget.o(i._sys_seek)
    i._sys_write                             0x080061a0   Section        0  mbed/TARGET_NUCLEO_F070RB/TOOLCHAIN_ARM_STD/retarget.o(i._sys_write)
    i.core_util_critical_section_enter       0x0800620c   Section        0  mbed/TARGET_NUCLEO_F070RB/TOOLCHAIN_ARM_STD/mbed.ar(mbed_critical.o)(i.core_util_critical_section_enter)
    i.core_util_critical_section_exit        0x08006298   Section        0  mbed/TARGET_NUCLEO_F070RB/TOOLCHAIN_ARM_STD/mbed.ar(mbed_critical.o)(i.core_util_critical_section_exit)
    i.error                                  0x080062f0   Section        0  mbed/TARGET_NUCLEO_F070RB/TOOLCHAIN_ARM_STD/mbed.ar(mbed_error.o)(i.error)
    i.exit                                   0x08006304   Section        0  mbed/TARGET_NUCLEO_F070RB/TOOLCHAIN_ARM_STD/retarget.o(i.exit)
    i.fgetc                                  0x08006324   Section        0  C:\Keil_v5\ARM\ARMCC\Bin\..\lib\armlib\c_p.l(fgetc.o)(i.fgetc)
    i.fputc                                  0x08006340   Section        0  C:\Keil_v5\ARM\ARMCC\Bin\..\lib\armlib\c_p.l(fputc.o)(i.fputc)
    i.get_us_ticker_data                     0x08006360   Section        0  mbed/TARGET_NUCLEO_F070RB/TOOLCHAIN_ARM_STD/mbed.ar(mbed_us_ticker_api.o)(i.get_us_ticker_data)
    i.gpio_dir                               0x08006368   Section        0  mbed/TARGET_NUCLEO_F070RB/TOOLCHAIN_ARM_STD/gpio_api.o(i.gpio_dir)
    i.gpio_init                              0x080063b4   Section        0  mbed/TARGET_NUCLEO_F070RB/TOOLCHAIN_ARM_STD/gpio_api.o(i.gpio_init)
    i.gpio_init_in                           0x080063ec   Section        0  mbed/TARGET_NUCLEO_F070RB/TOOLCHAIN_ARM_STD/mbed.ar(mbed_gpio.o)(i.gpio_init_in)
    i.gpio_mode                              0x0800640e   Section        0  mbed/TARGET_NUCLEO_F070RB/TOOLCHAIN_ARM_STD/gpio_api.o(i.gpio_mode)
    i.init_uart                              0x0800641c   Section        0  mbed/TARGET_NUCLEO_F070RB/TOOLCHAIN_ARM_STD/serial_api.o(i.init_uart)
    init_uart                                0x0800641d   Thumb Code    98  mbed/TARGET_NUCLEO_F070RB/TOOLCHAIN_ARM_STD/serial_api.o(i.init_uart)
    i.main                                   0x0800649c   Section        0  .\build\main.o(i.main)
    i.mbed_assert_internal                   0x0800685c   Section        0  mbed/TARGET_NUCLEO_F070RB/TOOLCHAIN_ARM_STD/mbed.ar(mbed_assert.o)(i.mbed_assert_internal)
    i.mbed_die                               0x080068b0   Section        0  mbed/TARGET_NUCLEO_F070RB/TOOLCHAIN_ARM_STD/mbed_board.o(i.mbed_die)
    i.mbed_error_printf                      0x080068c4   Section        0  mbed/TARGET_NUCLEO_F070RB/TOOLCHAIN_ARM_STD/mbed_board.o(i.mbed_error_printf)
    i.mbed_error_vfprintf                    0x0800691c   Section        0  mbed/TARGET_NUCLEO_F070RB/TOOLCHAIN_ARM_STD/mbed_board.o(i.mbed_error_vfprintf)
    i.mbed_main                              0x0800696c   Section        0  mbed/TARGET_NUCLEO_F070RB/TOOLCHAIN_ARM_STD/retarget.o(i.mbed_main)
    i.mbed_sdk_init                          0x0800696e   Section        0  mbed/TARGET_NUCLEO_F070RB/TOOLCHAIN_ARM_STD/mbed_overrides.o(i.mbed_sdk_init)
    i.pin_function                           0x0800697c   Section        0  mbed/TARGET_NUCLEO_F070RB/TOOLCHAIN_ARM_STD/pinmap.o(i.pin_function)
    i.pin_mode                               0x080069e8   Section        0  mbed/TARGET_NUCLEO_F070RB/TOOLCHAIN_ARM_STD/pinmap.o(i.pin_mode)
    i.pinmap_merge                           0x08006a3c   Section        0  mbed/TARGET_NUCLEO_F070RB/TOOLCHAIN_ARM_STD/mbed.ar(mbed_pinmap_common.o)(i.pinmap_merge)
    i.pinmap_peripheral                      0x08006a70   Section        0  mbed/TARGET_NUCLEO_F070RB/TOOLCHAIN_ARM_STD/mbed.ar(mbed_pinmap_common.o)(i.pinmap_peripheral)
    i.pinmap_pinout                          0x08006acc   Section        0  mbed/TARGET_NUCLEO_F070RB/TOOLCHAIN_ARM_STD/mbed.ar(mbed_pinmap_common.o)(i.pinmap_pinout)
    i.serial_baud                            0x08006b20   Section        0  mbed/TARGET_NUCLEO_F070RB/TOOLCHAIN_ARM_STD/serial_api.o(i.serial_baud)
    i.serial_getc                            0x08006b2c   Section        0  mbed/TARGET_NUCLEO_F070RB/TOOLCHAIN_ARM_STD/serial_api.o(i.serial_getc)
    i.serial_init                            0x08006b50   Section        0  mbed/TARGET_NUCLEO_F070RB/TOOLCHAIN_ARM_STD/serial_api.o(i.serial_init)
    i.serial_irq_handler                     0x08006cc4   Section        0  mbed/TARGET_NUCLEO_F070RB/TOOLCHAIN_ARM_STD/serial_api.o(i.serial_irq_handler)
    i.serial_irq_handler_asynch              0x08006cdc   Section        0  mbed/TARGET_NUCLEO_F070RB/TOOLCHAIN_ARM_STD/serial_api.o(i.serial_irq_handler_asynch)
    i.serial_irq_set                         0x08006e30   Section        0  mbed/TARGET_NUCLEO_F070RB/TOOLCHAIN_ARM_STD/serial_api.o(i.serial_irq_set)
    i.serial_putc                            0x08006ef8   Section        0  mbed/TARGET_NUCLEO_F070RB/TOOLCHAIN_ARM_STD/serial_api.o(i.serial_putc)
    i.serial_readable                        0x08006f1c   Section        0  mbed/TARGET_NUCLEO_F070RB/TOOLCHAIN_ARM_STD/serial_api.o(i.serial_readable)
    i.serial_writable                        0x08006f38   Section        0  mbed/TARGET_NUCLEO_F070RB/TOOLCHAIN_ARM_STD/serial_api.o(i.serial_writable)
    i.set_compare                            0x08006f54   Section        0  mbed/TARGET_NUCLEO_F070RB/TOOLCHAIN_ARM_STD/us_ticker.o(i.set_compare)
    i.ticker_insert_event                    0x08006f70   Section        0  mbed/TARGET_NUCLEO_F070RB/TOOLCHAIN_ARM_STD/mbed.ar(mbed_ticker_api.o)(i.ticker_insert_event)
    i.ticker_irq_handler                     0x08006fb4   Section        0  mbed/TARGET_NUCLEO_F070RB/TOOLCHAIN_ARM_STD/mbed.ar(mbed_ticker_api.o)(i.ticker_irq_handler)
    i.ticker_read                            0x08006ffe   Section        0  mbed/TARGET_NUCLEO_F070RB/TOOLCHAIN_ARM_STD/mbed.ar(mbed_ticker_api.o)(i.ticker_read)
    i.ticker_remove_event                    0x08007004   Section        0  mbed/TARGET_NUCLEO_F070RB/TOOLCHAIN_ARM_STD/mbed.ar(mbed_ticker_api.o)(i.ticker_remove_event)
    i.ticker_set_handler                     0x0800704a   Section        0  mbed/TARGET_NUCLEO_F070RB/TOOLCHAIN_ARM_STD/mbed.ar(mbed_ticker_api.o)(i.ticker_set_handler)
    i.timer_oc_irq_handler                   0x0800705c   Section        0  mbed/TARGET_NUCLEO_F070RB/TOOLCHAIN_ARM_STD/hal_tick.o(i.timer_oc_irq_handler)
    i.timer_update_irq_handler               0x08007100   Section        0  mbed/TARGET_NUCLEO_F070RB/TOOLCHAIN_ARM_STD/hal_tick.o(i.timer_update_irq_handler)
    i.uart1_irq                              0x08007130   Section        0  mbed/TARGET_NUCLEO_F070RB/TOOLCHAIN_ARM_STD/serial_api.o(i.uart1_irq)
    uart1_irq                                0x08007131   Thumb Code    10  mbed/TARGET_NUCLEO_F070RB/TOOLCHAIN_ARM_STD/serial_api.o(i.uart1_irq)
    i.uart2_irq                              0x0800713a   Section        0  mbed/TARGET_NUCLEO_F070RB/TOOLCHAIN_ARM_STD/serial_api.o(i.uart2_irq)
    uart2_irq                                0x0800713b   Thumb Code    10  mbed/TARGET_NUCLEO_F070RB/TOOLCHAIN_ARM_STD/serial_api.o(i.uart2_irq)
    i.uart3_irq                              0x08007144   Section        0  mbed/TARGET_NUCLEO_F070RB/TOOLCHAIN_ARM_STD/serial_api.o(i.uart3_irq)
    uart3_irq                                0x08007145   Thumb Code    10  mbed/TARGET_NUCLEO_F070RB/TOOLCHAIN_ARM_STD/serial_api.o(i.uart3_irq)
    i.uart4_irq                              0x0800714e   Section        0  mbed/TARGET_NUCLEO_F070RB/TOOLCHAIN_ARM_STD/serial_api.o(i.uart4_irq)
    uart4_irq                                0x0800714f   Thumb Code    10  mbed/TARGET_NUCLEO_F070RB/TOOLCHAIN_ARM_STD/serial_api.o(i.uart4_irq)
    i.uart_irq                               0x08007158   Section        0  mbed/TARGET_NUCLEO_F070RB/TOOLCHAIN_ARM_STD/serial_api.o(i.uart_irq)
    uart_irq                                 0x08007159   Thumb Code   102  mbed/TARGET_NUCLEO_F070RB/TOOLCHAIN_ARM_STD/serial_api.o(i.uart_irq)
    i.us_ticker_clear_interrupt              0x080071cc   Section        0  mbed/TARGET_NUCLEO_F070RB/TOOLCHAIN_ARM_STD/us_ticker.o(i.us_ticker_clear_interrupt)
    i.us_ticker_disable_interrupt            0x080071ec   Section        0  mbed/TARGET_NUCLEO_F070RB/TOOLCHAIN_ARM_STD/us_ticker.o(i.us_ticker_disable_interrupt)
    i.us_ticker_init                         0x08007204   Section        0  mbed/TARGET_NUCLEO_F070RB/TOOLCHAIN_ARM_STD/us_ticker.o(i.us_ticker_init)
    i.us_ticker_irq_handler                  0x08007220   Section        0  mbed/TARGET_NUCLEO_F070RB/TOOLCHAIN_ARM_STD/mbed.ar(mbed_us_ticker_api.o)(i.us_ticker_irq_handler)
    i.us_ticker_read                         0x08007230   Section        0  mbed/TARGET_NUCLEO_F070RB/TOOLCHAIN_ARM_STD/us_ticker.o(i.us_ticker_read)
    i.us_ticker_set_interrupt                0x08007268   Section        0  mbed/TARGET_NUCLEO_F070RB/TOOLCHAIN_ARM_STD/us_ticker.o(i.us_ticker_set_interrupt)
    i.wait_ms                                0x080072f4   Section        0  mbed/TARGET_NUCLEO_F070RB/TOOLCHAIN_ARM_STD/mbed.ar(mbed_wait_api_no_rtos.o)(i.wait_ms)
    locale$$code                             0x08007310   Section       44  C:\Keil_v5\ARM\ARMCC\Bin\..\lib\armlib\c_p.l(lc_numeric_c.o)(locale$$code)
    locale$$code                             0x0800733c   Section       44  C:\Keil_v5\ARM\ARMCC\Bin\..\lib\armlib\c_p.l(lc_ctype_c.o)(locale$$code)
    t._ZN12SingletonPtrI13PlatformMutexEptEv 0x08007368   Section        0  mbed/TARGET_NUCLEO_F070RB/TOOLCHAIN_ARM_STD/mbed.ar(FileBase.o)(t._ZN12SingletonPtrI13PlatformMutexEptEv)
    t._ZN4mbed8CallbackIFviEED1Ev            0x08007394   Section        0  .\build\main.o(t._ZN4mbed8CallbackIFviEED1Ev)
    t._ZN4mbed8CallbackIFvvEE13function_callINS2_14method_contextI14BufferedSerialMS5_FvvEEEEEvPKv 0x080073aa   Section        0  .\build\bufferedserial.o(t._ZN4mbed8CallbackIFvvEE13function_callINS2_14method_contextI14BufferedSerialMS5_FvvEEEEEvPKv)
    t._ZN4mbed8CallbackIFvvEE13function_callIPS1_EEvPKv 0x080073d8   Section        0  mbed/TARGET_NUCLEO_F070RB/TOOLCHAIN_ARM_STD/mbed.ar(SerialBase.o)(t._ZN4mbed8CallbackIFvvEE13function_callIPS1_EEvPKv)
    t._ZN4mbed8CallbackIFvvEE13function_dtorINS2_14method_contextI14BufferedSerialMS5_FvvEEEEEvPv 0x080073dc   Section        0  .\build\bufferedserial.o(t._ZN4mbed8CallbackIFvvEE13function_dtorINS2_14method_contextI14BufferedSerialMS5_FvvEEEEEvPv)
    t._ZN4mbed8CallbackIFvvEE13function_dtorIPS1_EEvPv 0x080073de   Section        0  mbed/TARGET_NUCLEO_F070RB/TOOLCHAIN_ARM_STD/mbed.ar(SerialBase.o)(t._ZN4mbed8CallbackIFvvEE13function_dtorIPS1_EEvPv)
    t._ZN4mbed8CallbackIFvvEE13function_moveINS2_14method_contextI14BufferedSerialMS5_FvvEEEEEvPvPKv 0x080073e0   Section        0  .\build\bufferedserial.o(t._ZN4mbed8CallbackIFvvEE13function_moveINS2_14method_contextI14BufferedSerialMS5_FvvEEEEEvPvPKv)
    t._ZN4mbed8CallbackIFvvEE13function_moveIPS1_EEvPvPKv 0x080073f4   Section        0  mbed/TARGET_NUCLEO_F070RB/TOOLCHAIN_ARM_STD/mbed.ar(SerialBase.o)(t._ZN4mbed8CallbackIFvvEE13function_moveIPS1_EEvPvPKv)
    t._ZN4mbed8CallbackIFvvEEC1EPS1_         0x08007400   Section        0  .\build\main.o(t._ZN4mbed8CallbackIFvvEEC1EPS1_)
    t._ZN4mbed8CallbackIFvvEED1Ev            0x08007430   Section        0  mbed/TARGET_NUCLEO_F070RB/TOOLCHAIN_ARM_STD/mbed.ar(RawSerial.o)(t._ZN4mbed8CallbackIFvvEED1Ev)
    t._ZN4mbed8callbackI14BufferedSerialvEENS_8CallbackIFT0_vEEEPT_MS6_FS3_vE 0x08007444   Section        0  .\build\bufferedserial.o(t._ZN4mbed8callbackI14BufferedSerialvEENS_8CallbackIFT0_vEEEPT_MS6_FS3_vE)
    t._ZN6CThunkIN4mbed10SerialBaseEE10trampolineEPS1_PvPMS1_FvS4_E 0x0800749c   Section        0  mbed/TARGET_NUCLEO_F070RB/TOOLCHAIN_ARM_STD/mbed.ar(SerialBase.o)(t._ZN6CThunkIN4mbed10SerialBaseEE10trampolineEPS1_PvPMS1_FvS4_E)
    t._ZN8MyBufferIcE3getEv                  0x080074ca   Section        0  .\build\bufferedserial.o(t._ZN8MyBufferIcE3getEv)
    t._ZN8MyBufferIcE5clearEv                0x080074f6   Section        0  .\build\mybuffer.o(t._ZN8MyBufferIcE5clearEv)
    t._ZN8MyBufferIcE9availableEv            0x0800750a   Section        0  .\build\bufferedserial.o(t._ZN8MyBufferIcE9availableEv)
    t._ZN8MyBufferIcEC1Ej                    0x0800751c   Section        0  .\build\mybuffer.o(t._ZN8MyBufferIcEC1Ej)
    t._ZN8MyBufferIcED1Ev                    0x08007536   Section        0  .\build\mybuffer.o(t._ZN8MyBufferIcED1Ev)
    t._ZN8MyBufferIcEaSEc                    0x08007544   Section        0  .\build\bufferedserial.o(t._ZN8MyBufferIcEaSEc)
    x$fpl$printf1                            0x08007578   Section       16  C:\Keil_v5\ARM\ARMCC\Bin\..\lib\armlib\fz_ps.l(printf1.o)(x$fpl$printf1)
    x$fpl$printf2                            0x08007588   Section       16  C:\Keil_v5\ARM\ARMCC\Bin\..\lib\armlib\fz_ps.l(printf2.o)(x$fpl$printf2)
    .constdata                               0x08007598   Section      108  mbed/TARGET_NUCLEO_F070RB/TOOLCHAIN_ARM_STD/PeripheralPins.o(.constdata)
    x$fpl$usenofp                            0x08007598   Section        0  C:\Keil_v5\ARM\ARMCC\Bin\..\lib\armlib\fz_ps.l(usenofp.o)(x$fpl$usenofp)
    .constdata                               0x08007604   Section      108  mbed/TARGET_NUCLEO_F070RB/TOOLCHAIN_ARM_STD/PeripheralPins.o(.constdata)
    .constdata                               0x08007670   Section       52  mbed/TARGET_NUCLEO_F070RB/TOOLCHAIN_ARM_STD/pinmap.o(.constdata)
    gpio_mode                                0x08007670   Data          52  mbed/TARGET_NUCLEO_F070RB/TOOLCHAIN_ARM_STD/pinmap.o(.constdata)
    .constdata                               0x080076a4   Section       23  mbed/TARGET_NUCLEO_F070RB/TOOLCHAIN_ARM_STD/retarget.o(.constdata)
    .constdata                               0x080076bb   Section       16  mbed/TARGET_NUCLEO_F070RB/TOOLCHAIN_ARM_STD/system_stm32f0xx.o(.constdata)
    .constdata                               0x080076cb   Section        8  mbed/TARGET_NUCLEO_F070RB/TOOLCHAIN_ARM_STD/system_stm32f0xx.o(.constdata)
    .constdata                               0x080076d3   Section        4  .\build\main.o(.constdata)
    EPCTab                                   0x080076d3   Data           4  .\build\main.o(.constdata)
    .constdata                               0x080076d8   Section       16  .\build\bufferedserial.o(.constdata)
    <Data1>                                  0x080076d8   Data           8  .\build\bufferedserial.o(.constdata)
    <Data2>                                  0x080076e0   Data           8  .\build\bufferedserial.o(.constdata)
    .constdata                               0x080076e8   Section       16  mbed/TARGET_NUCLEO_F070RB/TOOLCHAIN_ARM_STD/mbed.ar(SerialBase.o)(.constdata)
    <Data1>                                  0x080076e8   Data           8  mbed/TARGET_NUCLEO_F070RB/TOOLCHAIN_ARM_STD/mbed.ar(SerialBase.o)(.constdata)
    <Data2>                                  0x080076f0   Data           8  mbed/TARGET_NUCLEO_F070RB/TOOLCHAIN_ARM_STD/mbed.ar(SerialBase.o)(.constdata)
    .constdata                               0x080076f8   Section       20  mbed/TARGET_NUCLEO_F070RB/TOOLCHAIN_ARM_STD/mbed.ar(mbed_us_ticker_api.o)(.constdata)
    us_interface                             0x080076f8   Data          20  mbed/TARGET_NUCLEO_F070RB/TOOLCHAIN_ARM_STD/mbed.ar(mbed_us_ticker_api.o)(.constdata)
    .constdata                               0x0800770c   Section        8  mbed/TARGET_NUCLEO_F070RB/TOOLCHAIN_ARM_STD/mbed.ar(mbed_us_ticker_api.o)(.constdata)
    us_data                                  0x0800770c   Data           8  mbed/TARGET_NUCLEO_F070RB/TOOLCHAIN_ARM_STD/mbed.ar(mbed_us_ticker_api.o)(.constdata)
    .constdata                               0x08007714   Section       40  C:\Keil_v5\ARM\ARMCC\Bin\..\lib\armlib\c_p.l(_printf_hex_int_ll_ptr.o)(.constdata)
    uc_hextab                                0x08007714   Data          20  C:\Keil_v5\ARM\ARMCC\Bin\..\lib\armlib\c_p.l(_printf_hex_int_ll_ptr.o)(.constdata)
    lc_hextab                                0x08007728   Data          20  C:\Keil_v5\ARM\ARMCC\Bin\..\lib\armlib\c_p.l(_printf_hex_int_ll_ptr.o)(.constdata)
    .constdata                               0x0800773c   Section       17  C:\Keil_v5\ARM\ARMCC\Bin\..\lib\armlib\c_p.l(__printf_flags_ss_wp.o)(.constdata)
    maptable                                 0x0800773c   Data          17  C:\Keil_v5\ARM\ARMCC\Bin\..\lib\armlib\c_p.l(__printf_flags_ss_wp.o)(.constdata)
    .constdata                               0x0800774d   Section      128  C:\Keil_v5\ARM\ARMCC\Bin\..\lib\armlib\fz_ps.l(ddiv.o)(.constdata)
    ddiv_reciptbl                            0x0800774d   Data         128  C:\Keil_v5\ARM\ARMCC\Bin\..\lib\armlib\fz_ps.l(ddiv.o)(.constdata)
    .constdata                               0x080077cd   Section       64  C:\Keil_v5\ARM\ARMCC\Bin\..\lib\armlib\fz_ps.l(fdiv.o)(.constdata)
    fdiv_tab                                 0x080077cd   Data          64  C:\Keil_v5\ARM\ARMCC\Bin\..\lib\armlib\fz_ps.l(fdiv.o)(.constdata)
    .constdata                               0x08007810   Section        8  C:\Keil_v5\ARM\ARMCC\Bin\..\lib\armlib\c_p.l(_printf_wctomb.o)(.constdata)
    initial_mbstate                          0x08007810   Data           8  C:\Keil_v5\ARM\ARMCC\Bin\..\lib\armlib\c_p.l(_printf_wctomb.o)(.constdata)
    .constdata                               0x08007818   Section       38  C:\Keil_v5\ARM\ARMCC\Bin\..\lib\armlib\c_p.l(_printf_fp_hex.o)(.constdata)
    lc_hextab                                0x08007818   Data          19  C:\Keil_v5\ARM\ARMCC\Bin\..\lib\armlib\c_p.l(_printf_fp_hex.o)(.constdata)
    uc_hextab                                0x0800782b   Data          19  C:\Keil_v5\ARM\ARMCC\Bin\..\lib\armlib\c_p.l(_printf_fp_hex.o)(.constdata)
    .constdata                               0x08007840   Section      148  C:\Keil_v5\ARM\ARMCC\Bin\..\lib\armlib\c_p.l(bigflt0.o)(.constdata)
    tenpwrs_x                                0x08007840   Data          60  C:\Keil_v5\ARM\ARMCC\Bin\..\lib\armlib\c_p.l(bigflt0.o)(.constdata)
    tenpwrs_i                                0x0800787c   Data          64  C:\Keil_v5\ARM\ARMCC\Bin\..\lib\armlib\c_p.l(bigflt0.o)(.constdata)
    .constdata__ZTV14BufferedSerial          0x080078d4   Section       52  .\build\bufferedserial.o(.constdata__ZTV14BufferedSerial)
    .constdata__ZTVN4mbed10FileHandleE       0x08007908   Section       52  mbed/TARGET_NUCLEO_F070RB/TOOLCHAIN_ARM_STD/retarget.o(.constdata__ZTVN4mbed10FileHandleE)
    .constdata__ZTVN4mbed10SerialBaseE       0x0800793c   Section       24  mbed/TARGET_NUCLEO_F070RB/TOOLCHAIN_ARM_STD/mbed.ar(SerialBase.o)(.constdata__ZTVN4mbed10SerialBaseE)
    .constdata__ZTVN4mbed10TimerEventE       0x08007954   Section       20  mbed/TARGET_NUCLEO_F070RB/TOOLCHAIN_ARM_STD/mbed.ar(TimerEvent.o)(.constdata__ZTVN4mbed10TimerEventE)
    .constdata__ZTVN4mbed6SerialE            0x08007968   Section      108  mbed/TARGET_NUCLEO_F070RB/TOOLCHAIN_ARM_STD/mbed.ar(Serial.o)(.constdata__ZTVN4mbed6SerialE)
    .constdata__ZTVN4mbed6StreamE            0x080079d4   Section       76  mbed/TARGET_NUCLEO_F070RB/TOOLCHAIN_ARM_STD/mbed.ar(Stream.o)(.constdata__ZTVN4mbed6StreamE)
    .constdata__ZTVN4mbed6TickerE            0x08007a20   Section       20  mbed/TARGET_NUCLEO_F070RB/TOOLCHAIN_ARM_STD/mbed.ar(Ticker.o)(.constdata__ZTVN4mbed6TickerE)
    .constdata__ZTVN4mbed8FileBaseE          0x08007a34   Section       16  mbed/TARGET_NUCLEO_F070RB/TOOLCHAIN_ARM_STD/mbed.ar(FileBase.o)(.constdata__ZTVN4mbed8FileBaseE)
    .constdata__ZTVN4mbed8FileLikeE          0x08007a44   Section       68  mbed/TARGET_NUCLEO_F070RB/TOOLCHAIN_ARM_STD/mbed.ar(FileLike.o)(.constdata__ZTVN4mbed8FileLikeE)
    .constdata__ZTVN4mbed9RawSerialE         0x08007a88   Section       24  mbed/TARGET_NUCLEO_F070RB/TOOLCHAIN_ARM_STD/mbed.ar(RawSerial.o)(.constdata__ZTVN4mbed9RawSerialE)
    .constdata__ZZN12SingletonPtrI13PlatformMutexE3getEvEs 0x08007aa0   Section       20  mbed/TARGET_NUCLEO_F070RB/TOOLCHAIN_ARM_STD/retarget.o(.constdata__ZZN12SingletonPtrI13PlatformMutexE3getEvEs)
    .constdata__ZZN12SingletonPtrI13PlatformMutexE3getEvEs_0 0x08007ab4   Section       78  mbed/TARGET_NUCLEO_F070RB/TOOLCHAIN_ARM_STD/retarget.o(.constdata__ZZN12SingletonPtrI13PlatformMutexE3getEvEs_0)
    .constdata__ZZN4mbed8CallbackIFvvEE8generateINS2_14method_contextI14BufferedSerialMS5_FvvEEEEEvRKT_E3ops 0x08007b04   Section       12  .\build\bufferedserial.o(.constdata__ZZN4mbed8CallbackIFvvEE8generateINS2_14method_contextI14BufferedSerialMS5_FvvEEEEEvRKT_E3ops)
    .constdata__ZZN4mbed8CallbackIFvvEE8generateIPS1_EEvRKT_E3ops 0x08007b10   Section       12  mbed/TARGET_NUCLEO_F070RB/TOOLCHAIN_ARM_STD/mbed.ar(SerialBase.o)(.constdata__ZZN4mbed8CallbackIFvvEE8generateIPS1_EEvRKT_E3ops)
    .constdata__ZZNK4mbed8CallbackIFvvEE4callEvEs 0x08007b1c   Section        5  mbed/TARGET_NUCLEO_F070RB/TOOLCHAIN_ARM_STD/mbed.ar(SerialBase.o)(.constdata__ZZNK4mbed8CallbackIFvvEE4callEvEs)
    .constdata__ZZNK4mbed8CallbackIFvvEE4callEvEs_0 0x08007b21   Section       74  mbed/TARGET_NUCLEO_F070RB/TOOLCHAIN_ARM_STD/mbed.ar(SerialBase.o)(.constdata__ZZNK4mbed8CallbackIFvvEE4callEvEs_0)
    .conststring                             0x08007b6c   Section       87  mbed/TARGET_NUCLEO_F070RB/TOOLCHAIN_ARM_STD/gpio_api.o(.conststring)
    .conststring                             0x08007bc4   Section       85  mbed/TARGET_NUCLEO_F070RB/TOOLCHAIN_ARM_STD/pinmap.o(.conststring)
    .conststring                             0x08007c1c   Section       89  mbed/TARGET_NUCLEO_F070RB/TOOLCHAIN_ARM_STD/serial_api.o(.conststring)
    .conststring                             0x08007c78   Section       66  .\build\main.o(.conststring)
    .conststring                             0x08007cbc   Section       67  mbed/TARGET_NUCLEO_F070RB/TOOLCHAIN_ARM_STD/mbed.ar(mbed_critical.o)(.conststring)
    locale$$data                             0x08007d20   Section       28  C:\Keil_v5\ARM\ARMCC\Bin\..\lib\armlib\c_p.l(lc_numeric_c.o)(locale$$data)
    __lcnum_c_name                           0x08007d24   Data           2  C:\Keil_v5\ARM\ARMCC\Bin\..\lib\armlib\c_p.l(lc_numeric_c.o)(locale$$data)
    __lcnum_c_start                          0x08007d2c   Data           0  C:\Keil_v5\ARM\ARMCC\Bin\..\lib\armlib\c_p.l(lc_numeric_c.o)(locale$$data)
    __lcnum_c_point                          0x08007d38   Data           0  C:\Keil_v5\ARM\ARMCC\Bin\..\lib\armlib\c_p.l(lc_numeric_c.o)(locale$$data)
    __lcnum_c_thousands                      0x08007d3a   Data           0  C:\Keil_v5\ARM\ARMCC\Bin\..\lib\armlib\c_p.l(lc_numeric_c.o)(locale$$data)
    __lcnum_c_grouping                       0x08007d3b   Data           0  C:\Keil_v5\ARM\ARMCC\Bin\..\lib\armlib\c_p.l(lc_numeric_c.o)(locale$$data)
    locale$$data                             0x08007d3c   Section      272  C:\Keil_v5\ARM\ARMCC\Bin\..\lib\armlib\c_p.l(lc_ctype_c.o)(locale$$data)
    __lcnum_c_end                            0x08007d3c   Data           0  C:\Keil_v5\ARM\ARMCC\Bin\..\lib\armlib\c_p.l(lc_numeric_c.o)(locale$$data)
    __lcctype_c_name                         0x08007d40   Data           2  C:\Keil_v5\ARM\ARMCC\Bin\..\lib\armlib\c_p.l(lc_ctype_c.o)(locale$$data)
    __lcctype_c_start                        0x08007d48   Data           0  C:\Keil_v5\ARM\ARMCC\Bin\..\lib\armlib\c_p.l(lc_ctype_c.o)(locale$$data)
    .init_array                              0x08007e4c   Section        4  .\build\main.o(.init_array)
    __lcctype_c_end                          0x08007e4c   Data           0  C:\Keil_v5\ARM\ARMCC\Bin\..\lib\armlib\c_p.l(lc_ctype_c.o)(locale$$data)
    .init_array                              0x08007e50   Section        0  C:\Keil_v5\ARM\ARMCC\Bin\..\lib\armlib\c_p.l(init_aeabi.o)(.init_array)
    .data                                    0x200000c0   Section        4  mbed/TARGET_NUCLEO_F070RB/TOOLCHAIN_ARM_STD/hal_tick.o(.data)
    .data                                    0x200000c4   Section        8  mbed/TARGET_NUCLEO_F070RB/TOOLCHAIN_ARM_STD/retarget.o(.data)
    filehandle_mutex                         0x200000c4   Data           8  mbed/TARGET_NUCLEO_F070RB/TOOLCHAIN_ARM_STD/retarget.o(.data)
    .data                                    0x200000cc   Section        8  mbed/TARGET_NUCLEO_F070RB/TOOLCHAIN_ARM_STD/serial_api.o(.data)
    irq_handler                              0x200000d0   Data           4  mbed/TARGET_NUCLEO_F070RB/TOOLCHAIN_ARM_STD/serial_api.o(.data)
    .data                                    0x200000d4   Section        4  mbed/TARGET_NUCLEO_F070RB/TOOLCHAIN_ARM_STD/stm32f0xx_hal.o(.data)
    .data                                    0x200000d8   Section        4  mbed/TARGET_NUCLEO_F070RB/TOOLCHAIN_ARM_STD/system_stm32f0xx.o(.data)
    .data                                    0x200000dc   Section       16  mbed/TARGET_NUCLEO_F070RB/TOOLCHAIN_ARM_STD/us_ticker.o(.data)
    us_ticker_inited                         0x200000e0   Data           4  mbed/TARGET_NUCLEO_F070RB/TOOLCHAIN_ARM_STD/us_ticker.o(.data)
    .data                                    0x200000ec   Section       18  .\build\main.o(.data)
    .data                                    0x200000fe   Section       32  .\build\rfid.o(.data)
    crctable                                 0x200000fe   Data          32  .\build\rfid.o(.data)
    .data                                    0x20000120   Section        8  mbed/TARGET_NUCLEO_F070RB/TOOLCHAIN_ARM_STD/mbed.ar(mbed_us_ticker_api.o)(.data)
    events                                   0x20000120   Data           8  mbed/TARGET_NUCLEO_F070RB/TOOLCHAIN_ARM_STD/mbed.ar(mbed_us_ticker_api.o)(.data)
    .data                                    0x20000128   Section        8  mbed/TARGET_NUCLEO_F070RB/TOOLCHAIN_ARM_STD/mbed.ar(mbed_critical.o)(.data)
    critical_interrupts_disabled             0x20000128   Data           1  mbed/TARGET_NUCLEO_F070RB/TOOLCHAIN_ARM_STD/mbed.ar(mbed_critical.o)(.data)
    interrupt_enable_counter                 0x2000012c   Data           4  mbed/TARGET_NUCLEO_F070RB/TOOLCHAIN_ARM_STD/mbed.ar(mbed_critical.o)(.data)
    .data                                    0x20000130   Section       12  mbed/TARGET_NUCLEO_F070RB/TOOLCHAIN_ARM_STD/mbed.ar(FileBase.o)(.data)
    .data                                    0x2000013c   Section        4  C:\Keil_v5\ARM\ARMCC\Bin\..\lib\armlib\c_p.l(stdio_streams.o)(.data)
    .data                                    0x20000140   Section        4  C:\Keil_v5\ARM\ARMCC\Bin\..\lib\armlib\c_p.l(stdio_streams.o)(.data)
    .data                                    0x20000144   Section        4  C:\Keil_v5\ARM\ARMCC\Bin\..\lib\armlib\c_p.l(stdio_streams.o)(.data)
    .data                                    0x20000148   Section        4  C:\Keil_v5\ARM\ARMCC\Bin\..\lib\armlib\c_p.l(heapauxa.o)(.data)
    __rt_heap_escrow_base                    0x20000148   Data           4  C:\Keil_v5\ARM\ARMCC\Bin\..\lib\armlib\c_p.l(heapauxa.o)(.data)
    .bss                                     0x2000014c   Section       60  mbed/TARGET_NUCLEO_F070RB/TOOLCHAIN_ARM_STD/hal_tick.o(.bss)
    .bss                                     0x20000188   Section       64  mbed/TARGET_NUCLEO_F070RB/TOOLCHAIN_ARM_STD/retarget.o(.bss)
    filehandles                              0x20000188   Data          64  mbed/TARGET_NUCLEO_F070RB/TOOLCHAIN_ARM_STD/retarget.o(.bss)
    .bss                                     0x200001c8   Section      540  mbed/TARGET_NUCLEO_F070RB/TOOLCHAIN_ARM_STD/serial_api.o(.bss)
    serial_irq_ids                           0x200001c8   Data          16  mbed/TARGET_NUCLEO_F070RB/TOOLCHAIN_ARM_STD/serial_api.o(.bss)
    uart_handlers                            0x200001d8   Data         448  mbed/TARGET_NUCLEO_F070RB/TOOLCHAIN_ARM_STD/serial_api.o(.bss)
    .bss                                     0x200003e4   Section       60  mbed/TARGET_NUCLEO_F070RB/TOOLCHAIN_ARM_STD/us_ticker.o(.bss)
    TimMasterHandle                          0x200003e4   Data          60  mbed/TARGET_NUCLEO_F070RB/TOOLCHAIN_ARM_STD/us_ticker.o(.bss)
    .bss                                     0x20000420   Section      772  .\build\main.o(.bss)
    .bss                                     0x20000724   Section       84  C:\Keil_v5\ARM\ARMCC\Bin\..\lib\armlib\c_p.l(stdio_streams.o)(.bss)
    .bss                                     0x20000778   Section       84  C:\Keil_v5\ARM\ARMCC\Bin\..\lib\armlib\c_p.l(stdio_streams.o)(.bss)
    .bss                                     0x200007cc   Section       84  C:\Keil_v5\ARM\ARMCC\Bin\..\lib\armlib\c_p.l(stdio_streams.o)(.bss)
    .bss                                     0x20000820   Section        4  C:\Keil_v5\ARM\ARMCC\Bin\..\lib\armlib\c_p.l(rt_heap_descriptor.o)(.bss)
    __rt_heap_descriptor_data                0x20000820   Data           4  C:\Keil_v5\ARM\ARMCC\Bin\..\lib\armlib\c_p.l(rt_heap_descriptor.o)(.bss)
    .bss                                     0x20000824   Section       20  C:\Keil_v5\ARM\ARMCC\Bin\..\lib\armlib\c_p.l(rt_locale.o)(.bss)
    __rt_locale_data                         0x20000824   Data          20  C:\Keil_v5\ARM\ARMCC\Bin\..\lib\armlib\c_p.l(rt_locale.o)(.bss)
    .bss                                     0x20000838   Section        4  C:\Keil_v5\ARM\ARMCC\Bin\..\lib\armlib\c_p.l(rt_errno_addr.o)(.bss)
    __aeabi_errno_addr_data                  0x20000838   Data           4  C:\Keil_v5\ARM\ARMCC\Bin\..\lib\armlib\c_p.l(rt_errno_addr.o)(.bss)

    Global Symbols

    Symbol Name                              Value     Ov Type        Size  Object(Section)

    BuildAttributes$$THM_ISAv3M$S$PE$A:L22$X:L11$S22$IEEE1$IW$USESV6$~STKCKD$USESV7$~SHL$OTIME$ROPI$IEEEX$EBA8$UX$STANDARDLIB$REQ8$PRES8$EABIv2 0x00000000   Number         0  anon$$obj.o ABSOLUTE
    __ARM_use_no_argv                        0x00000000   Number         0  .\build\main.o ABSOLUTE
    _printf_flags                            0x00000000   Number         0  C:\Keil_v5\ARM\ARMCC\Bin\..\lib\armlib\c_p.l(printf_stubs.o) ABSOLUTE
    _printf_return_value                     0x00000000   Number         0  C:\Keil_v5\ARM\ARMCC\Bin\..\lib\armlib\c_p.l(printf_stubs.o) ABSOLUTE
    _printf_sizespec                         0x00000000   Number         0  C:\Keil_v5\ARM\ARMCC\Bin\..\lib\armlib\c_p.l(printf_stubs.o) ABSOLUTE
    _printf_widthprec                        0x00000000   Number         0  C:\Keil_v5\ARM\ARMCC\Bin\..\lib\armlib\c_p.l(printf_stubs.o) ABSOLUTE
    SHT$$ARM_EXIDX$$Base                      - Undefined Reference
    SHT$$ARM_EXIDX$$Limit                     - Undefined Reference
    __ARM::default_unexpected_handler()       - Undefined Weak Reference
    __ARM_exceptions_buffer_required          - Undefined Weak Reference
    __ARM_exceptions_init                     - Undefined Weak Reference
    __aeabi_unwind_cpp_pr1                    - Undefined Weak Reference
    __aeabi_unwind_cpp_pr2                    - Undefined Weak Reference
    __alloca_initialize                       - Undefined Weak Reference
    __arm_preinit_                            - Undefined Weak Reference
    __cxa_begin_cleanup                       - Undefined Weak Reference
    __cxa_call_unexpected                     - Undefined Weak Reference
    __cxa_type_match                          - Undefined Weak Reference
    __rt_lib_shutdown                         - Undefined Weak Reference
    __sigvec_lookup                           - Undefined Weak Reference
    __user_heap_extent                        - Undefined Weak Reference
    _atexit_init                              - Undefined Weak Reference
    _clock_init                               - Undefined Weak Reference
    _fp_trap_init                             - Undefined Weak Reference
    _fp_trap_shutdown                         - Undefined Weak Reference
    _get_lc_collate                           - Undefined Weak Reference
    _get_lc_monetary                          - Undefined Weak Reference
    _get_lc_time                              - Undefined Weak Reference
    _getenv_init                              - Undefined Weak Reference
    _handle_redirection                       - Undefined Weak Reference
    _mutex_acquire                            - Undefined Weak Reference
    _mutex_free                               - Undefined Weak Reference
    _mutex_release                            - Undefined Weak Reference
    _printf_mbtowc                            - Undefined Weak Reference
    _printf_wc                                - Undefined Weak Reference
    _rand_init                                - Undefined Weak Reference
    _signal_finish                            - Undefined Weak Reference
    _signal_init                              - Undefined Weak Reference
    __Vectors_Size                           0x000000c0   Number         0  mbed/TARGET_NUCLEO_F070RB/TOOLCHAIN_ARM_STD/startup_stm32f070xb.o ABSOLUTE
    __Vectors                                0x08000000   Data           4  mbed/TARGET_NUCLEO_F070RB/TOOLCHAIN_ARM_STD/startup_stm32f070xb.o(RESET)
    __dso_handle                             0x08000000   Number         0  mbed/TARGET_NUCLEO_F070RB/TOOLCHAIN_ARM_STD/startup_stm32f070xb.o(RESET)
    __Vectors_End                            0x080000c0   Data           0  mbed/TARGET_NUCLEO_F070RB/TOOLCHAIN_ARM_STD/startup_stm32f070xb.o(RESET)
    __main                                   0x080000c1   Thumb Code     8  C:\Keil_v5\ARM\ARMCC\Bin\..\lib\armlib\c_p.l(__main.o)(!!!main)
    __scatterload                            0x080000c9   Thumb Code     0  C:\Keil_v5\ARM\ARMCC\Bin\..\lib\armlib\c_p.l(__scatter.o)(!!!scatter)
    __scatterload_rt2                        0x080000c9   Thumb Code    52  C:\Keil_v5\ARM\ARMCC\Bin\..\lib\armlib\c_p.l(__scatter.o)(!!!scatter)
    __scatterload_rt2_thumb_only             0x080000c9   Thumb Code     0  C:\Keil_v5\ARM\ARMCC\Bin\..\lib\armlib\c_p.l(__scatter.o)(!!!scatter)
    __scatterload_null                       0x080000d9   Thumb Code     0  C:\Keil_v5\ARM\ARMCC\Bin\..\lib\armlib\c_p.l(__scatter.o)(!!!scatter)
    __scatterload_copy                       0x08000105   Thumb Code    26  C:\Keil_v5\ARM\ARMCC\Bin\..\lib\armlib\c_p.l(__scatter_copy.o)(!!handler_copy)
    __scatterload_zeroinit                   0x08000121   Thumb Code    28  C:\Keil_v5\ARM\ARMCC\Bin\..\lib\armlib\c_p.l(__scatter_zi.o)(!!handler_zi)
    _printf_percent                          0x0800013d   Thumb Code     0  C:\Keil_v5\ARM\ARMCC\Bin\..\lib\armlib\c_p.l(_printf_percent.o)(.ARM.Collect$$_printf_percent$$00000000)
    _printf_n                                0x0800013f   Thumb Code     0  C:\Keil_v5\ARM\ARMCC\Bin\..\lib\armlib\c_p.l(_printf_n.o)(.ARM.Collect$$_printf_percent$$00000001)
    _printf_p                                0x08000149   Thumb Code     0  C:\Keil_v5\ARM\ARMCC\Bin\..\lib\armlib\c_p.l(_printf_p.o)(.ARM.Collect$$_printf_percent$$00000002)
    _printf_f                                0x08000153   Thumb Code     0  C:\Keil_v5\ARM\ARMCC\Bin\..\lib\armlib\c_p.l(_printf_f.o)(.ARM.Collect$$_printf_percent$$00000003)
    _printf_e                                0x0800015d   Thumb Code     0  C:\Keil_v5\ARM\ARMCC\Bin\..\lib\armlib\c_p.l(_printf_e.o)(.ARM.Collect$$_printf_percent$$00000004)
    _printf_g                                0x08000167   Thumb Code     0  C:\Keil_v5\ARM\ARMCC\Bin\..\lib\armlib\c_p.l(_printf_g.o)(.ARM.Collect$$_printf_percent$$00000005)
    _printf_a                                0x08000171   Thumb Code     0  C:\Keil_v5\ARM\ARMCC\Bin\..\lib\armlib\c_p.l(_printf_a.o)(.ARM.Collect$$_printf_percent$$00000006)
    _printf_ll                               0x0800017b   Thumb Code     0  C:\Keil_v5\ARM\ARMCC\Bin\..\lib\armlib\c_p.l(_printf_ll.o)(.ARM.Collect$$_printf_percent$$00000007)
    _printf_i                                0x08000185   Thumb Code     0  C:\Keil_v5\ARM\ARMCC\Bin\..\lib\armlib\c_p.l(_printf_i.o)(.ARM.Collect$$_printf_percent$$00000008)
    _printf_d                                0x0800018f   Thumb Code     0  C:\Keil_v5\ARM\ARMCC\Bin\..\lib\armlib\c_p.l(_printf_d.o)(.ARM.Collect$$_printf_percent$$00000009)
    _printf_u                                0x08000199   Thumb Code     0  C:\Keil_v5\ARM\ARMCC\Bin\..\lib\armlib\c_p.l(_printf_u.o)(.ARM.Collect$$_printf_percent$$0000000A)
    _printf_o                                0x080001a3   Thumb Code     0  C:\Keil_v5\ARM\ARMCC\Bin\..\lib\armlib\c_p.l(_printf_o.o)(.ARM.Collect$$_printf_percent$$0000000B)
    _printf_x                                0x080001ad   Thumb Code     0  C:\Keil_v5\ARM\ARMCC\Bin\..\lib\armlib\c_p.l(_printf_x.o)(.ARM.Collect$$_printf_percent$$0000000C)
    _printf_lli                              0x080001b7   Thumb Code     0  C:\Keil_v5\ARM\ARMCC\Bin\..\lib\armlib\c_p.l(_printf_lli.o)(.ARM.Collect$$_printf_percent$$0000000D)
    _printf_lld                              0x080001c1   Thumb Code     0  C:\Keil_v5\ARM\ARMCC\Bin\..\lib\armlib\c_p.l(_printf_lld.o)(.ARM.Collect$$_printf_percent$$0000000E)
    _printf_llu                              0x080001cb   Thumb Code     0  C:\Keil_v5\ARM\ARMCC\Bin\..\lib\armlib\c_p.l(_printf_llu.o)(.ARM.Collect$$_printf_percent$$0000000F)
    _printf_llo                              0x080001d5   Thumb Code     0  C:\Keil_v5\ARM\ARMCC\Bin\..\lib\armlib\c_p.l(_printf_llo.o)(.ARM.Collect$$_printf_percent$$00000010)
    _printf_llx                              0x080001df   Thumb Code     0  C:\Keil_v5\ARM\ARMCC\Bin\..\lib\armlib\c_p.l(_printf_llx.o)(.ARM.Collect$$_printf_percent$$00000011)
    _printf_l                                0x080001e9   Thumb Code     0  C:\Keil_v5\ARM\ARMCC\Bin\..\lib\armlib\c_p.l(_printf_l.o)(.ARM.Collect$$_printf_percent$$00000012)
    _printf_c                                0x080001f3   Thumb Code     0  C:\Keil_v5\ARM\ARMCC\Bin\..\lib\armlib\c_p.l(_printf_c.o)(.ARM.Collect$$_printf_percent$$00000013)
    _printf_s                                0x080001fd   Thumb Code     0  C:\Keil_v5\ARM\ARMCC\Bin\..\lib\armlib\c_p.l(_printf_s.o)(.ARM.Collect$$_printf_percent$$00000014)
    _printf_lc                               0x08000207   Thumb Code     0  C:\Keil_v5\ARM\ARMCC\Bin\..\lib\armlib\c_p.l(_printf_lc.o)(.ARM.Collect$$_printf_percent$$00000015)
    _printf_ls                               0x08000211   Thumb Code     0  C:\Keil_v5\ARM\ARMCC\Bin\..\lib\armlib\c_p.l(_printf_ls.o)(.ARM.Collect$$_printf_percent$$00000016)
    _printf_percent_end                      0x0800021b   Thumb Code     0  C:\Keil_v5\ARM\ARMCC\Bin\..\lib\armlib\c_p.l(_printf_percent_end.o)(.ARM.Collect$$_printf_percent$$00000017)
    __rt_lib_init                            0x0800021f   Thumb Code     0  C:\Keil_v5\ARM\ARMCC\Bin\..\lib\armlib\c_p.l(libinit.o)(.ARM.Collect$$libinit$$00000000)
    __rt_lib_init_fp_1                       0x08000221   Thumb Code     0  C:\Keil_v5\ARM\ARMCC\Bin\..\lib\armlib\c_p.l(libinit2.o)(.ARM.Collect$$libinit$$00000002)
    __rt_lib_init_heap_2                     0x08000221   Thumb Code     0  C:\Keil_v5\ARM\ARMCC\Bin\..\lib\armlib\c_p.l(libinit2.o)(.ARM.Collect$$libinit$$00000005)
    __rt_lib_init_preinit_1                  0x08000221   Thumb Code     0  C:\Keil_v5\ARM\ARMCC\Bin\..\lib\armlib\c_p.l(libinit2.o)(.ARM.Collect$$libinit$$00000004)
    __rt_lib_init_heap_1                     0x08000229   Thumb Code     0  C:\Keil_v5\ARM\ARMCC\Bin\..\lib\armlib\c_p.l(libinit2.o)(.ARM.Collect$$libinit$$0000000A)
    __rt_lib_init_lc_common                  0x08000229   Thumb Code     0  C:\Keil_v5\ARM\ARMCC\Bin\..\lib\armlib\c_p.l(libinit2.o)(.ARM.Collect$$libinit$$0000000F)
    __rt_lib_init_rand_1                     0x08000229   Thumb Code     0  C:\Keil_v5\ARM\ARMCC\Bin\..\lib\armlib\c_p.l(libinit2.o)(.ARM.Collect$$libinit$$0000000E)
    __rt_lib_init_user_alloc_1               0x08000229   Thumb Code     0  C:\Keil_v5\ARM\ARMCC\Bin\..\lib\armlib\c_p.l(libinit2.o)(.ARM.Collect$$libinit$$0000000C)
    __rt_lib_init_lc_collate_1               0x0800022f   Thumb Code     0  C:\Keil_v5\ARM\ARMCC\Bin\..\lib\armlib\c_p.l(libinit2.o)(.ARM.Collect$$libinit$$00000011)
    __rt_lib_init_lc_ctype_2                 0x0800022f   Thumb Code     0  C:\Keil_v5\ARM\ARMCC\Bin\..\lib\armlib\c_p.l(libinit2.o)(.ARM.Collect$$libinit$$00000012)
    __rt_lib_init_lc_ctype_1                 0x0800023b   Thumb Code     0  C:\Keil_v5\ARM\ARMCC\Bin\..\lib\armlib\c_p.l(libinit2.o)(.ARM.Collect$$libinit$$00000013)
    __rt_lib_init_lc_monetary_1              0x0800023b   Thumb Code     0  C:\Keil_v5\ARM\ARMCC\Bin\..\lib\armlib\c_p.l(libinit2.o)(.ARM.Collect$$libinit$$00000015)
    __rt_lib_init_lc_numeric_2               0x0800023b   Thumb Code     0  C:\Keil_v5\ARM\ARMCC\Bin\..\lib\armlib\c_p.l(libinit2.o)(.ARM.Collect$$libinit$$00000016)
    __rt_lib_init_atexit_1                   0x08000245   Thumb Code     0  C:\Keil_v5\ARM\ARMCC\Bin\..\lib\armlib\c_p.l(libinit2.o)(.ARM.Collect$$libinit$$0000001B)
    __rt_lib_init_clock_1                    0x08000245   Thumb Code     0  C:\Keil_v5\ARM\ARMCC\Bin\..\lib\armlib\c_p.l(libinit2.o)(.ARM.Collect$$libinit$$00000021)
    __rt_lib_init_fp_trap_1                  0x08000245   Thumb Code     0  C:\Keil_v5\ARM\ARMCC\Bin\..\lib\armlib\c_p.l(libinit2.o)(.ARM.Collect$$libinit$$0000001F)
    __rt_lib_init_getenv_1                   0x08000245   Thumb Code     0  C:\Keil_v5\ARM\ARMCC\Bin\..\lib\armlib\c_p.l(libinit2.o)(.ARM.Collect$$libinit$$00000023)
    __rt_lib_init_lc_numeric_1               0x08000245   Thumb Code     0  C:\Keil_v5\ARM\ARMCC\Bin\..\lib\armlib\c_p.l(libinit2.o)(.ARM.Collect$$libinit$$00000017)
    __rt_lib_init_lc_time_1                  0x08000245   Thumb Code     0  C:\Keil_v5\ARM\ARMCC\Bin\..\lib\armlib\c_p.l(libinit2.o)(.ARM.Collect$$libinit$$00000019)
    __rt_lib_init_signal_1                   0x08000245   Thumb Code     0  C:\Keil_v5\ARM\ARMCC\Bin\..\lib\armlib\c_p.l(libinit2.o)(.ARM.Collect$$libinit$$0000001D)
    __rt_lib_init_stdio_2                    0x08000245   Thumb Code     0  C:\Keil_v5\ARM\ARMCC\Bin\..\lib\armlib\c_p.l(libinit2.o)(.ARM.Collect$$libinit$$00000024)
    __rt_lib_init_alloca_1                   0x08000249   Thumb Code     0  C:\Keil_v5\ARM\ARMCC\Bin\..\lib\armlib\c_p.l(libinit2.o)(.ARM.Collect$$libinit$$0000002E)
    __rt_lib_init_argv_1                     0x08000249   Thumb Code     0  C:\Keil_v5\ARM\ARMCC\Bin\..\lib\armlib\c_p.l(libinit2.o)(.ARM.Collect$$libinit$$0000002C)
    __rt_lib_init_cpp_2                      0x08000249   Thumb Code     0  C:\Keil_v5\ARM\ARMCC\Bin\..\lib\armlib\c_p.l(libinit2.o)(.ARM.Collect$$libinit$$00000031)
    __rt_lib_init_exceptions_1               0x08000249   Thumb Code     0  C:\Keil_v5\ARM\ARMCC\Bin\..\lib\armlib\c_p.l(libinit2.o)(.ARM.Collect$$libinit$$00000030)
    __rt_lib_init_stdio_1                    0x08000249   Thumb Code     0  C:\Keil_v5\ARM\ARMCC\Bin\..\lib\armlib\c_p.l(libinit2.o)(.ARM.Collect$$libinit$$00000025)
    __rt_lib_init_cpp_1                      0x0800024d   Thumb Code     0  C:\Keil_v5\ARM\ARMCC\Bin\..\lib\armlib\c_p.l(libinit2.o)(.ARM.Collect$$libinit$$00000032)
    __rt_lib_init_return                     0x0800024d   Thumb Code     0  C:\Keil_v5\ARM\ARMCC\Bin\..\lib\armlib\c_p.l(libinit2.o)(.ARM.Collect$$libinit$$00000033)
    __rt_entry                               0x0800024f   Thumb Code     0  C:\Keil_v5\ARM\ARMCC\Bin\..\lib\armlib\c_p.l(__rtentry.o)(.ARM.Collect$$rtentry$$00000000)
    __rt_entry_presh_1                       0x0800024f   Thumb Code     0  C:\Keil_v5\ARM\ARMCC\Bin\..\lib\armlib\c_p.l(__rtentry2.o)(.ARM.Collect$$rtentry$$00000002)
    __rt_entry_sh                            0x0800024f   Thumb Code     0  C:\Keil_v5\ARM\ARMCC\Bin\..\lib\armlib\c_p.l(__rtentry4.o)(.ARM.Collect$$rtentry$$00000004)
    __rt_lib_shutdown_stdio_2                0x0800024f   Thumb Code     0  C:\Keil_v5\ARM\ARMCC\Bin\..\lib\armlib\c_p.l(libshutdown2.o)(.ARM.Collect$$libshutdown$$00000004)
    __rt_entry_postsh_1                      0x08000255   Thumb Code     0  C:\Keil_v5\ARM\ARMCC\Bin\..\lib\armlib\c_p.l(__rtentry2.o)(.ARM.Collect$$rtentry$$00000008)
    __rt_entry_li                            0x0800025d   Thumb Code     0  C:\Keil_v5\ARM\ARMCC\Bin\..\lib\armlib\c_p.l(__rtentry2.o)(.ARM.Collect$$rtentry$$0000000A)
    __rt_entry_main                          0x08000261   Thumb Code     0  C:\Keil_v5\ARM\ARMCC\Bin\..\lib\armlib\c_p.l(__rtentry2.o)(.ARM.Collect$$rtentry$$0000000D)
    __rt_entry_postli_1                      0x08000261   Thumb Code     0  C:\Keil_v5\ARM\ARMCC\Bin\..\lib\armlib\c_p.l(__rtentry2.o)(.ARM.Collect$$rtentry$$0000000C)
    __aeabi_memcpy4                          0x08000269   Thumb Code    56  C:\Keil_v5\ARM\ARMCC\Bin\..\lib\armlib\c_p.l(rt_memcpy.o)(.emb_text)
    __aeabi_memcpy8                          0x08000269   Thumb Code     0  C:\Keil_v5\ARM\ARMCC\Bin\..\lib\armlib\c_p.l(rt_memcpy.o)(.emb_text)
    Reset_Handler                            0x080002a1   Thumb Code     8  mbed/TARGET_NUCLEO_F070RB/TOOLCHAIN_ARM_STD/startup_stm32f070xb.o(.text)
    _maybe_terminate_alloc                   0x080002a1   Thumb Code     0  C:\Keil_v5\ARM\ARMCC\Bin\..\lib\armlib\c_p.l(maybetermalloc1.o)(.emb_text)
    NMI_Handler                              0x080002a9   Thumb Code     2  mbed/TARGET_NUCLEO_F070RB/TOOLCHAIN_ARM_STD/startup_stm32f070xb.o(.text)
    HardFault_Handler                        0x080002ab   Thumb Code     2  mbed/TARGET_NUCLEO_F070RB/TOOLCHAIN_ARM_STD/startup_stm32f070xb.o(.text)
    SVC_Handler                              0x080002ad   Thumb Code     2  mbed/TARGET_NUCLEO_F070RB/TOOLCHAIN_ARM_STD/startup_stm32f070xb.o(.text)
    PendSV_Handler                           0x080002af   Thumb Code     2  mbed/TARGET_NUCLEO_F070RB/TOOLCHAIN_ARM_STD/startup_stm32f070xb.o(.text)
    SysTick_Handler                          0x080002b1   Thumb Code     2  mbed/TARGET_NUCLEO_F070RB/TOOLCHAIN_ARM_STD/startup_stm32f070xb.o(.text)
    ADC1_IRQHandler                          0x080002b3   Thumb Code     0  mbed/TARGET_NUCLEO_F070RB/TOOLCHAIN_ARM_STD/startup_stm32f070xb.o(.text)
    DMA1_Channel1_IRQHandler                 0x080002b3   Thumb Code     0  mbed/TARGET_NUCLEO_F070RB/TOOLCHAIN_ARM_STD/startup_stm32f070xb.o(.text)
    DMA1_Channel2_3_IRQHandler               0x080002b3   Thumb Code     0  mbed/TARGET_NUCLEO_F070RB/TOOLCHAIN_ARM_STD/startup_stm32f070xb.o(.text)
    DMA1_Channel4_5_IRQHandler               0x080002b3   Thumb Code     0  mbed/TARGET_NUCLEO_F070RB/TOOLCHAIN_ARM_STD/startup_stm32f070xb.o(.text)
    EXTI0_1_IRQHandler                       0x080002b3   Thumb Code     0  mbed/TARGET_NUCLEO_F070RB/TOOLCHAIN_ARM_STD/startup_stm32f070xb.o(.text)
    EXTI2_3_IRQHandler                       0x080002b3   Thumb Code     0  mbed/TARGET_NUCLEO_F070RB/TOOLCHAIN_ARM_STD/startup_stm32f070xb.o(.text)
    EXTI4_15_IRQHandler                      0x080002b3   Thumb Code     0  mbed/TARGET_NUCLEO_F070RB/TOOLCHAIN_ARM_STD/startup_stm32f070xb.o(.text)
    FLASH_IRQHandler                         0x080002b3   Thumb Code     0  mbed/TARGET_NUCLEO_F070RB/TOOLCHAIN_ARM_STD/startup_stm32f070xb.o(.text)
    I2C1_IRQHandler                          0x080002b3   Thumb Code     0  mbed/TARGET_NUCLEO_F070RB/TOOLCHAIN_ARM_STD/startup_stm32f070xb.o(.text)
    I2C2_IRQHandler                          0x080002b3   Thumb Code     0  mbed/TARGET_NUCLEO_F070RB/TOOLCHAIN_ARM_STD/startup_stm32f070xb.o(.text)
    RCC_IRQHandler                           0x080002b3   Thumb Code     0  mbed/TARGET_NUCLEO_F070RB/TOOLCHAIN_ARM_STD/startup_stm32f070xb.o(.text)
    RTC_IRQHandler                           0x080002b3   Thumb Code     0  mbed/TARGET_NUCLEO_F070RB/TOOLCHAIN_ARM_STD/startup_stm32f070xb.o(.text)
    SPI1_IRQHandler                          0x080002b3   Thumb Code     0  mbed/TARGET_NUCLEO_F070RB/TOOLCHAIN_ARM_STD/startup_stm32f070xb.o(.text)
    SPI2_IRQHandler                          0x080002b3   Thumb Code     0  mbed/TARGET_NUCLEO_F070RB/TOOLCHAIN_ARM_STD/startup_stm32f070xb.o(.text)
    TIM14_IRQHandler                         0x080002b3   Thumb Code     0  mbed/TARGET_NUCLEO_F070RB/TOOLCHAIN_ARM_STD/startup_stm32f070xb.o(.text)
    TIM15_IRQHandler                         0x080002b3   Thumb Code     0  mbed/TARGET_NUCLEO_F070RB/TOOLCHAIN_ARM_STD/startup_stm32f070xb.o(.text)
    TIM16_IRQHandler                         0x080002b3   Thumb Code     0  mbed/TARGET_NUCLEO_F070RB/TOOLCHAIN_ARM_STD/startup_stm32f070xb.o(.text)
    TIM17_IRQHandler                         0x080002b3   Thumb Code     0  mbed/TARGET_NUCLEO_F070RB/TOOLCHAIN_ARM_STD/startup_stm32f070xb.o(.text)
    TIM1_BRK_UP_TRG_COM_IRQHandler           0x080002b3   Thumb Code     0  mbed/TARGET_NUCLEO_F070RB/TOOLCHAIN_ARM_STD/startup_stm32f070xb.o(.text)
    TIM1_CC_IRQHandler                       0x080002b3   Thumb Code     0  mbed/TARGET_NUCLEO_F070RB/TOOLCHAIN_ARM_STD/startup_stm32f070xb.o(.text)
    TIM3_IRQHandler                          0x080002b3   Thumb Code     0  mbed/TARGET_NUCLEO_F070RB/TOOLCHAIN_ARM_STD/startup_stm32f070xb.o(.text)
    TIM6_IRQHandler                          0x080002b3   Thumb Code     0  mbed/TARGET_NUCLEO_F070RB/TOOLCHAIN_ARM_STD/startup_stm32f070xb.o(.text)
    TIM7_IRQHandler                          0x080002b3   Thumb Code     0  mbed/TARGET_NUCLEO_F070RB/TOOLCHAIN_ARM_STD/startup_stm32f070xb.o(.text)
    USART1_IRQHandler                        0x080002b3   Thumb Code     0  mbed/TARGET_NUCLEO_F070RB/TOOLCHAIN_ARM_STD/startup_stm32f070xb.o(.text)
    USART2_IRQHandler                        0x080002b3   Thumb Code     0  mbed/TARGET_NUCLEO_F070RB/TOOLCHAIN_ARM_STD/startup_stm32f070xb.o(.text)
    USART3_4_IRQHandler                      0x080002b3   Thumb Code     0  mbed/TARGET_NUCLEO_F070RB/TOOLCHAIN_ARM_STD/startup_stm32f070xb.o(.text)
    USB_IRQHandler                           0x080002b3   Thumb Code     0  mbed/TARGET_NUCLEO_F070RB/TOOLCHAIN_ARM_STD/startup_stm32f070xb.o(.text)
    WWDG_IRQHandler                          0x080002b3   Thumb Code     0  mbed/TARGET_NUCLEO_F070RB/TOOLCHAIN_ARM_STD/startup_stm32f070xb.o(.text)
    malloc                                   0x080002bd   Thumb Code    98  C:\Keil_v5\ARM\ARMCC\Bin\..\lib\armlib\c_p.l(h1_alloc.o)(.text)
    free                                     0x0800031f   Thumb Code    76  C:\Keil_v5\ARM\ARMCC\Bin\..\lib\armlib\c_p.l(h1_free.o)(.text)
    vsprintf                                 0x0800036d   Thumb Code    32  C:\Keil_v5\ARM\ARMCC\Bin\..\lib\armlib\c_p.l(vsprintf.o)(.text)
    __c89vfprintf                            0x08000391   Thumb Code    14  C:\Keil_v5\ARM\ARMCC\Bin\..\lib\armlib\c_p.l(c89vfprintf.o)(.text)
    __2sprintf                               0x080003a1   Thumb Code    40  C:\Keil_v5\ARM\ARMCC\Bin\..\lib\armlib\c_p.l(__2sprintf.o)(.text)
    _printf_longlong_hex                     0x080003cd   Thumb Code    88  C:\Keil_v5\ARM\ARMCC\Bin\..\lib\armlib\c_p.l(_printf_hex_int_ll_ptr.o)(.text)
    _printf_int_hex                          0x08000425   Thumb Code    28  C:\Keil_v5\ARM\ARMCC\Bin\..\lib\armlib\c_p.l(_printf_hex_int_ll_ptr.o)(.text)
    _printf_ll_hex                           0x08000441   Thumb Code    10  C:\Keil_v5\ARM\ARMCC\Bin\..\lib\armlib\c_p.l(_printf_hex_int_ll_ptr.o)(.text)
    _printf_hex_ptr                          0x0800044b   Thumb Code    22  C:\Keil_v5\ARM\ARMCC\Bin\..\lib\armlib\c_p.l(_printf_hex_int_ll_ptr.o)(.text)
    __printf                                 0x08000465   Thumb Code   386  C:\Keil_v5\ARM\ARMCC\Bin\..\lib\armlib\c_p.l(__printf_flags_ss_wp.o)(.text)
    __0sscanf                                0x080005ed   Thumb Code    54  C:\Keil_v5\ARM\ARMCC\Bin\..\lib\armlib\c_p.l(__0sscanf.o)(.text)
    _scanf_int                               0x0800062d   Thumb Code   330  C:\Keil_v5\ARM\ARMCC\Bin\..\lib\armlib\c_p.l(_scanf_int.o)(.text)
    _do_fflush                               0x08000779   Thumb Code    54  C:\Keil_v5\ARM\ARMCC\Bin\..\lib\armlib\c_p.l(fflush.o)(.text)
    fflush                                   0x080007af   Thumb Code    46  C:\Keil_v5\ARM\ARMCC\Bin\..\lib\armlib\c_p.l(fflush.o)(.text)
    freopen                                  0x080007e1   Thumb Code   148  C:\Keil_v5\ARM\ARMCC\Bin\..\lib\armlib\c_p.l(fopen.o)(.text)
    fopen                                    0x08000875   Thumb Code    76  C:\Keil_v5\ARM\ARMCC\Bin\..\lib\armlib\c_p.l(fopen.o)(.text)
    setbuf                                   0x080008c9   Thumb Code    26  C:\Keil_v5\ARM\ARMCC\Bin\..\lib\armlib\c_p.l(setbuf.o)(.text)
    _fclose_internal                         0x080008e5   Thumb Code    72  C:\Keil_v5\ARM\ARMCC\Bin\..\lib\armlib\c_p.l(fclose.o)(.text)
    fclose                                   0x080008e5   Thumb Code     0  C:\Keil_v5\ARM\ARMCC\Bin\..\lib\armlib\c_p.l(fclose.o)(.text)
    strlen                                   0x08000931   Thumb Code    62  C:\Keil_v5\ARM\ARMCC\Bin\..\lib\armlib\c_p.l(strlen.o)(.text)
    strncmp                                  0x08000975   Thumb Code   154  C:\Keil_v5\ARM\ARMCC\Bin\..\lib\armlib\c_p.l(strncmp.o)(.text)
    _memset_w                                0x08000a15   Thumb Code    26  C:\Keil_v5\ARM\ARMCC\Bin\..\lib\armlib\c_p.l(rt_memclr.o)(.text)
    _memset                                  0x08000a2f   Thumb Code    30  C:\Keil_v5\ARM\ARMCC\Bin\..\lib\armlib\c_p.l(rt_memclr.o)(.text)
    __aeabi_memclr                           0x08000a4d   Thumb Code     4  C:\Keil_v5\ARM\ARMCC\Bin\..\lib\armlib\c_p.l(rt_memclr.o)(.text)
    __rt_memclr                              0x08000a4d   Thumb Code     0  C:\Keil_v5\ARM\ARMCC\Bin\..\lib\armlib\c_p.l(rt_memclr.o)(.text)
    __aeabi_memclr4                          0x08000a51   Thumb Code     0  C:\Keil_v5\ARM\ARMCC\Bin\..\lib\armlib\c_p.l(rt_memclr.o)(.text)
    __aeabi_memclr8                          0x08000a51   Thumb Code     0  C:\Keil_v5\ARM\ARMCC\Bin\..\lib\armlib\c_p.l(rt_memclr.o)(.text)
    __rt_memclr_w                            0x08000a51   Thumb Code     4  C:\Keil_v5\ARM\ARMCC\Bin\..\lib\armlib\c_p.l(rt_memclr.o)(.text)
    strcmp                                   0x08000a55   Thumb Code   160  C:\Keil_v5\ARM\ARMCC\Bin\..\lib\armlib\c_p.l(strcmpv6m.o)(.text)
    __aeabi_uidiv                            0x08000af5   Thumb Code     0  C:\Keil_v5\ARM\ARMCC\Bin\..\lib\armlib\c_p.l(aeabi_sdivfast.o)(.text)
    __aeabi_uidivmod                         0x08000af5   Thumb Code    28  C:\Keil_v5\ARM\ARMCC\Bin\..\lib\armlib\c_p.l(aeabi_sdivfast.o)(.text)
    __aeabi_idiv                             0x08000b11   Thumb Code     0  C:\Keil_v5\ARM\ARMCC\Bin\..\lib\armlib\c_p.l(aeabi_sdivfast.o)(.text)
    __aeabi_idivmod                          0x08000b11   Thumb Code   460  C:\Keil_v5\ARM\ARMCC\Bin\..\lib\armlib\c_p.l(aeabi_sdivfast.o)(.text)
    __cpp_initialize__aeabi_                 0x08000cdd   Thumb Code    26  C:\Keil_v5\ARM\ARMCC\Bin\..\lib\armlib\c_p.l(init_aeabi.o)(.text)
    __aeabi_vec_dtor                         0x08000d01   Thumb Code    34  C:\Keil_v5\ARM\ARMCC\Bin\..\lib\cpplib\cpprt_p.l(aeabi_vec_dtor_noexceptions.o)(.text)
    __aeabi_ddiv                             0x08000d25   Thumb Code     0  C:\Keil_v5\ARM\ARMCC\Bin\..\lib\armlib\fz_ps.l(ddiv.o)(.text)
    _ddiv                                    0x08000d25   Thumb Code  1072  C:\Keil_v5\ARM\ARMCC\Bin\..\lib\armlib\fz_ps.l(ddiv.o)(.text)
    _drdiv                                   0x08001155   Thumb Code    20  C:\Keil_v5\ARM\ARMCC\Bin\..\lib\armlib\fz_ps.l(ddiv.o)(.text)
    __aeabi_i2d_normalise                    0x0800116d   Thumb Code    66  C:\Keil_v5\ARM\ARMCC\Bin\..\lib\armlib\fz_ps.l(dflti.o)(.text)
    __aeabi_i2d                              0x080011af   Thumb Code    16  C:\Keil_v5\ARM\ARMCC\Bin\..\lib\armlib\fz_ps.l(dflti.o)(.text)
    _dflt                                    0x080011af   Thumb Code     0  C:\Keil_v5\ARM\ARMCC\Bin\..\lib\armlib\fz_ps.l(dflti.o)(.text)
    __aeabi_ui2d                             0x080011bf   Thumb Code     6  C:\Keil_v5\ARM\ARMCC\Bin\..\lib\armlib\fz_ps.l(dflti.o)(.text)
    _dfltu                                   0x080011bf   Thumb Code     0  C:\Keil_v5\ARM\ARMCC\Bin\..\lib\armlib\fz_ps.l(dflti.o)(.text)
    __aeabi_dmul                             0x080011c5   Thumb Code     0  C:\Keil_v5\ARM\ARMCC\Bin\..\lib\armlib\fz_ps.l(dmul.o)(.text)
    _dmul                                    0x080011c5   Thumb Code   558  C:\Keil_v5\ARM\ARMCC\Bin\..\lib\armlib\fz_ps.l(dmul.o)(.text)
    __aeabi_f2d                              0x0800140d   Thumb Code     0  C:\Keil_v5\ARM\ARMCC\Bin\..\lib\armlib\fz_ps.l(f2d.o)(.text)
    _f2d                                     0x0800140d   Thumb Code    80  C:\Keil_v5\ARM\ARMCC\Bin\..\lib\armlib\fz_ps.l(f2d.o)(.text)
    __aeabi_fdiv                             0x08001461   Thumb Code     0  C:\Keil_v5\ARM\ARMCC\Bin\..\lib\armlib\fz_ps.l(fdiv.o)(.text)
    _fdiv                                    0x08001461   Thumb Code   334  C:\Keil_v5\ARM\ARMCC\Bin\..\lib\armlib\fz_ps.l(fdiv.o)(.text)
    _frdiv                                   0x080015af   Thumb Code     8  C:\Keil_v5\ARM\ARMCC\Bin\..\lib\armlib\fz_ps.l(fdiv.o)(.text)
    __aeabi_i2f_normalise                    0x080015c1   Thumb Code    72  C:\Keil_v5\ARM\ARMCC\Bin\..\lib\armlib\fz_ps.l(fflti.o)(.text)
    __aeabi_i2f                              0x08001609   Thumb Code    16  C:\Keil_v5\ARM\ARMCC\Bin\..\lib\armlib\fz_ps.l(fflti.o)(.text)
    _fflt                                    0x08001609   Thumb Code     0  C:\Keil_v5\ARM\ARMCC\Bin\..\lib\armlib\fz_ps.l(fflti.o)(.text)
    __aeabi_ui2f                             0x08001619   Thumb Code     6  C:\Keil_v5\ARM\ARMCC\Bin\..\lib\armlib\fz_ps.l(fflti.o)(.text)
    _ffltu                                   0x08001619   Thumb Code     0  C:\Keil_v5\ARM\ARMCC\Bin\..\lib\armlib\fz_ps.l(fflti.o)(.text)
    __rt_heap_descriptor                     0x08001621   Thumb Code     8  C:\Keil_v5\ARM\ARMCC\Bin\..\lib\armlib\c_p.l(rt_heap_descriptor.o)(.text)
    __use_no_heap                            0x08001629   Thumb Code     2  C:\Keil_v5\ARM\ARMCC\Bin\..\lib\armlib\c_p.l(hguard.o)(.text)
    __heap$guard                             0x0800162b   Thumb Code     2  C:\Keil_v5\ARM\ARMCC\Bin\..\lib\armlib\c_p.l(hguard.o)(.text)
    _terminate_user_alloc                    0x0800162d   Thumb Code     2  C:\Keil_v5\ARM\ARMCC\Bin\..\lib\armlib\c_p.l(init_alloc.o)(.text)
    _init_user_alloc                         0x0800162f   Thumb Code     2  C:\Keil_v5\ARM\ARMCC\Bin\..\lib\armlib\c_p.l(init_alloc.o)(.text)
    __Heap_Full                              0x08001631   Thumb Code    32  C:\Keil_v5\ARM\ARMCC\Bin\..\lib\armlib\c_p.l(init_alloc.o)(.text)
    __Heap_Broken                            0x08001651   Thumb Code    10  C:\Keil_v5\ARM\ARMCC\Bin\..\lib\armlib\c_p.l(init_alloc.o)(.text)
    _init_alloc                              0x0800165b   Thumb Code    90  C:\Keil_v5\ARM\ARMCC\Bin\..\lib\armlib\c_p.l(init_alloc.o)(.text)
    __Heap_Initialize                        0x080016b5   Thumb Code    10  C:\Keil_v5\ARM\ARMCC\Bin\..\lib\armlib\c_p.l(h1_init.o)(.text)
    __Heap_DescSize                          0x080016bf   Thumb Code     4  C:\Keil_v5\ARM\ARMCC\Bin\..\lib\armlib\c_p.l(h1_init.o)(.text)
    _printf_pre_padding                      0x080016c3   Thumb Code    44  C:\Keil_v5\ARM\ARMCC\Bin\..\lib\armlib\c_p.l(_printf_pad.o)(.text)
    _printf_post_padding                     0x080016ef   Thumb Code    34  C:\Keil_v5\ARM\ARMCC\Bin\..\lib\armlib\c_p.l(_printf_pad.o)(.text)
    _printf_truncate_signed                  0x08001711   Thumb Code    18  C:\Keil_v5\ARM\ARMCC\Bin\..\lib\armlib\c_p.l(_printf_truncate.o)(.text)
    _printf_truncate_unsigned                0x08001723   Thumb Code    18  C:\Keil_v5\ARM\ARMCC\Bin\..\lib\armlib\c_p.l(_printf_truncate.o)(.text)
    _printf_str                              0x08001735   Thumb Code    82  C:\Keil_v5\ARM\ARMCC\Bin\..\lib\armlib\c_p.l(_printf_str.o)(.text)
    _printf_int_common                       0x08001787   Thumb Code   176  C:\Keil_v5\ARM\ARMCC\Bin\..\lib\armlib\c_p.l(_printf_intcommon.o)(.text)
    _printf_int_dec                          0x08001839   Thumb Code    90  C:\Keil_v5\ARM\ARMCC\Bin\..\lib\armlib\c_p.l(_printf_dec.o)(.text)
    _printf_charcount                        0x080018a5   Thumb Code    38  C:\Keil_v5\ARM\ARMCC\Bin\..\lib\armlib\c_p.l(_printf_charcount.o)(.text)
    _printf_char_common                      0x080018d7   Thumb Code    32  C:\Keil_v5\ARM\ARMCC\Bin\..\lib\armlib\c_p.l(_printf_char_common.o)(.text)
    _sputc                                   0x080018fd   Thumb Code    10  C:\Keil_v5\ARM\ARMCC\Bin\..\lib\armlib\c_p.l(_sputc.o)(.text)
    _printf_char_file                        0x08001909   Thumb Code    34  C:\Keil_v5\ARM\ARMCC\Bin\..\lib\armlib\c_p.l(_printf_char_file.o)(.text)
    _printf_wctomb                           0x08001931   Thumb Code   182  C:\Keil_v5\ARM\ARMCC\Bin\..\lib\armlib\c_p.l(_printf_wctomb.o)(.text)
    _printf_longlong_dec                     0x080019ed   Thumb Code    94  C:\Keil_v5\ARM\ARMCC\Bin\..\lib\armlib\c_p.l(_printf_longlong_dec.o)(.text)
    _printf_longlong_oct                     0x08001a5d   Thumb Code    68  C:\Keil_v5\ARM\ARMCC\Bin\..\lib\armlib\c_p.l(_printf_oct_int_ll.o)(.text)
    _printf_int_oct                          0x08001aa1   Thumb Code    24  C:\Keil_v5\ARM\ARMCC\Bin\..\lib\armlib\c_p.l(_printf_oct_int_ll.o)(.text)
    _printf_ll_oct                           0x08001ab9   Thumb Code    10  C:\Keil_v5\ARM\ARMCC\Bin\..\lib\armlib\c_p.l(_printf_oct_int_ll.o)(.text)
    _chval                                   0x08001acd   Thumb Code    30  C:\Keil_v5\ARM\ARMCC\Bin\..\lib\armlib\c_p.l(_chval.o)(.text)
    __vfscanf_char                           0x08001af9   Thumb Code    28  C:\Keil_v5\ARM\ARMCC\Bin\..\lib\armlib\c_p.l(scanf_char.o)(.text)
    _sgetc                                   0x08001b1d   Thumb Code    32  C:\Keil_v5\ARM\ARMCC\Bin\..\lib\armlib\c_p.l(_sgetc.o)(.text)
    _sbackspace                              0x08001b3d   Thumb Code    36  C:\Keil_v5\ARM\ARMCC\Bin\..\lib\armlib\c_p.l(_sgetc.o)(.text)
    ferror                                   0x08001b61   Thumb Code     8  C:\Keil_v5\ARM\ARMCC\Bin\..\lib\armlib\c_p.l(ferror.o)(.text)
    _readbuf                                 0x08001b69   Thumb Code    56  C:\Keil_v5\ARM\ARMCC\Bin\..\lib\armlib\c_p.l(filbuf.o)(.text)
    _seteof                                  0x08001ba1   Thumb Code    40  C:\Keil_v5\ARM\ARMCC\Bin\..\lib\armlib\c_p.l(filbuf.o)(.text)
    __filbuf                                 0x08001bc9   Thumb Code   486  C:\Keil_v5\ARM\ARMCC\Bin\..\lib\armlib\c_p.l(filbuf.o)(.text)
    __filbuf_byte                            0x08001bc9   Thumb Code     0  C:\Keil_v5\ARM\ARMCC\Bin\..\lib\armlib\c_p.l(filbuf.o)(.text)
    __filbuf_wide                            0x08001bc9   Thumb Code     0  C:\Keil_v5\ARM\ARMCC\Bin\..\lib\armlib\c_p.l(filbuf.o)(.text)
    __flsbuf                                 0x08001dbd   Thumb Code   486  C:\Keil_v5\ARM\ARMCC\Bin\..\lib\armlib\c_p.l(flsbuf.o)(.text)
    __flsbuf_byte                            0x08001dbd   Thumb Code     0  C:\Keil_v5\ARM\ARMCC\Bin\..\lib\armlib\c_p.l(flsbuf.o)(.text)
    __flsbuf_wide                            0x08001dbd   Thumb Code     0  C:\Keil_v5\ARM\ARMCC\Bin\..\lib\armlib\c_p.l(flsbuf.o)(.text)
    _fseek                                   0x08001fad   Thumb Code   240  C:\Keil_v5\ARM\ARMCC\Bin\..\lib\armlib\c_p.l(fseek.o)(.text)
    fseek                                    0x08001fad   Thumb Code     0  C:\Keil_v5\ARM\ARMCC\Bin\..\lib\armlib\c_p.l(fseek.o)(.text)
    setvbuf                                  0x080020a1   Thumb Code    72  C:\Keil_v5\ARM\ARMCC\Bin\..\lib\armlib\c_p.l(setvbuf.o)(.text)
    _seterr                                  0x080020ed   Thumb Code    20  C:\Keil_v5\ARM\ARMCC\Bin\..\lib\armlib\c_p.l(stdio.o)(.text)
    _writebuf                                0x08002101   Thumb Code    76  C:\Keil_v5\ARM\ARMCC\Bin\..\lib\armlib\c_p.l(stdio.o)(.text)
    _fflush                                  0x0800214d   Thumb Code    76  C:\Keil_v5\ARM\ARMCC\Bin\..\lib\armlib\c_p.l(stdio.o)(.text)
    _deferredlazyseek                        0x08002199   Thumb Code    60  C:\Keil_v5\ARM\ARMCC\Bin\..\lib\armlib\c_p.l(stdio.o)(.text)
    _initio                                  0x080021dd   Thumb Code   216  C:\Keil_v5\ARM\ARMCC\Bin\..\lib\armlib\c_p.l(initio.o)(.text)
    _terminateio                             0x080022b5   Thumb Code    56  C:\Keil_v5\ARM\ARMCC\Bin\..\lib\armlib\c_p.l(initio.o)(.text)
    __rt_SIGPVFN                             0x08002319   Thumb Code    12  C:\Keil_v5\ARM\ARMCC\Bin\..\lib\armlib\c_p.l(defsig_pvfn_outer.o)(.text)
    __Heap_ProvideMemory                     0x08002325   Thumb Code    52  C:\Keil_v5\ARM\ARMCC\Bin\..\lib\armlib\c_p.l(h1_extend.o)(.text)
    _ll_udiv10                               0x08002359   Thumb Code   122  C:\Keil_v5\ARM\ARMCC\Bin\..\lib\armlib\c_p.l(lludiv10.o)(.text)
    isspace                                  0x080023d3   Thumb Code    18  C:\Keil_v5\ARM\ARMCC\Bin\..\lib\armlib\c_p.l(isspace.o)(.text)
    __lib_sel_fp_printf                      0x080023e5   Thumb Code     2  C:\Keil_v5\ARM\ARMCC\Bin\..\lib\armlib\c_p.l(_printf_fp_dec.o)(.text)
    _printf_fp_dec_real                      0x08002583   Thumb Code   620  C:\Keil_v5\ARM\ARMCC\Bin\..\lib\armlib\c_p.l(_printf_fp_dec.o)(.text)
    _printf_fp_hex_real                      0x080027fd   Thumb Code   718  C:\Keil_v5\ARM\ARMCC\Bin\..\lib\armlib\c_p.l(_printf_fp_hex.o)(.text)
    _printf_cs_common                        0x08002ad5   Thumb Code    22  C:\Keil_v5\ARM\ARMCC\Bin\..\lib\armlib\c_p.l(_printf_char.o)(.text)
    _printf_char                             0x08002aeb   Thumb Code    16  C:\Keil_v5\ARM\ARMCC\Bin\..\lib\armlib\c_p.l(_printf_char.o)(.text)
    _printf_string                           0x08002afb   Thumb Code     8  C:\Keil_v5\ARM\ARMCC\Bin\..\lib\armlib\c_p.l(_printf_char.o)(.text)
    _printf_lcs_common                       0x08002b03   Thumb Code    22  C:\Keil_v5\ARM\ARMCC\Bin\..\lib\armlib\c_p.l(_printf_wchar.o)(.text)
    _printf_wchar                            0x08002b19   Thumb Code    16  C:\Keil_v5\ARM\ARMCC\Bin\..\lib\armlib\c_p.l(_printf_wchar.o)(.text)
    _printf_wstring                          0x08002b29   Thumb Code     8  C:\Keil_v5\ARM\ARMCC\Bin\..\lib\armlib\c_p.l(_printf_wchar.o)(.text)
    __vfscanf                                0x08002b31   Thumb Code   880  C:\Keil_v5\ARM\ARMCC\Bin\..\lib\armlib\c_p.l(_scanf.o)(.text)
    _ftell_internal                          0x08002eb1   Thumb Code    66  C:\Keil_v5\ARM\ARMCC\Bin\..\lib\armlib\c_p.l(ftell.o)(.text)
    ftell                                    0x08002eb1   Thumb Code     0  C:\Keil_v5\ARM\ARMCC\Bin\..\lib\armlib\c_p.l(ftell.o)(.text)
    _flushlinebuffered                       0x08002ef5   Thumb Code    46  C:\Keil_v5\ARM\ARMCC\Bin\..\lib\armlib\c_p.l(flushlinebuffered.o)(.text)
    _wcrtomb                                 0x08002f2d   Thumb Code    64  C:\Keil_v5\ARM\ARMCC\Bin\..\lib\armlib\c_p.l(_wcrtomb.o)(.text)
    __sig_exit                               0x08002f6d   Thumb Code    12  C:\Keil_v5\ARM\ARMCC\Bin\..\lib\armlib\c_p.l(defsig_exit.o)(.text)
    __rt_SIGRTRED                            0x08002f79   Thumb Code    12  C:\Keil_v5\ARM\ARMCC\Bin\..\lib\armlib\c_p.l(defsig_rtred_outer.o)(.text)
    __rt_SIGRTMEM                            0x08002f85   Thumb Code    12  C:\Keil_v5\ARM\ARMCC\Bin\..\lib\armlib\c_p.l(defsig_rtmem_outer.o)(.text)
    __rt_SIGPVFN_inner                       0x08002f91   Thumb Code    14  C:\Keil_v5\ARM\ARMCC\Bin\..\lib\armlib\c_p.l(defsig_pvfn_inner.o)(.text)
    __rt_udiv10                              0x08002fc1   Thumb Code    40  C:\Keil_v5\ARM\ARMCC\Bin\..\lib\armlib\c_p.l(rtudiv10.o)(.text)
    __rt_heap_escrow                         0x08002fe9   Thumb Code    24  C:\Keil_v5\ARM\ARMCC\Bin\..\lib\armlib\c_p.l(heapauxa.o)(.text)
    __rt_heap_expand                         0x08003001   Thumb Code    52  C:\Keil_v5\ARM\ARMCC\Bin\..\lib\armlib\c_p.l(heapauxa.o)(.text)
    _sys_exit                                0x08003039   Thumb Code     8  C:\Keil_v5\ARM\ARMCC\Bin\..\lib\armlib\c_p.l(sys_exit.o)(.text)
    __rt_ctype_table                         0x08003045   Thumb Code    16  C:\Keil_v5\ARM\ARMCC\Bin\..\lib\armlib\c_p.l(rt_ctype_table.o)(.text)
    __rt_locale                              0x08003055   Thumb Code     8  C:\Keil_v5\ARM\ARMCC\Bin\..\lib\armlib\c_p.l(rt_locale.o)(.text)
    __aeabi_errno_addr                       0x0800305d   Thumb Code     8  C:\Keil_v5\ARM\ARMCC\Bin\..\lib\armlib\c_p.l(rt_errno_addr.o)(.text)
    __errno                                  0x0800305d   Thumb Code     0  C:\Keil_v5\ARM\ARMCC\Bin\..\lib\armlib\c_p.l(rt_errno_addr.o)(.text)
    __rt_errno_addr                          0x0800305d   Thumb Code     0  C:\Keil_v5\ARM\ARMCC\Bin\..\lib\armlib\c_p.l(rt_errno_addr.o)(.text)
